Product: MDK-ARM Professional 5.10
Component: ARM Compiler 5.04 update 1 (build 49)
Tool: armlink [5040049]

==============================================================================

Section Cross References

    startup_stm32l053xx.o(RESET) refers to startup_stm32l053xx.o(STACK) for __initial_sp
    startup_stm32l053xx.o(RESET) refers to startup_stm32l053xx.o(.text) for Reset_Handler
    startup_stm32l053xx.o(RESET) refers to stm32l0xx_it.o(i.NMI_Handler) for NMI_Handler
    startup_stm32l053xx.o(RESET) refers to stm32l0xx_it.o(i.HardFault_Handler) for HardFault_Handler
    startup_stm32l053xx.o(RESET) refers to stm32l0xx_it.o(i.SVC_Handler) for SVC_Handler
    startup_stm32l053xx.o(RESET) refers to stm32l0xx_it.o(i.DebugMon_Handler) for DebugMon_Handler
    startup_stm32l053xx.o(RESET) refers to stm32l0xx_it.o(i.PendSV_Handler) for PendSV_Handler
    startup_stm32l053xx.o(RESET) refers to stm32l0xx_it.o(i.SysTick_Handler) for SysTick_Handler
    startup_stm32l053xx.o(RESET) refers to stm32l0xx_it.o(i.EXTI0_1_IRQHandler) for EXTI0_1_IRQHandler
    startup_stm32l053xx.o(RESET) refers to stm32l0xx_it.o(i.EXTI4_15_IRQHandler) for EXTI4_15_IRQHandler
    startup_stm32l053xx.o(RESET) refers to stm32l0xx_it.o(i.USB_IRQHandler) for USB_IRQHandler
    startup_stm32l053xx.o(.text) refers to system_stm32l0xx.o(i.SystemInit) for SystemInit
    startup_stm32l053xx.o(.text) refers to entry.o(.ARM.Collect$$$$00000000) for __main
    bsp.o(i.BSP_TSL_Init) refers to stm32l0xx_hal_tsc.o(i.HAL_TSC_Init) for HAL_TSC_Init
    bsp.o(i.BSP_TSL_Init) refers to tsl_user.o(i.tsl_user_Init) for tsl_user_Init
    bsp.o(i.BSP_TSL_Init) refers to bsp.o(.bss) for .bss
    bsp.o(i.BSP_USB_Init) refers to usbd_core.o(i.USBD_Init) for USBD_Init
    bsp.o(i.BSP_USB_Init) refers to usbd_core.o(i.USBD_RegisterClass) for USBD_RegisterClass
    bsp.o(i.BSP_USB_Init) refers to usbd_core.o(i.USBD_Start) for USBD_Start
    bsp.o(i.BSP_USB_Init) refers to usbd_desc.o(.data) for HID_Desc
    bsp.o(i.BSP_USB_Init) refers to bsp.o(.bss) for .bss
    bsp.o(i.BSP_USB_Init) refers to usbd_hid.o(.data) for USBD_HID
    bsp.o(i.Bsp_Init) refers to stm32l0538_discovery.o(i.BSP_LED_Init) for BSP_LED_Init
    bsp.o(i.Bsp_Init) refers to stm32l0538_discovery.o(i.BSP_PB_Init) for BSP_PB_Init
    bsp.o(i.Bsp_Init) refers to stm32l0538_discovery_epd.o(i.BSP_EPD_Init) for BSP_EPD_Init
    bsp.o(i.Bsp_Init) refers to bsp.o(i.BSP_TSL_Init) for BSP_TSL_Init
    main.o(i.main) refers to stm32l0xx_hal.o(i.HAL_Init) for HAL_Init
    main.o(i.main) refers to menu.o(i.SystemClock_Config) for SystemClock_Config
    main.o(i.main) refers to bsp.o(i.Bsp_Init) for Bsp_Init
    main.o(i.main) refers to menu.o(i.Menu_Process) for Menu_Process
    menu.o(i.HAL_GPIO_EXTI_Callback) refers to menu.o(.data) for .data
    menu.o(i.IDD_RestoreContext) refers to stm32l0538_discovery.o(i.BSP_PB_Init) for BSP_PB_Init
    menu.o(i.IDD_RestoreContext) refers to bsp.o(i.BSP_TSL_Init) for BSP_TSL_Init
    menu.o(i.IDD_RestoreContext) refers to stm32l0538_discovery_epd.o(i.BSP_EPD_Init) for BSP_EPD_Init
    menu.o(i.IDD_RestoreContext) refers to menu.o(.data) for .data
    menu.o(i.IDD_SaveContext) refers to stm32l0xx_hal_gpio.o(i.HAL_GPIO_Init) for HAL_GPIO_Init
    menu.o(i.IDD_SaveContext) refers to stm32l0xx_hal_tsc.o(i.HAL_TSC_DeInit) for HAL_TSC_DeInit
    menu.o(i.IDD_SaveContext) refers to menu.o(.data) for .data
    menu.o(i.IDD_SaveContext) refers to bsp.o(.bss) for TscHandle
    menu.o(i.Menu_Process) refers to menu.o(i.__ARM_common_switch8) for __ARM_common_switch8
    menu.o(i.Menu_Process) refers to stm32l0538_discovery_epd.o(i.BSP_EPD_SetFont) for BSP_EPD_SetFont
    menu.o(i.Menu_Process) refers to stm32l0538_discovery_epd.o(i.BSP_EPD_DrawImage) for BSP_EPD_DrawImage
    menu.o(i.Menu_Process) refers to stm32l0538_discovery_epd.o(i.BSP_EPD_DisplayStringAt) for BSP_EPD_DisplayStringAt
    menu.o(i.Menu_Process) refers to stm32l0538_discovery_epd.o(i.BSP_EPD_RefreshDisplay) for BSP_EPD_RefreshDisplay
    menu.o(i.Menu_Process) refers to stm32l0xx_hal.o(i.HAL_Delay) for HAL_Delay
    menu.o(i.Menu_Process) refers to stm32l0538_discovery_epd.o(i.BSP_EPD_Clear) for BSP_EPD_Clear
    menu.o(i.Menu_Process) refers to tsl_user.o(i.tsl_user_Exec) for tsl_user_Exec
    menu.o(i.Menu_Process) refers to stm32l0538_discovery_epd.o(i.BSP_EPD_DrawRect) for BSP_EPD_DrawRect
    menu.o(i.Menu_Process) refers to menu.o(i.USBClock_Enable) for USBClock_Enable
    menu.o(i.Menu_Process) refers to bsp.o(i.BSP_USB_Init) for BSP_USB_Init
    menu.o(i.Menu_Process) refers to usbdapp.o(i.USB_process) for USB_process
    menu.o(i.Menu_Process) refers to menu.o(i.USBClock_Disable) for USBClock_Disable
    menu.o(i.Menu_Process) refers to usbd_core.o(i.USBD_DeInit) for USBD_DeInit
    menu.o(i.Menu_Process) refers to stm32l0538_discovery.o(i.BSP_LED_Off) for BSP_LED_Off
    menu.o(i.Menu_Process) refers to power.o(i.Idd_Run_process) for Idd_Run_process
    menu.o(i.Menu_Process) refers to power.o(i.Idd_Sleep_process) for Idd_Sleep_process
    menu.o(i.Menu_Process) refers to power.o(i.Idd_LPSleep_process) for Idd_LPSleep_process
    menu.o(i.Menu_Process) refers to menu.o(.data) for .data
    menu.o(i.Menu_Process) refers to tsl_user.o(.constdata) for MyLinRots
    menu.o(i.Menu_Process) refers to stm32l0538_discovery_epd.o(.data) for Font16
    menu.o(i.Menu_Process) refers to stm32l0538_discovery_epd.o(.data) for Font8
    menu.o(i.Menu_Process) refers to bsp.o(.bss) for USBD_Device
    menu.o(i.Menu_Process) refers to power.o(.bss) for str
    menu.o(i.SystemClock_Config) refers to stm32l0xx_hal_rcc.o(i.HAL_RCC_OscConfig) for HAL_RCC_OscConfig
    menu.o(i.SystemClock_Config) refers to stm32l0xx_hal_rcc.o(i.HAL_RCC_ClockConfig) for HAL_RCC_ClockConfig
    menu.o(i.USBClock_Disable) refers to stm32l0xx_hal_rcc.o(i.HAL_RCC_OscConfig) for HAL_RCC_OscConfig
    menu.o(i.USBClock_Enable) refers to stm32l0xx_hal_rcc.o(i.HAL_RCC_OscConfig) for HAL_RCC_OscConfig
    menu.o(i.USBClock_Enable) refers to stm32l0xx_hal_rcc_ex.o(i.HAL_RCCEx_PeriphCLKConfig) for HAL_RCCEx_PeriphCLKConfig
    menu.o(i.USBClock_Enable) refers to stm32l0xx_hal_rcc_ex.o(i.HAL_RCCEx_CRSConfig) for HAL_RCCEx_CRSConfig
    menu.o(i.USBClock_Enable) refers to menu.o(.bss) for .bss
    stm32l0xx_hal_msp.o(i.HAL_I2C_MspDeInit) refers to stm32l0xx_hal_gpio.o(i.HAL_GPIO_DeInit) for HAL_GPIO_DeInit
    stm32l0xx_hal_msp.o(i.HAL_I2C_MspDeInit) refers to stm32l0xx_hal_cortex.o(i.HAL_NVIC_DisableIRQ) for HAL_NVIC_DisableIRQ
    stm32l0xx_hal_msp.o(i.HAL_I2C_MspInit) refers to stm32l0xx_hal_gpio.o(i.HAL_GPIO_Init) for HAL_GPIO_Init
    stm32l0xx_hal_msp.o(i.HAL_I2C_MspInit) refers to stm32l0xx_hal_cortex.o(i.HAL_NVIC_SetPriority) for HAL_NVIC_SetPriority
    stm32l0xx_hal_msp.o(i.HAL_I2C_MspInit) refers to stm32l0xx_hal_cortex.o(i.HAL_NVIC_EnableIRQ) for HAL_NVIC_EnableIRQ
    stm32l0xx_hal_msp.o(i.HAL_TSC_MspDeInit) refers to stm32l0xx_hal_gpio.o(i.HAL_GPIO_DeInit) for HAL_GPIO_DeInit
    stm32l0xx_hal_msp.o(i.HAL_TSC_MspInit) refers to stm32l0xx_hal_gpio.o(i.HAL_GPIO_Init) for HAL_GPIO_Init
    stm32l0xx_it.o(i.EXTI0_1_IRQHandler) refers to stm32l0xx_hal_gpio.o(i.HAL_GPIO_EXTI_IRQHandler) for HAL_GPIO_EXTI_IRQHandler
    stm32l0xx_it.o(i.EXTI4_15_IRQHandler) refers to stm32l0xx_hal_gpio.o(i.HAL_GPIO_EXTI_IRQHandler) for HAL_GPIO_EXTI_IRQHandler
    stm32l0xx_it.o(i.SysTick_Handler) refers to stm32l0xx_hal.o(i.HAL_IncTick) for HAL_IncTick
    stm32l0xx_it.o(i.SysTick_Handler) refers to stm32l0538_discovery.o(i.BSP_LED_Toggle) for BSP_LED_Toggle
    stm32l0xx_it.o(i.SysTick_Handler) refers to power.o(.data) for RunModeMeasure
    stm32l0xx_it.o(i.SysTick_Handler) refers to stm32l0xx_it.o(.data) for .data
    stm32l0xx_it.o(i.USB_IRQHandler) refers to stm32l0xx_hal_pcd.o(i.HAL_PCD_IRQHandler) for HAL_PCD_IRQHandler
    stm32l0xx_it.o(i.USB_IRQHandler) refers to usbd_conf.o(.bss) for hpcd
    tsl_user.o(i.tsl_user_Exec) refers to tsl_acq_tsc.o(i.TSL_acq_BankConfig) for TSL_acq_BankConfig
    tsl_user.o(i.tsl_user_Exec) refers to tsl_acq_tsc.o(i.TSL_acq_BankStartAcq) for TSL_acq_BankStartAcq
    tsl_user.o(i.tsl_user_Exec) refers to tsl_acq_tsc.o(i.TSL_acq_BankWaitEOC) for TSL_acq_BankWaitEOC
    tsl_user.o(i.tsl_user_Exec) refers to tsl_acq.o(i.TSL_acq_BankGetResult) for TSL_acq_BankGetResult
    tsl_user.o(i.tsl_user_Exec) refers to tsl_object.o(i.TSL_obj_GroupProcess) for TSL_obj_GroupProcess
    tsl_user.o(i.tsl_user_Exec) refers to tsl_dxs.o(i.TSL_dxs_FirstObj) for TSL_dxs_FirstObj
    tsl_user.o(i.tsl_user_Exec) refers to tsl_time.o(i.TSL_tim_CheckDelay_ms) for TSL_tim_CheckDelay_ms
    tsl_user.o(i.tsl_user_Exec) refers to tsl_ecs.o(i.TSL_ecs_Process) for TSL_ecs_Process
    tsl_user.o(i.tsl_user_Exec) refers to tsl_user.o(.data) for .data
    tsl_user.o(i.tsl_user_Init) refers to tsl_object.o(i.TSL_obj_GroupInit) for TSL_obj_GroupInit
    tsl_user.o(i.tsl_user_Init) refers to tsl.o(i.TSL_Init) for TSL_Init
    tsl_user.o(i.tsl_user_Init) refers to tsl_user.o(.data) for .data
    tsl_user.o(i.tsl_user_Init) refers to tsl_user.o(.constdata) for .constdata
    tsl_user.o(.constdata) refers to tsl_user.o(.constdata) for MyChannels_Src
    tsl_user.o(.constdata) refers to tsl_user.o(.constdata) for MyChannels_Dest
    tsl_user.o(.constdata) refers to tsl_user.o(.bss) for MyChannels_Data
    tsl_user.o(.constdata) refers to tsl_linrot.o(i.TSL_linrot_CalibrationStateProcess) for TSL_linrot_CalibrationStateProcess
    tsl_user.o(.constdata) refers to tsl_linrot.o(i.TSL_linrot_DebCalibrationStateProcess) for TSL_linrot_DebCalibrationStateProcess
    tsl_user.o(.constdata) refers to tsl_linrot.o(i.TSL_linrot_ReleaseStateProcess) for TSL_linrot_ReleaseStateProcess
    tsl_user.o(.constdata) refers to tsl_linrot.o(i.TSL_linrot_DebReleaseProxStateProcess) for TSL_linrot_DebReleaseProxStateProcess
    tsl_user.o(.constdata) refers to tsl_linrot.o(i.TSL_linrot_DebReleaseDetectStateProcess) for TSL_linrot_DebReleaseDetectStateProcess
    tsl_user.o(.constdata) refers to tsl_linrot.o(i.TSL_linrot_DebReleaseTouchStateProcess) for TSL_linrot_DebReleaseTouchStateProcess
    tsl_user.o(.constdata) refers to tsl_linrot.o(i.TSL_linrot_ProxStateProcess) for TSL_linrot_ProxStateProcess
    tsl_user.o(.constdata) refers to tsl_linrot.o(i.TSL_linrot_DebProxStateProcess) for TSL_linrot_DebProxStateProcess
    tsl_user.o(.constdata) refers to tsl_linrot.o(i.TSL_linrot_DebProxDetectStateProcess) for TSL_linrot_DebProxDetectStateProcess
    tsl_user.o(.constdata) refers to tsl_linrot.o(i.TSL_linrot_DebProxTouchStateProcess) for TSL_linrot_DebProxTouchStateProcess
    tsl_user.o(.constdata) refers to tsl_linrot.o(i.TSL_linrot_DetectStateProcess) for TSL_linrot_DetectStateProcess
    tsl_user.o(.constdata) refers to tsl_linrot.o(i.TSL_linrot_DebDetectStateProcess) for TSL_linrot_DebDetectStateProcess
    tsl_user.o(.constdata) refers to tsl_linrot.o(i.TSL_linrot_TouchStateProcess) for TSL_linrot_TouchStateProcess
    tsl_user.o(.constdata) refers to tsl_user.o(i.MyLinRots_ErrorStateProcess) for MyLinRots_ErrorStateProcess
    tsl_user.o(.constdata) refers to tsl_linrot.o(i.TSL_linrot_DebErrorStateProcess) for TSL_linrot_DebErrorStateProcess
    tsl_user.o(.constdata) refers to tsl_user.o(i.MyLinRots_OffStateProcess) for MyLinRots_OffStateProcess
    tsl_user.o(.constdata) refers to tsl_linrot.o(i.TSL_linrot_Init) for TSL_linrot_Init
    tsl_user.o(.constdata) refers to tsl_linrot.o(i.TSL_linrot_Process) for TSL_linrot_Process
    tsl_user.o(.constdata) refers to tsl_linrot.o(i.TSL_linrot_CalcPos) for TSL_linrot_CalcPos
    tsl_user.o(.constdata) refers to tsl_user.o(.data) for MyLinRots_Data
    tsl_user.o(.constdata) refers to tsl_user.o(.bss) for MyLinRots_Param
    tsl_user.o(.constdata) refers to tsl_user.o(.bss) for MyChannels_Data
    tsl_user.o(.constdata) refers to tsl_user.o(.constdata) for MyLinRot0_DeltaCoeff
    tsl_user.o(.constdata) refers to tsl_linrot.o(.constdata) for TSL_POSOFF_3CH_LIN_H
    tsl_user.o(.constdata) refers to tsl_user.o(.constdata) for MyLinRots_StateMachine
    tsl_user.o(.constdata) refers to tsl_user.o(.constdata) for MyLinRots_Methods
    tsl_user.o(.constdata) refers to tsl_user.o(.constdata) for MyLinRots
    tsl_user.o(.data) refers to tsl_user.o(.constdata) for MyObjects
    tsl_user.o(.data) refers to tsl_user.o(.constdata) for MyLinRots_StateMachine
    tsl_user.o(.data) refers to tsl_user.o(.constdata) for MyLinRots_Methods
    power.o(i.I2C_Config) refers to stm32l0xx_hal_i2c.o(i.HAL_I2C_DeInit) for HAL_I2C_DeInit
    power.o(i.I2C_Config) refers to stm32l0xx_hal_i2c.o(i.HAL_I2C_Init) for HAL_I2C_Init
    power.o(i.I2C_Config) refers to power.o(.bss) for .bss
    power.o(i.Idd_LPSleep_process) refers to menu.o(i.IDD_SaveContext) for IDD_SaveContext
    power.o(i.Idd_LPSleep_process) refers to power.o(i.I2C_Config) for I2C_Config
    power.o(i.Idd_LPSleep_process) refers to stm32l0xx_hal_i2c.o(i.HAL_I2C_Mem_Write) for HAL_I2C_Mem_Write
    power.o(i.Idd_LPSleep_process) refers to stm32l0xx_hal.o(i.HAL_Delay) for HAL_Delay
    power.o(i.Idd_LPSleep_process) refers to stm32l0xx_hal_rcc.o(i.HAL_RCC_OscConfig) for HAL_RCC_OscConfig
    power.o(i.Idd_LPSleep_process) refers to stm32l0xx_hal_rcc.o(i.HAL_RCC_ClockConfig) for HAL_RCC_ClockConfig
    power.o(i.Idd_LPSleep_process) refers to stm32l0xx_hal_pwr_ex.o(i.HAL_PWREx_EnableUltraLowPower) for HAL_PWREx_EnableUltraLowPower
    power.o(i.Idd_LPSleep_process) refers to stm32l0xx_hal_pwr_ex.o(i.HAL_PWREx_EnableFastWakeUp) for HAL_PWREx_EnableFastWakeUp
    power.o(i.Idd_LPSleep_process) refers to stm32l0xx_hal_i2c.o(i.HAL_I2C_DeInit) for HAL_I2C_DeInit
    power.o(i.Idd_LPSleep_process) refers to stm32l0xx_hal_gpio.o(i.HAL_GPIO_Init) for HAL_GPIO_Init
    power.o(i.Idd_LPSleep_process) refers to stm32l0xx_hal_cortex.o(i.HAL_NVIC_SetPriority) for HAL_NVIC_SetPriority
    power.o(i.Idd_LPSleep_process) refers to stm32l0xx_hal_cortex.o(i.HAL_NVIC_EnableIRQ) for HAL_NVIC_EnableIRQ
    power.o(i.Idd_LPSleep_process) refers to stm32l0xx_hal.o(i.HAL_SuspendTick) for HAL_SuspendTick
    power.o(i.Idd_LPSleep_process) refers to stm32l0xx_hal_pwr.o(i.HAL_PWR_EnterSLEEPMode) for HAL_PWR_EnterSLEEPMode
    power.o(i.Idd_LPSleep_process) refers to stm32l0xx_hal.o(i.HAL_ResumeTick) for HAL_ResumeTick
    power.o(i.Idd_LPSleep_process) refers to menu.o(i.SystemClock_Config) for SystemClock_Config
    power.o(i.Idd_LPSleep_process) refers to menu.o(i.IDD_RestoreContext) for IDD_RestoreContext
    power.o(i.Idd_LPSleep_process) refers to stm32l0xx_hal_i2c.o(i.HAL_I2C_Mem_Read) for HAL_I2C_Mem_Read
    power.o(i.Idd_LPSleep_process) refers to idiv.o(.text) for __aeabi_idivmod
    power.o(i.Idd_LPSleep_process) refers to printf1.o(i.__0sprintf$1) for __2sprintf
    power.o(i.Idd_LPSleep_process) refers to power.o(.bss) for .bss
    power.o(i.Idd_LPSleep_process) refers to power.o(.data) for .data
    power.o(i.Idd_Run_process) refers to power.o(i.I2C_Config) for I2C_Config
    power.o(i.Idd_Run_process) refers to stm32l0xx_hal_i2c.o(i.HAL_I2C_Mem_Write) for HAL_I2C_Mem_Write
    power.o(i.Idd_Run_process) refers to stm32l0xx_hal.o(i.HAL_Delay) for HAL_Delay
    power.o(i.Idd_Run_process) refers to stm32l0538_discovery.o(i.BSP_LED_Off) for BSP_LED_Off
    power.o(i.Idd_Run_process) refers to stm32l0xx_hal_i2c.o(i.HAL_I2C_Mem_Read) for HAL_I2C_Mem_Read
    power.o(i.Idd_Run_process) refers to idiv.o(.text) for __aeabi_idivmod
    power.o(i.Idd_Run_process) refers to printf1.o(i.__0sprintf$1) for __2sprintf
    power.o(i.Idd_Run_process) refers to power.o(.bss) for .bss
    power.o(i.Idd_Run_process) refers to power.o(.data) for .data
    power.o(i.Idd_Sleep_process) refers to power.o(i.I2C_Config) for I2C_Config
    power.o(i.Idd_Sleep_process) refers to stm32l0xx_hal_i2c.o(i.HAL_I2C_Mem_Write) for HAL_I2C_Mem_Write
    power.o(i.Idd_Sleep_process) refers to stm32l0xx_hal.o(i.HAL_Delay) for HAL_Delay
    power.o(i.Idd_Sleep_process) refers to menu.o(i.IDD_SaveContext) for IDD_SaveContext
    power.o(i.Idd_Sleep_process) refers to stm32l0xx_hal_i2c.o(i.HAL_I2C_DeInit) for HAL_I2C_DeInit
    power.o(i.Idd_Sleep_process) refers to stm32l0xx_hal_gpio.o(i.HAL_GPIO_Init) for HAL_GPIO_Init
    power.o(i.Idd_Sleep_process) refers to stm32l0xx_hal_cortex.o(i.HAL_NVIC_SetPriority) for HAL_NVIC_SetPriority
    power.o(i.Idd_Sleep_process) refers to stm32l0xx_hal_cortex.o(i.HAL_NVIC_EnableIRQ) for HAL_NVIC_EnableIRQ
    power.o(i.Idd_Sleep_process) refers to stm32l0xx_hal.o(i.HAL_SuspendTick) for HAL_SuspendTick
    power.o(i.Idd_Sleep_process) refers to stm32l0xx_hal_pwr.o(i.HAL_PWR_EnterSLEEPMode) for HAL_PWR_EnterSLEEPMode
    power.o(i.Idd_Sleep_process) refers to stm32l0xx_hal.o(i.HAL_ResumeTick) for HAL_ResumeTick
    power.o(i.Idd_Sleep_process) refers to menu.o(i.IDD_RestoreContext) for IDD_RestoreContext
    power.o(i.Idd_Sleep_process) refers to stm32l0xx_hal_i2c.o(i.HAL_I2C_Mem_Read) for HAL_I2C_Mem_Read
    power.o(i.Idd_Sleep_process) refers to idiv.o(.text) for __aeabi_idivmod
    power.o(i.Idd_Sleep_process) refers to printf1.o(i.__0sprintf$1) for __2sprintf
    power.o(i.Idd_Sleep_process) refers to power.o(.bss) for .bss
    power.o(i.Idd_Sleep_process) refers to power.o(.data) for .data
    power.o(i.Idd_Stop_process) refers to power.o(i.I2C_Config) for I2C_Config
    power.o(i.Idd_Stop_process) refers to stm32l0xx_hal_i2c.o(i.HAL_I2C_Mem_Write) for HAL_I2C_Mem_Write
    power.o(i.Idd_Stop_process) refers to stm32l0xx_hal.o(i.HAL_Delay) for HAL_Delay
    power.o(i.Idd_Stop_process) refers to menu.o(i.IDD_SaveContext) for IDD_SaveContext
    power.o(i.Idd_Stop_process) refers to stm32l0xx_hal_i2c.o(i.HAL_I2C_DeInit) for HAL_I2C_DeInit
    power.o(i.Idd_Stop_process) refers to stm32l0xx_hal_gpio.o(i.HAL_GPIO_Init) for HAL_GPIO_Init
    power.o(i.Idd_Stop_process) refers to stm32l0xx_hal_cortex.o(i.HAL_NVIC_SetPriority) for HAL_NVIC_SetPriority
    power.o(i.Idd_Stop_process) refers to stm32l0xx_hal_cortex.o(i.HAL_NVIC_EnableIRQ) for HAL_NVIC_EnableIRQ
    power.o(i.Idd_Stop_process) refers to stm32l0xx_hal_pwr_ex.o(i.HAL_PWREx_EnableUltraLowPower) for HAL_PWREx_EnableUltraLowPower
    power.o(i.Idd_Stop_process) refers to stm32l0xx_hal_pwr_ex.o(i.HAL_PWREx_EnableFastWakeUp) for HAL_PWREx_EnableFastWakeUp
    power.o(i.Idd_Stop_process) refers to stm32l0xx_hal_pwr.o(i.HAL_PWR_EnterSTOPMode) for HAL_PWR_EnterSTOPMode
    power.o(i.Idd_Stop_process) refers to menu.o(i.IDD_RestoreContext) for IDD_RestoreContext
    power.o(i.Idd_Stop_process) refers to stm32l0xx_hal_i2c.o(i.HAL_I2C_Mem_Read) for HAL_I2C_Mem_Read
    power.o(i.Idd_Stop_process) refers to printf1.o(i.__0sprintf$1) for __2sprintf
    power.o(i.Idd_Stop_process) refers to power.o(.bss) for .bss
    power.o(i.Idd_Stop_process) refers to power.o(.data) for .data
    usbd_conf.o(i.HAL_PCD_ConnectCallback) refers to usbd_core.o(i.USBD_LL_DevConnected) for USBD_LL_DevConnected
    usbd_conf.o(i.HAL_PCD_DataInStageCallback) refers to usbd_core.o(i.USBD_LL_DataInStage) for USBD_LL_DataInStage
    usbd_conf.o(i.HAL_PCD_DataOutStageCallback) refers to usbd_core.o(i.USBD_LL_DataOutStage) for USBD_LL_DataOutStage
    usbd_conf.o(i.HAL_PCD_DisconnectCallback) refers to usbd_core.o(i.USBD_LL_DevDisconnected) for USBD_LL_DevDisconnected
    usbd_conf.o(i.HAL_PCD_ISOINIncompleteCallback) refers to usbd_core.o(i.USBD_LL_IsoINIncomplete) for USBD_LL_IsoINIncomplete
    usbd_conf.o(i.HAL_PCD_ISOOUTIncompleteCallback) refers to usbd_core.o(i.USBD_LL_IsoOUTIncomplete) for USBD_LL_IsoOUTIncomplete
    usbd_conf.o(i.HAL_PCD_MspDeInit) refers to stm32l0xx_hal_gpio.o(i.HAL_GPIO_DeInit) for HAL_GPIO_DeInit
    usbd_conf.o(i.HAL_PCD_MspDeInit) refers to stm32l0xx_hal_cortex.o(i.HAL_NVIC_DisableIRQ) for HAL_NVIC_DisableIRQ
    usbd_conf.o(i.HAL_PCD_MspInit) refers to stm32l0xx_hal_gpio.o(i.HAL_GPIO_Init) for HAL_GPIO_Init
    usbd_conf.o(i.HAL_PCD_MspInit) refers to stm32l0xx_hal_cortex.o(i.HAL_NVIC_SetPriority) for HAL_NVIC_SetPriority
    usbd_conf.o(i.HAL_PCD_MspInit) refers to stm32l0xx_hal_cortex.o(i.HAL_NVIC_EnableIRQ) for HAL_NVIC_EnableIRQ
    usbd_conf.o(i.HAL_PCD_ResetCallback) refers to usbd_core.o(i.USBD_LL_SetSpeed) for USBD_LL_SetSpeed
    usbd_conf.o(i.HAL_PCD_ResetCallback) refers to usbd_core.o(i.USBD_LL_Reset) for USBD_LL_Reset
    usbd_conf.o(i.HAL_PCD_SOFCallback) refers to usbd_core.o(i.USBD_LL_SOF) for USBD_LL_SOF
    usbd_conf.o(i.HAL_PCD_SetupStageCallback) refers to usbd_core.o(i.USBD_LL_SetupStage) for USBD_LL_SetupStage
    usbd_conf.o(i.USBD_LL_ClearStallEP) refers to stm32l0xx_hal_pcd.o(i.HAL_PCD_EP_ClrStall) for HAL_PCD_EP_ClrStall
    usbd_conf.o(i.USBD_LL_CloseEP) refers to stm32l0xx_hal_pcd.o(i.HAL_PCD_EP_Close) for HAL_PCD_EP_Close
    usbd_conf.o(i.USBD_LL_DeInit) refers to stm32l0xx_hal_pcd.o(i.HAL_PCD_DeInit) for HAL_PCD_DeInit
    usbd_conf.o(i.USBD_LL_Delay) refers to stm32l0xx_hal.o(i.HAL_Delay) for HAL_Delay
    usbd_conf.o(i.USBD_LL_FlushEP) refers to stm32l0xx_hal_pcd.o(i.HAL_PCD_EP_Flush) for HAL_PCD_EP_Flush
    usbd_conf.o(i.USBD_LL_GetRxDataSize) refers to stm32l0xx_hal_pcd.o(i.HAL_PCD_EP_GetRxCount) for HAL_PCD_EP_GetRxCount
    usbd_conf.o(i.USBD_LL_Init) refers to stm32l0xx_hal_pcd.o(i.HAL_PCD_Init) for HAL_PCD_Init
    usbd_conf.o(i.USBD_LL_Init) refers to stm32l0xx_hal_pcd_ex.o(i.HAL_PCDEx_PMAConfig) for HAL_PCDEx_PMAConfig
    usbd_conf.o(i.USBD_LL_Init) refers to usbd_conf.o(.bss) for .bss
    usbd_conf.o(i.USBD_LL_OpenEP) refers to stm32l0xx_hal_pcd.o(i.HAL_PCD_EP_Open) for HAL_PCD_EP_Open
    usbd_conf.o(i.USBD_LL_PrepareReceive) refers to stm32l0xx_hal_pcd.o(i.HAL_PCD_EP_Receive) for HAL_PCD_EP_Receive
    usbd_conf.o(i.USBD_LL_SetUSBAddress) refers to stm32l0xx_hal_pcd.o(i.HAL_PCD_SetAddress) for HAL_PCD_SetAddress
    usbd_conf.o(i.USBD_LL_StallEP) refers to stm32l0xx_hal_pcd.o(i.HAL_PCD_EP_SetStall) for HAL_PCD_EP_SetStall
    usbd_conf.o(i.USBD_LL_Start) refers to stm32l0xx_hal_pcd.o(i.HAL_PCD_Start) for HAL_PCD_Start
    usbd_conf.o(i.USBD_LL_Stop) refers to stm32l0xx_hal_pcd.o(i.HAL_PCD_Stop) for HAL_PCD_Stop
    usbd_conf.o(i.USBD_LL_Transmit) refers to stm32l0xx_hal_pcd.o(i.HAL_PCD_EP_Transmit) for HAL_PCD_EP_Transmit
    usbd_conf.o(i.USBD_static_malloc) refers to usbd_conf.o(.bss) for .bss
    usbd_desc.o(i.USBD_HID_ConfigStrDescriptor) refers to usbd_ctlreq.o(i.USBD_GetString) for USBD_GetString
    usbd_desc.o(i.USBD_HID_ConfigStrDescriptor) refers to usbd_desc.o(.bss) for .bss
    usbd_desc.o(i.USBD_HID_DeviceDescriptor) refers to usbd_desc.o(.constdata) for .constdata
    usbd_desc.o(i.USBD_HID_InterfaceStrDescriptor) refers to usbd_ctlreq.o(i.USBD_GetString) for USBD_GetString
    usbd_desc.o(i.USBD_HID_InterfaceStrDescriptor) refers to usbd_desc.o(.bss) for .bss
    usbd_desc.o(i.USBD_HID_LangIDStrDescriptor) refers to usbd_desc.o(.constdata) for .constdata
    usbd_desc.o(i.USBD_HID_ManufacturerStrDescriptor) refers to usbd_ctlreq.o(i.USBD_GetString) for USBD_GetString
    usbd_desc.o(i.USBD_HID_ManufacturerStrDescriptor) refers to usbd_desc.o(.bss) for .bss
    usbd_desc.o(i.USBD_HID_ProductStrDescriptor) refers to usbd_ctlreq.o(i.USBD_GetString) for USBD_GetString
    usbd_desc.o(i.USBD_HID_ProductStrDescriptor) refers to usbd_desc.o(.bss) for .bss
    usbd_desc.o(i.USBD_HID_SerialStrDescriptor) refers to usbd_desc.o(i.IntToUnicode) for IntToUnicode
    usbd_desc.o(i.USBD_HID_SerialStrDescriptor) refers to usbd_desc.o(.data) for .data
    usbd_desc.o(.data) refers to usbd_desc.o(i.USBD_HID_DeviceDescriptor) for USBD_HID_DeviceDescriptor
    usbd_desc.o(.data) refers to usbd_desc.o(i.USBD_HID_LangIDStrDescriptor) for USBD_HID_LangIDStrDescriptor
    usbd_desc.o(.data) refers to usbd_desc.o(i.USBD_HID_ManufacturerStrDescriptor) for USBD_HID_ManufacturerStrDescriptor
    usbd_desc.o(.data) refers to usbd_desc.o(i.USBD_HID_ProductStrDescriptor) for USBD_HID_ProductStrDescriptor
    usbd_desc.o(.data) refers to usbd_desc.o(i.USBD_HID_SerialStrDescriptor) for USBD_HID_SerialStrDescriptor
    usbd_desc.o(.data) refers to usbd_desc.o(i.USBD_HID_ConfigStrDescriptor) for USBD_HID_ConfigStrDescriptor
    usbd_desc.o(.data) refers to usbd_desc.o(i.USBD_HID_InterfaceStrDescriptor) for USBD_HID_InterfaceStrDescriptor
    usbdapp.o(i.GetPointerData) refers to tsl_user.o(.constdata) for MyLinRots
    usbdapp.o(i.USB_process) refers to usbdapp.o(i.GetPointerData) for GetPointerData
    usbdapp.o(i.USB_process) refers to usbd_hid.o(i.USBD_HID_SendReport) for USBD_HID_SendReport
    usbdapp.o(i.USB_process) refers to tsl_user.o(.constdata) for MyLinRots
    usbdapp.o(i.USB_process) refers to usbdapp.o(.data) for .data
    usbdapp.o(i.USB_process) refers to bsp.o(.bss) for USBD_Device
    gde021a1.o(i.gde021a1_CloseChargePump) refers to stm32l0538_discovery.o(i.EPD_IO_WriteReg) for EPD_IO_WriteReg
    gde021a1.o(i.gde021a1_CloseChargePump) refers to stm32l0538_discovery.o(i.EPD_IO_WriteData) for EPD_IO_WriteData
    gde021a1.o(i.gde021a1_DrawImage) refers to stm32l0538_discovery.o(i.EPD_IO_WriteReg) for EPD_IO_WriteReg
    gde021a1.o(i.gde021a1_DrawImage) refers to stm32l0538_discovery.o(i.EPD_IO_WriteData) for EPD_IO_WriteData
    gde021a1.o(i.gde021a1_DrawImage) refers to uidiv.o(.text) for __aeabi_uidivmod
    gde021a1.o(i.gde021a1_Init) refers to stm32l0538_discovery.o(i.EPD_IO_Init) for EPD_IO_Init
    gde021a1.o(i.gde021a1_Init) refers to stm32l0538_discovery.o(i.EPD_IO_WriteReg) for EPD_IO_WriteReg
    gde021a1.o(i.gde021a1_Init) refers to stm32l0538_discovery.o(i.EPD_IO_WriteData) for EPD_IO_WriteData
    gde021a1.o(i.gde021a1_Init) refers to gde021a1.o(.constdata) for .constdata
    gde021a1.o(i.gde021a1_ReadReg) refers to stm32l0538_discovery.o(i.EPD_IO_WriteReg) for EPD_IO_WriteReg
    gde021a1.o(i.gde021a1_ReadReg) refers to stm32l0538_discovery.o(i.EPD_IO_ReadData) for EPD_IO_ReadData
    gde021a1.o(i.gde021a1_RefreshDisplay) refers to stm32l0538_discovery.o(i.EPD_IO_WriteReg) for EPD_IO_WriteReg
    gde021a1.o(i.gde021a1_RefreshDisplay) refers to stm32l0538_discovery.o(i.EPD_IO_WriteData) for EPD_IO_WriteData
    gde021a1.o(i.gde021a1_SetDisplayWindow) refers to stm32l0538_discovery.o(i.EPD_IO_WriteReg) for EPD_IO_WriteReg
    gde021a1.o(i.gde021a1_SetDisplayWindow) refers to stm32l0538_discovery.o(i.EPD_IO_WriteData) for EPD_IO_WriteData
    gde021a1.o(i.gde021a1_WritePixel) refers to stm32l0538_discovery.o(i.EPD_IO_WriteReg) for EPD_IO_WriteReg
    gde021a1.o(i.gde021a1_WritePixel) refers to stm32l0538_discovery.o(i.EPD_IO_WriteData) for EPD_IO_WriteData
    gde021a1.o(i.gde021a1_WriteReg) refers to stm32l0538_discovery.o(i.EPD_IO_WriteReg) for EPD_IO_WriteReg
    gde021a1.o(i.gde021a1_WriteReg) refers to stm32l0538_discovery.o(i.EPD_IO_WriteData) for EPD_IO_WriteData
    gde021a1.o(.data) refers to gde021a1.o(i.gde021a1_Init) for gde021a1_Init
    gde021a1.o(.data) refers to gde021a1.o(i.gde021a1_WritePixel) for gde021a1_WritePixel
    gde021a1.o(.data) refers to gde021a1.o(i.gde021a1_SetDisplayWindow) for gde021a1_SetDisplayWindow
    gde021a1.o(.data) refers to gde021a1.o(i.gde021a1_RefreshDisplay) for gde021a1_RefreshDisplay
    gde021a1.o(.data) refers to gde021a1.o(i.gde021a1_CloseChargePump) for gde021a1_CloseChargePump
    gde021a1.o(.data) refers to gde021a1.o(i.gde021a1_GetEpdPixelWidth) for gde021a1_GetEpdPixelWidth
    gde021a1.o(.data) refers to gde021a1.o(i.gde021a1_GetEpdPixelHeight) for gde021a1_GetEpdPixelHeight
    gde021a1.o(.data) refers to gde021a1.o(i.gde021a1_DrawImage) for gde021a1_DrawImage
    stm32l0538_discovery.o(i.BSP_LED_Init) refers to stm32l0xx_hal_gpio.o(i.HAL_GPIO_Init) for HAL_GPIO_Init
    stm32l0538_discovery.o(i.BSP_LED_Init) refers to stm32l0xx_hal_gpio.o(i.HAL_GPIO_WritePin) for HAL_GPIO_WritePin
    stm32l0538_discovery.o(i.BSP_LED_Init) refers to stm32l0538_discovery.o(.constdata) for .constdata
    stm32l0538_discovery.o(i.BSP_LED_Init) refers to stm32l0538_discovery.o(.data) for .data
    stm32l0538_discovery.o(i.BSP_LED_Off) refers to stm32l0xx_hal_gpio.o(i.HAL_GPIO_WritePin) for HAL_GPIO_WritePin
    stm32l0538_discovery.o(i.BSP_LED_Off) refers to stm32l0538_discovery.o(.constdata) for .constdata
    stm32l0538_discovery.o(i.BSP_LED_Off) refers to stm32l0538_discovery.o(.data) for .data
    stm32l0538_discovery.o(i.BSP_LED_On) refers to stm32l0xx_hal_gpio.o(i.HAL_GPIO_WritePin) for HAL_GPIO_WritePin
    stm32l0538_discovery.o(i.BSP_LED_On) refers to stm32l0538_discovery.o(.constdata) for .constdata
    stm32l0538_discovery.o(i.BSP_LED_On) refers to stm32l0538_discovery.o(.data) for .data
    stm32l0538_discovery.o(i.BSP_LED_Toggle) refers to stm32l0xx_hal_gpio.o(i.HAL_GPIO_TogglePin) for HAL_GPIO_TogglePin
    stm32l0538_discovery.o(i.BSP_LED_Toggle) refers to stm32l0538_discovery.o(.constdata) for .constdata
    stm32l0538_discovery.o(i.BSP_LED_Toggle) refers to stm32l0538_discovery.o(.data) for .data
    stm32l0538_discovery.o(i.BSP_PB_GetState) refers to stm32l0xx_hal_gpio.o(i.HAL_GPIO_ReadPin) for HAL_GPIO_ReadPin
    stm32l0538_discovery.o(i.BSP_PB_GetState) refers to stm32l0538_discovery.o(.constdata) for .constdata
    stm32l0538_discovery.o(i.BSP_PB_GetState) refers to stm32l0538_discovery.o(.data) for .data
    stm32l0538_discovery.o(i.BSP_PB_Init) refers to stm32l0xx_hal_gpio.o(i.HAL_GPIO_Init) for HAL_GPIO_Init
    stm32l0538_discovery.o(i.BSP_PB_Init) refers to stm32l0xx_hal_cortex.o(i.HAL_NVIC_SetPriority) for HAL_NVIC_SetPriority
    stm32l0538_discovery.o(i.BSP_PB_Init) refers to stm32l0xx_hal_cortex.o(i.HAL_NVIC_EnableIRQ) for HAL_NVIC_EnableIRQ
    stm32l0538_discovery.o(i.BSP_PB_Init) refers to stm32l0538_discovery.o(.constdata) for .constdata
    stm32l0538_discovery.o(i.BSP_PB_Init) refers to stm32l0538_discovery.o(.data) for .data
    stm32l0538_discovery.o(i.EPD_Delay) refers to stm32l0xx_hal.o(i.HAL_Delay) for HAL_Delay
    stm32l0538_discovery.o(i.EPD_IO_Init) refers to stm32l0xx_hal_gpio.o(i.HAL_GPIO_Init) for HAL_GPIO_Init
    stm32l0538_discovery.o(i.EPD_IO_Init) refers to stm32l0xx_hal_gpio.o(i.HAL_GPIO_WritePin) for HAL_GPIO_WritePin
    stm32l0538_discovery.o(i.EPD_IO_Init) refers to stm32l0xx_hal.o(i.HAL_Delay) for HAL_Delay
    stm32l0538_discovery.o(i.EPD_IO_Init) refers to stm32l0538_discovery.o(i.SPIx_Init) for SPIx_Init
    stm32l0538_discovery.o(i.EPD_IO_ReadData) refers to stm32l0xx_hal_gpio.o(i.HAL_GPIO_WritePin) for HAL_GPIO_WritePin
    stm32l0538_discovery.o(i.EPD_IO_ReadData) refers to stm32l0xx_hal_spi.o(i.HAL_SPI_TransmitReceive) for HAL_SPI_TransmitReceive
    stm32l0538_discovery.o(i.EPD_IO_ReadData) refers to stm32l0538_discovery.o(i.SPIx_Error) for SPIx_Error
    stm32l0538_discovery.o(i.EPD_IO_ReadData) refers to stm32l0538_discovery.o(.bss) for .bss
    stm32l0538_discovery.o(i.EPD_IO_WriteData) refers to stm32l0xx_hal_gpio.o(i.HAL_GPIO_WritePin) for HAL_GPIO_WritePin
    stm32l0538_discovery.o(i.EPD_IO_WriteData) refers to stm32l0538_discovery.o(i.SPIx_Write) for SPIx_Write
    stm32l0538_discovery.o(i.EPD_IO_WriteReg) refers to stm32l0xx_hal_gpio.o(i.HAL_GPIO_WritePin) for HAL_GPIO_WritePin
    stm32l0538_discovery.o(i.EPD_IO_WriteReg) refers to stm32l0538_discovery.o(i.SPIx_Write) for SPIx_Write
    stm32l0538_discovery.o(i.SPIx_Error) refers to stm32l0xx_hal_spi.o(i.HAL_SPI_DeInit) for HAL_SPI_DeInit
    stm32l0538_discovery.o(i.SPIx_Error) refers to stm32l0538_discovery.o(i.SPIx_Init) for SPIx_Init
    stm32l0538_discovery.o(i.SPIx_Error) refers to stm32l0538_discovery.o(.bss) for .bss
    stm32l0538_discovery.o(i.SPIx_Init) refers to stm32l0xx_hal_spi.o(i.HAL_SPI_GetState) for HAL_SPI_GetState
    stm32l0538_discovery.o(i.SPIx_Init) refers to stm32l0xx_hal_gpio.o(i.HAL_GPIO_Init) for HAL_GPIO_Init
    stm32l0538_discovery.o(i.SPIx_Init) refers to stm32l0xx_hal_spi.o(i.HAL_SPI_Init) for HAL_SPI_Init
    stm32l0538_discovery.o(i.SPIx_Init) refers to stm32l0538_discovery.o(.bss) for .bss
    stm32l0538_discovery.o(i.SPIx_Write) refers to stm32l0xx_hal_spi.o(i.HAL_SPI_Transmit) for HAL_SPI_Transmit
    stm32l0538_discovery.o(i.SPIx_Write) refers to stm32l0538_discovery.o(i.SPIx_Error) for SPIx_Error
    stm32l0538_discovery.o(i.SPIx_Write) refers to stm32l0538_discovery.o(.bss) for .bss
    stm32l0538_discovery_epd.o(i.BSP_EPD_Clear) refers to stm32l0538_discovery_epd.o(.data) for .data
    stm32l0538_discovery_epd.o(i.BSP_EPD_CloseChargePump) refers to stm32l0538_discovery.o(i.EPD_Delay) for EPD_Delay
    stm32l0538_discovery_epd.o(i.BSP_EPD_CloseChargePump) refers to stm32l0538_discovery_epd.o(.data) for .data
    stm32l0538_discovery_epd.o(i.BSP_EPD_DisplayChar) refers to stm32l0538_discovery_epd.o(.data) for .data
    stm32l0538_discovery_epd.o(i.BSP_EPD_DisplayStringAt) refers to stm32l0538_discovery_epd.o(i.BSP_EPD_GetXSize) for BSP_EPD_GetXSize
    stm32l0538_discovery_epd.o(i.BSP_EPD_DisplayStringAt) refers to uidiv.o(.text) for __aeabi_uidivmod
    stm32l0538_discovery_epd.o(i.BSP_EPD_DisplayStringAt) refers to stm32l0538_discovery_epd.o(i.BSP_EPD_DisplayChar) for BSP_EPD_DisplayChar
    stm32l0538_discovery_epd.o(i.BSP_EPD_DisplayStringAt) refers to stm32l0538_discovery_epd.o(.data) for .data
    stm32l0538_discovery_epd.o(i.BSP_EPD_DisplayStringAtLine) refers to stm32l0538_discovery_epd.o(i.BSP_EPD_DisplayStringAt) for BSP_EPD_DisplayStringAt
    stm32l0538_discovery_epd.o(i.BSP_EPD_DisplayStringAtLine) refers to stm32l0538_discovery_epd.o(.data) for .data
    stm32l0538_discovery_epd.o(i.BSP_EPD_DrawHLine) refers to stm32l0538_discovery_epd.o(.data) for .data
    stm32l0538_discovery_epd.o(i.BSP_EPD_DrawImage) refers to stm32l0538_discovery_epd.o(i.BSP_EPD_GetYSize) for BSP_EPD_GetYSize
    stm32l0538_discovery_epd.o(i.BSP_EPD_DrawImage) refers to stm32l0538_discovery_epd.o(i.BSP_EPD_GetXSize) for BSP_EPD_GetXSize
    stm32l0538_discovery_epd.o(i.BSP_EPD_DrawImage) refers to stm32l0538_discovery_epd.o(.data) for .data
    stm32l0538_discovery_epd.o(i.BSP_EPD_DrawRect) refers to stm32l0538_discovery_epd.o(i.BSP_EPD_DrawHLine) for BSP_EPD_DrawHLine
    stm32l0538_discovery_epd.o(i.BSP_EPD_DrawRect) refers to stm32l0538_discovery_epd.o(i.BSP_EPD_DrawVLine) for BSP_EPD_DrawVLine
    stm32l0538_discovery_epd.o(i.BSP_EPD_DrawVLine) refers to stm32l0538_discovery_epd.o(.data) for .data
    stm32l0538_discovery_epd.o(i.BSP_EPD_FillRect) refers to stm32l0538_discovery_epd.o(.data) for .data
    stm32l0538_discovery_epd.o(i.BSP_EPD_GetFont) refers to stm32l0538_discovery_epd.o(.data) for .data
    stm32l0538_discovery_epd.o(i.BSP_EPD_GetXSize) refers to stm32l0538_discovery_epd.o(.data) for .data
    stm32l0538_discovery_epd.o(i.BSP_EPD_GetYSize) refers to stm32l0538_discovery_epd.o(.data) for .data
    stm32l0538_discovery_epd.o(i.BSP_EPD_Init) refers to stm32l0538_discovery_epd.o(i.BSP_EPD_Clear) for BSP_EPD_Clear
    stm32l0538_discovery_epd.o(i.BSP_EPD_Init) refers to stm32l0538_discovery_epd.o(.data) for .data
    stm32l0538_discovery_epd.o(i.BSP_EPD_Init) refers to gde021a1.o(.data) for gde021a1_drv
    stm32l0538_discovery_epd.o(i.BSP_EPD_RefreshDisplay) refers to stm32l0xx_hal_gpio.o(i.HAL_GPIO_ReadPin) for HAL_GPIO_ReadPin
    stm32l0538_discovery_epd.o(i.BSP_EPD_RefreshDisplay) refers to stm32l0xx_hal_gpio.o(i.HAL_GPIO_WritePin) for HAL_GPIO_WritePin
    stm32l0538_discovery_epd.o(i.BSP_EPD_RefreshDisplay) refers to stm32l0538_discovery.o(i.EPD_Delay) for EPD_Delay
    stm32l0538_discovery_epd.o(i.BSP_EPD_RefreshDisplay) refers to stm32l0538_discovery_epd.o(.data) for .data
    stm32l0538_discovery_epd.o(i.BSP_EPD_SetFont) refers to stm32l0538_discovery_epd.o(.data) for .data
    stm32l0538_discovery_epd.o(.data) refers to stm32l0538_discovery_epd.o(.constdata) for Font20_Table
    stm32l0538_discovery_epd.o(.data) refers to stm32l0538_discovery_epd.o(.constdata) for Font16_Table
    stm32l0538_discovery_epd.o(.data) refers to stm32l0538_discovery_epd.o(.constdata) for Font12_Table
    stm32l0538_discovery_epd.o(.data) refers to stm32l0538_discovery_epd.o(.constdata) for Font8_Table
    system_stm32l0xx.o(i.SystemCoreClockUpdate) refers to uidiv.o(.text) for __aeabi_uidivmod
    system_stm32l0xx.o(i.SystemCoreClockUpdate) refers to system_stm32l0xx.o(.data) for .data
    stm32l0xx_hal.o(i.HAL_DeInit) refers to stm32l0xx_hal_msp.o(i.HAL_MspDeInit) for HAL_MspDeInit
    stm32l0xx_hal.o(i.HAL_Delay) refers to stm32l0xx_hal.o(i.HAL_GetTick) for HAL_GetTick
    stm32l0xx_hal.o(i.HAL_GetTick) refers to stm32l0xx_hal.o(.data) for .data
    stm32l0xx_hal.o(i.HAL_IncTick) refers to stm32l0xx_hal.o(.data) for .data
    stm32l0xx_hal.o(i.HAL_Init) refers to stm32l0xx_hal.o(i.HAL_InitTick) for HAL_InitTick
    stm32l0xx_hal.o(i.HAL_Init) refers to stm32l0xx_hal_msp.o(i.HAL_MspInit) for HAL_MspInit
    stm32l0xx_hal.o(i.HAL_InitTick) refers to stm32l0xx_hal_rcc.o(i.HAL_RCC_GetHCLKFreq) for HAL_RCC_GetHCLKFreq
    stm32l0xx_hal.o(i.HAL_InitTick) refers to uidiv.o(.text) for __aeabi_uidivmod
    stm32l0xx_hal.o(i.HAL_InitTick) refers to stm32l0xx_hal_cortex.o(i.HAL_SYSTICK_Config) for HAL_SYSTICK_Config
    stm32l0xx_hal.o(i.HAL_InitTick) refers to stm32l0xx_hal_cortex.o(i.HAL_NVIC_SetPriority) for HAL_NVIC_SetPriority
    stm32l0xx_hal_cortex.o(i.HAL_NVIC_SetPriority) refers to stm32l0xx_hal_cortex.o(i.NVIC_SetPriority) for NVIC_SetPriority
    stm32l0xx_hal_cortex.o(i.HAL_SYSTICK_Config) refers to stm32l0xx_hal_cortex.o(i.NVIC_SetPriority) for NVIC_SetPriority
    stm32l0xx_hal_cortex.o(i.HAL_SYSTICK_IRQHandler) refers to stm32l0xx_hal_cortex.o(i.HAL_SYSTICK_Callback) for HAL_SYSTICK_Callback
    stm32l0xx_hal_dma.o(i.HAL_DMA_Abort) refers to stm32l0xx_hal.o(i.HAL_GetTick) for HAL_GetTick
    stm32l0xx_hal_dma.o(i.HAL_DMA_PollForTransfer) refers to stm32l0xx_hal.o(i.HAL_GetTick) for HAL_GetTick
    stm32l0xx_hal_dma.o(i.HAL_DMA_Start) refers to stm32l0xx_hal_dma.o(i.DMA_SetConfig) for DMA_SetConfig
    stm32l0xx_hal_dma.o(i.HAL_DMA_Start_IT) refers to stm32l0xx_hal_dma.o(i.DMA_SetConfig) for DMA_SetConfig
    stm32l0xx_hal_flash.o(i.FLASH_SetErrorCode) refers to stm32l0xx_hal_flash.o(.bss) for .bss
    stm32l0xx_hal_flash.o(i.FLASH_WaitForLastOperation) refers to stm32l0xx_hal.o(i.HAL_GetTick) for HAL_GetTick
    stm32l0xx_hal_flash.o(i.FLASH_WaitForLastOperation) refers to stm32l0xx_hal_flash.o(i.FLASH_SetErrorCode) for FLASH_SetErrorCode
    stm32l0xx_hal_flash.o(i.HAL_FLASH_GetError) refers to stm32l0xx_hal_flash.o(.bss) for .bss
    stm32l0xx_hal_flash.o(i.HAL_FLASH_IRQHandler) refers to stm32l0xx_hal_flash.o(i.HAL_FLASH_EndOfOperationCallback) for HAL_FLASH_EndOfOperationCallback
    stm32l0xx_hal_flash.o(i.HAL_FLASH_IRQHandler) refers to stm32l0xx_hal_flash.o(i.FLASH_Erase_Page) for FLASH_Erase_Page
    stm32l0xx_hal_flash.o(i.HAL_FLASH_IRQHandler) refers to stm32l0xx_hal_flash.o(i.FLASH_SetErrorCode) for FLASH_SetErrorCode
    stm32l0xx_hal_flash.o(i.HAL_FLASH_IRQHandler) refers to stm32l0xx_hal_flash.o(i.HAL_FLASH_OperationErrorCallback) for HAL_FLASH_OperationErrorCallback
    stm32l0xx_hal_flash.o(i.HAL_FLASH_IRQHandler) refers to stm32l0xx_hal_flash.o(.bss) for .bss
    stm32l0xx_hal_flash.o(i.HAL_FLASH_OB_Launch) refers to stm32l0xx_hal_flash.o(i.FLASH_WaitForLastOperation) for FLASH_WaitForLastOperation
    stm32l0xx_hal_flash.o(i.HAL_FLASH_Program) refers to stm32l0xx_hal_flash.o(i.FLASH_WaitForLastOperation) for FLASH_WaitForLastOperation
    stm32l0xx_hal_flash.o(i.HAL_FLASH_Program) refers to stm32l0xx_hal_flash.o(i.FLASH_Program_Word) for FLASH_Program_Word
    stm32l0xx_hal_flash.o(i.HAL_FLASH_Program) refers to stm32l0xx_hal_flash.o(.bss) for .bss
    stm32l0xx_hal_flash.o(i.HAL_FLASH_Program_IT) refers to stm32l0xx_hal_flash.o(i.FLASH_Program_Word) for FLASH_Program_Word
    stm32l0xx_hal_flash.o(i.HAL_FLASH_Program_IT) refers to stm32l0xx_hal_flash.o(.bss) for .bss
    stm32l0xx_hal_flash_ex.o(i.FLASH_OB_PCROPConfig) refers to stm32l0xx_hal_flash.o(i.FLASH_WaitForLastOperation) for FLASH_WaitForLastOperation
    stm32l0xx_hal_flash_ex.o(i.FLASH_OB_PCROPSelectionConfig) refers to stm32l0xx_hal_flash.o(i.FLASH_WaitForLastOperation) for FLASH_WaitForLastOperation
    stm32l0xx_hal_flash_ex.o(i.FLASH_OB_WRPConfig) refers to stm32l0xx_hal_flash.o(i.FLASH_WaitForLastOperation) for FLASH_WaitForLastOperation
    stm32l0xx_hal_flash_ex.o(i.HAL_FLASHEx_AdvOBProgram) refers to stm32l0xx_hal_flash_ex.o(i.FLASH_OB_PCROPConfig) for FLASH_OB_PCROPConfig
    stm32l0xx_hal_flash_ex.o(i.HAL_FLASHEx_AdvOBProgram) refers to stm32l0xx_hal_flash_ex.o(i.FLASH_OB_PCROPSelectionConfig) for FLASH_OB_PCROPSelectionConfig
    stm32l0xx_hal_flash_ex.o(i.HAL_FLASHEx_AdvOBProgram) refers to stm32l0xx_hal_flash.o(i.FLASH_WaitForLastOperation) for FLASH_WaitForLastOperation
    stm32l0xx_hal_flash_ex.o(i.HAL_FLASHEx_DATAEEPROM_Erase) refers to stm32l0xx_hal_flash.o(i.FLASH_WaitForLastOperation) for FLASH_WaitForLastOperation
    stm32l0xx_hal_flash_ex.o(i.HAL_FLASHEx_DATAEEPROM_Program) refers to stm32l0xx_hal_flash.o(i.FLASH_WaitForLastOperation) for FLASH_WaitForLastOperation
    stm32l0xx_hal_flash_ex.o(i.HAL_FLASHEx_DATAEEPROM_Program) refers to stm32l0xx_hal_flash.o(.bss) for pFlash
    stm32l0xx_hal_flash_ex.o(i.HAL_FLASHEx_Erase) refers to stm32l0xx_hal_flash.o(i.FLASH_WaitForLastOperation) for FLASH_WaitForLastOperation
    stm32l0xx_hal_flash_ex.o(i.HAL_FLASHEx_Erase) refers to stm32l0xx_hal_flash.o(i.FLASH_Erase_Page) for FLASH_Erase_Page
    stm32l0xx_hal_flash_ex.o(i.HAL_FLASHEx_Erase) refers to stm32l0xx_hal_flash.o(.bss) for pFlash
    stm32l0xx_hal_flash_ex.o(i.HAL_FLASHEx_Erase_IT) refers to stm32l0xx_hal_flash.o(i.FLASH_Erase_Page) for FLASH_Erase_Page
    stm32l0xx_hal_flash_ex.o(i.HAL_FLASHEx_Erase_IT) refers to stm32l0xx_hal_flash.o(.bss) for pFlash
    stm32l0xx_hal_flash_ex.o(i.HAL_FLASHEx_OBProgram) refers to stm32l0xx_hal_flash_ex.o(i.FLASH_OB_WRPConfig) for FLASH_OB_WRPConfig
    stm32l0xx_hal_flash_ex.o(i.HAL_FLASHEx_OBProgram) refers to stm32l0xx_hal_flash.o(i.FLASH_WaitForLastOperation) for FLASH_WaitForLastOperation
    stm32l0xx_hal_flash_ex.o(i.HAL_FLASHEx_OBProgram) refers to stm32l0xx_hal_flash.o(.bss) for pFlash
    stm32l0xx_hal_flash_ex.o(i.HAL_FLASHEx_OB_DeSelectPCROP) refers to stm32l0xx_hal_flash.o(i.FLASH_WaitForLastOperation) for FLASH_WaitForLastOperation
    stm32l0xx_hal_flash_ex.o(i.HAL_FLASHEx_OB_SelectPCROP) refers to stm32l0xx_hal_flash.o(i.FLASH_WaitForLastOperation) for FLASH_WaitForLastOperation
    stm32l0xx_hal_gpio.o(i.HAL_GPIO_EXTI_IRQHandler) refers to menu.o(i.HAL_GPIO_EXTI_Callback) for HAL_GPIO_EXTI_Callback
    stm32l0xx_hal_i2c.o(i.HAL_I2C_DeInit) refers to stm32l0xx_hal_msp.o(i.HAL_I2C_MspDeInit) for HAL_I2C_MspDeInit
    stm32l0xx_hal_i2c.o(i.HAL_I2C_ER_IRQHandler) refers to stm32l0xx_hal_i2c.o(i.HAL_I2C_ErrorCallback) for HAL_I2C_ErrorCallback
    stm32l0xx_hal_i2c.o(i.HAL_I2C_EV_IRQHandler) refers to stm32l0xx_hal_i2c.o(i.I2C_SlaveTransmit_ISR) for I2C_SlaveTransmit_ISR
    stm32l0xx_hal_i2c.o(i.HAL_I2C_EV_IRQHandler) refers to stm32l0xx_hal_i2c.o(i.I2C_MasterTransmit_ISR) for I2C_MasterTransmit_ISR
    stm32l0xx_hal_i2c.o(i.HAL_I2C_EV_IRQHandler) refers to stm32l0xx_hal_i2c.o(i.I2C_SlaveReceive_ISR) for I2C_SlaveReceive_ISR
    stm32l0xx_hal_i2c.o(i.HAL_I2C_EV_IRQHandler) refers to stm32l0xx_hal_i2c.o(i.I2C_MasterReceive_ISR) for I2C_MasterReceive_ISR
    stm32l0xx_hal_i2c.o(i.HAL_I2C_Init) refers to stm32l0xx_hal_msp.o(i.HAL_I2C_MspInit) for HAL_I2C_MspInit
    stm32l0xx_hal_i2c.o(i.HAL_I2C_IsDeviceReady) refers to stm32l0xx_hal.o(i.HAL_GetTick) for HAL_GetTick
    stm32l0xx_hal_i2c.o(i.HAL_I2C_IsDeviceReady) refers to stm32l0xx_hal_i2c.o(i.I2C_WaitOnFlagUntilTimeout) for I2C_WaitOnFlagUntilTimeout
    stm32l0xx_hal_i2c.o(i.HAL_I2C_Master_Receive) refers to stm32l0xx_hal_i2c.o(i.I2C_TransferConfig) for I2C_TransferConfig
    stm32l0xx_hal_i2c.o(i.HAL_I2C_Master_Receive) refers to stm32l0xx_hal_i2c.o(i.I2C_WaitOnFlagUntilTimeout) for I2C_WaitOnFlagUntilTimeout
    stm32l0xx_hal_i2c.o(i.HAL_I2C_Master_Receive) refers to stm32l0xx_hal_i2c.o(i.I2C_WaitOnSTOPFlagUntilTimeout) for I2C_WaitOnSTOPFlagUntilTimeout
    stm32l0xx_hal_i2c.o(i.HAL_I2C_Master_Receive_DMA) refers to stm32l0xx_hal_dma.o(i.HAL_DMA_Start_IT) for HAL_DMA_Start_IT
    stm32l0xx_hal_i2c.o(i.HAL_I2C_Master_Receive_DMA) refers to stm32l0xx_hal_i2c.o(i.I2C_TransferConfig) for I2C_TransferConfig
    stm32l0xx_hal_i2c.o(i.HAL_I2C_Master_Receive_DMA) refers to stm32l0xx_hal_i2c.o(i.I2C_WaitOnFlagUntilTimeout) for I2C_WaitOnFlagUntilTimeout
    stm32l0xx_hal_i2c.o(i.HAL_I2C_Master_Receive_DMA) refers to stm32l0xx_hal_i2c.o(i.I2C_DMAMasterReceiveCplt) for I2C_DMAMasterReceiveCplt
    stm32l0xx_hal_i2c.o(i.HAL_I2C_Master_Receive_DMA) refers to stm32l0xx_hal_i2c.o(i.I2C_DMAError) for I2C_DMAError
    stm32l0xx_hal_i2c.o(i.HAL_I2C_Master_Receive_IT) refers to stm32l0xx_hal_i2c.o(i.I2C_TransferConfig) for I2C_TransferConfig
    stm32l0xx_hal_i2c.o(i.HAL_I2C_Master_Transmit) refers to stm32l0xx_hal_i2c.o(i.I2C_TransferConfig) for I2C_TransferConfig
    stm32l0xx_hal_i2c.o(i.HAL_I2C_Master_Transmit) refers to stm32l0xx_hal_i2c.o(i.I2C_WaitOnTXISFlagUntilTimeout) for I2C_WaitOnTXISFlagUntilTimeout
    stm32l0xx_hal_i2c.o(i.HAL_I2C_Master_Transmit) refers to stm32l0xx_hal_i2c.o(i.I2C_WaitOnSTOPFlagUntilTimeout) for I2C_WaitOnSTOPFlagUntilTimeout
    stm32l0xx_hal_i2c.o(i.HAL_I2C_Master_Transmit) refers to stm32l0xx_hal_i2c.o(i.I2C_WaitOnFlagUntilTimeout) for I2C_WaitOnFlagUntilTimeout
    stm32l0xx_hal_i2c.o(i.HAL_I2C_Master_Transmit_DMA) refers to stm32l0xx_hal_dma.o(i.HAL_DMA_Start_IT) for HAL_DMA_Start_IT
    stm32l0xx_hal_i2c.o(i.HAL_I2C_Master_Transmit_DMA) refers to stm32l0xx_hal_i2c.o(i.I2C_TransferConfig) for I2C_TransferConfig
    stm32l0xx_hal_i2c.o(i.HAL_I2C_Master_Transmit_DMA) refers to stm32l0xx_hal_i2c.o(i.I2C_WaitOnTXISFlagUntilTimeout) for I2C_WaitOnTXISFlagUntilTimeout
    stm32l0xx_hal_i2c.o(i.HAL_I2C_Master_Transmit_DMA) refers to stm32l0xx_hal_i2c.o(i.I2C_DMAMasterTransmitCplt) for I2C_DMAMasterTransmitCplt
    stm32l0xx_hal_i2c.o(i.HAL_I2C_Master_Transmit_DMA) refers to stm32l0xx_hal_i2c.o(i.I2C_DMAError) for I2C_DMAError
    stm32l0xx_hal_i2c.o(i.HAL_I2C_Master_Transmit_IT) refers to stm32l0xx_hal_i2c.o(i.I2C_TransferConfig) for I2C_TransferConfig
    stm32l0xx_hal_i2c.o(i.HAL_I2C_Mem_Read) refers to stm32l0xx_hal_i2c.o(i.I2C_RequestMemoryRead) for I2C_RequestMemoryRead
    stm32l0xx_hal_i2c.o(i.HAL_I2C_Mem_Read) refers to stm32l0xx_hal_i2c.o(i.I2C_TransferConfig) for I2C_TransferConfig
    stm32l0xx_hal_i2c.o(i.HAL_I2C_Mem_Read) refers to stm32l0xx_hal_i2c.o(i.I2C_WaitOnFlagUntilTimeout) for I2C_WaitOnFlagUntilTimeout
    stm32l0xx_hal_i2c.o(i.HAL_I2C_Mem_Read) refers to stm32l0xx_hal_i2c.o(i.I2C_WaitOnSTOPFlagUntilTimeout) for I2C_WaitOnSTOPFlagUntilTimeout
    stm32l0xx_hal_i2c.o(i.HAL_I2C_Mem_Read_DMA) refers to stm32l0xx_hal_dma.o(i.HAL_DMA_Start_IT) for HAL_DMA_Start_IT
    stm32l0xx_hal_i2c.o(i.HAL_I2C_Mem_Read_DMA) refers to stm32l0xx_hal_i2c.o(i.I2C_RequestMemoryRead) for I2C_RequestMemoryRead
    stm32l0xx_hal_i2c.o(i.HAL_I2C_Mem_Read_DMA) refers to stm32l0xx_hal_i2c.o(i.I2C_TransferConfig) for I2C_TransferConfig
    stm32l0xx_hal_i2c.o(i.HAL_I2C_Mem_Read_DMA) refers to stm32l0xx_hal_i2c.o(i.I2C_WaitOnFlagUntilTimeout) for I2C_WaitOnFlagUntilTimeout
    stm32l0xx_hal_i2c.o(i.HAL_I2C_Mem_Read_DMA) refers to stm32l0xx_hal_i2c.o(i.I2C_DMAMemReceiveCplt) for I2C_DMAMemReceiveCplt
    stm32l0xx_hal_i2c.o(i.HAL_I2C_Mem_Read_DMA) refers to stm32l0xx_hal_i2c.o(i.I2C_DMAError) for I2C_DMAError
    stm32l0xx_hal_i2c.o(i.HAL_I2C_Mem_Read_IT) refers to stm32l0xx_hal_i2c.o(i.I2C_RequestMemoryRead) for I2C_RequestMemoryRead
    stm32l0xx_hal_i2c.o(i.HAL_I2C_Mem_Read_IT) refers to stm32l0xx_hal_i2c.o(i.I2C_TransferConfig) for I2C_TransferConfig
    stm32l0xx_hal_i2c.o(i.HAL_I2C_Mem_Write) refers to stm32l0xx_hal_i2c.o(i.I2C_RequestMemoryWrite) for I2C_RequestMemoryWrite
    stm32l0xx_hal_i2c.o(i.HAL_I2C_Mem_Write) refers to stm32l0xx_hal_i2c.o(i.I2C_TransferConfig) for I2C_TransferConfig
    stm32l0xx_hal_i2c.o(i.HAL_I2C_Mem_Write) refers to stm32l0xx_hal_i2c.o(i.I2C_WaitOnTXISFlagUntilTimeout) for I2C_WaitOnTXISFlagUntilTimeout
    stm32l0xx_hal_i2c.o(i.HAL_I2C_Mem_Write) refers to stm32l0xx_hal_i2c.o(i.I2C_WaitOnSTOPFlagUntilTimeout) for I2C_WaitOnSTOPFlagUntilTimeout
    stm32l0xx_hal_i2c.o(i.HAL_I2C_Mem_Write) refers to stm32l0xx_hal_i2c.o(i.I2C_WaitOnFlagUntilTimeout) for I2C_WaitOnFlagUntilTimeout
    stm32l0xx_hal_i2c.o(i.HAL_I2C_Mem_Write_DMA) refers to stm32l0xx_hal_dma.o(i.HAL_DMA_Start_IT) for HAL_DMA_Start_IT
    stm32l0xx_hal_i2c.o(i.HAL_I2C_Mem_Write_DMA) refers to stm32l0xx_hal_i2c.o(i.I2C_RequestMemoryWrite) for I2C_RequestMemoryWrite
    stm32l0xx_hal_i2c.o(i.HAL_I2C_Mem_Write_DMA) refers to stm32l0xx_hal_i2c.o(i.I2C_TransferConfig) for I2C_TransferConfig
    stm32l0xx_hal_i2c.o(i.HAL_I2C_Mem_Write_DMA) refers to stm32l0xx_hal_i2c.o(i.I2C_WaitOnTXISFlagUntilTimeout) for I2C_WaitOnTXISFlagUntilTimeout
    stm32l0xx_hal_i2c.o(i.HAL_I2C_Mem_Write_DMA) refers to stm32l0xx_hal_i2c.o(i.I2C_DMAMemTransmitCplt) for I2C_DMAMemTransmitCplt
    stm32l0xx_hal_i2c.o(i.HAL_I2C_Mem_Write_DMA) refers to stm32l0xx_hal_i2c.o(i.I2C_DMAError) for I2C_DMAError
    stm32l0xx_hal_i2c.o(i.HAL_I2C_Mem_Write_IT) refers to stm32l0xx_hal_i2c.o(i.I2C_RequestMemoryWrite) for I2C_RequestMemoryWrite
    stm32l0xx_hal_i2c.o(i.HAL_I2C_Mem_Write_IT) refers to stm32l0xx_hal_i2c.o(i.I2C_TransferConfig) for I2C_TransferConfig
    stm32l0xx_hal_i2c.o(i.HAL_I2C_Slave_Receive) refers to stm32l0xx_hal_i2c.o(i.I2C_WaitOnFlagUntilTimeout) for I2C_WaitOnFlagUntilTimeout
    stm32l0xx_hal_i2c.o(i.HAL_I2C_Slave_Receive) refers to stm32l0xx_hal_i2c.o(i.I2C_WaitOnRXNEFlagUntilTimeout) for I2C_WaitOnRXNEFlagUntilTimeout
    stm32l0xx_hal_i2c.o(i.HAL_I2C_Slave_Receive) refers to stm32l0xx_hal_i2c.o(i.I2C_WaitOnSTOPFlagUntilTimeout) for I2C_WaitOnSTOPFlagUntilTimeout
    stm32l0xx_hal_i2c.o(i.HAL_I2C_Slave_Receive_DMA) refers to stm32l0xx_hal_dma.o(i.HAL_DMA_Start_IT) for HAL_DMA_Start_IT
    stm32l0xx_hal_i2c.o(i.HAL_I2C_Slave_Receive_DMA) refers to stm32l0xx_hal_i2c.o(i.I2C_WaitOnFlagUntilTimeout) for I2C_WaitOnFlagUntilTimeout
    stm32l0xx_hal_i2c.o(i.HAL_I2C_Slave_Receive_DMA) refers to stm32l0xx_hal_i2c.o(i.I2C_DMASlaveReceiveCplt) for I2C_DMASlaveReceiveCplt
    stm32l0xx_hal_i2c.o(i.HAL_I2C_Slave_Receive_DMA) refers to stm32l0xx_hal_i2c.o(i.I2C_DMAError) for I2C_DMAError
    stm32l0xx_hal_i2c.o(i.HAL_I2C_Slave_Transmit) refers to stm32l0xx_hal_i2c.o(i.I2C_WaitOnFlagUntilTimeout) for I2C_WaitOnFlagUntilTimeout
    stm32l0xx_hal_i2c.o(i.HAL_I2C_Slave_Transmit) refers to stm32l0xx_hal_i2c.o(i.I2C_WaitOnTXISFlagUntilTimeout) for I2C_WaitOnTXISFlagUntilTimeout
    stm32l0xx_hal_i2c.o(i.HAL_I2C_Slave_Transmit) refers to stm32l0xx_hal_i2c.o(i.I2C_WaitOnSTOPFlagUntilTimeout) for I2C_WaitOnSTOPFlagUntilTimeout
    stm32l0xx_hal_i2c.o(i.HAL_I2C_Slave_Transmit_DMA) refers to stm32l0xx_hal_dma.o(i.HAL_DMA_Start_IT) for HAL_DMA_Start_IT
    stm32l0xx_hal_i2c.o(i.HAL_I2C_Slave_Transmit_DMA) refers to stm32l0xx_hal_i2c.o(i.I2C_WaitOnFlagUntilTimeout) for I2C_WaitOnFlagUntilTimeout
    stm32l0xx_hal_i2c.o(i.HAL_I2C_Slave_Transmit_DMA) refers to stm32l0xx_hal_i2c.o(i.I2C_DMASlaveTransmitCplt) for I2C_DMASlaveTransmitCplt
    stm32l0xx_hal_i2c.o(i.HAL_I2C_Slave_Transmit_DMA) refers to stm32l0xx_hal_i2c.o(i.I2C_DMAError) for I2C_DMAError
    stm32l0xx_hal_i2c.o(i.I2C_DMAError) refers to stm32l0xx_hal_i2c.o(i.HAL_I2C_ErrorCallback) for HAL_I2C_ErrorCallback
    stm32l0xx_hal_i2c.o(i.I2C_DMAMasterReceiveCplt) refers to stm32l0xx_hal_i2c.o(i.I2C_WaitOnFlagUntilTimeout) for I2C_WaitOnFlagUntilTimeout
    stm32l0xx_hal_i2c.o(i.I2C_DMAMasterReceiveCplt) refers to stm32l0xx_hal_i2c.o(i.I2C_WaitOnSTOPFlagUntilTimeout) for I2C_WaitOnSTOPFlagUntilTimeout
    stm32l0xx_hal_i2c.o(i.I2C_DMAMasterReceiveCplt) refers to stm32l0xx_hal_dma.o(i.HAL_DMA_Start_IT) for HAL_DMA_Start_IT
    stm32l0xx_hal_i2c.o(i.I2C_DMAMasterReceiveCplt) refers to stm32l0xx_hal_i2c.o(i.I2C_TransferConfig) for I2C_TransferConfig
    stm32l0xx_hal_i2c.o(i.I2C_DMAMasterReceiveCplt) refers to stm32l0xx_hal_i2c.o(i.HAL_I2C_ErrorCallback) for HAL_I2C_ErrorCallback
    stm32l0xx_hal_i2c.o(i.I2C_DMAMasterReceiveCplt) refers to stm32l0xx_hal_i2c.o(i.HAL_I2C_MasterRxCpltCallback) for HAL_I2C_MasterRxCpltCallback
    stm32l0xx_hal_i2c.o(i.I2C_DMAMasterTransmitCplt) refers to stm32l0xx_hal_i2c.o(i.I2C_WaitOnFlagUntilTimeout) for I2C_WaitOnFlagUntilTimeout
    stm32l0xx_hal_i2c.o(i.I2C_DMAMasterTransmitCplt) refers to stm32l0xx_hal_i2c.o(i.I2C_WaitOnSTOPFlagUntilTimeout) for I2C_WaitOnSTOPFlagUntilTimeout
    stm32l0xx_hal_i2c.o(i.I2C_DMAMasterTransmitCplt) refers to stm32l0xx_hal_dma.o(i.HAL_DMA_Start_IT) for HAL_DMA_Start_IT
    stm32l0xx_hal_i2c.o(i.I2C_DMAMasterTransmitCplt) refers to stm32l0xx_hal_i2c.o(i.I2C_TransferConfig) for I2C_TransferConfig
    stm32l0xx_hal_i2c.o(i.I2C_DMAMasterTransmitCplt) refers to stm32l0xx_hal_i2c.o(i.I2C_WaitOnTXISFlagUntilTimeout) for I2C_WaitOnTXISFlagUntilTimeout
    stm32l0xx_hal_i2c.o(i.I2C_DMAMasterTransmitCplt) refers to stm32l0xx_hal_i2c.o(i.HAL_I2C_ErrorCallback) for HAL_I2C_ErrorCallback
    stm32l0xx_hal_i2c.o(i.I2C_DMAMasterTransmitCplt) refers to stm32l0xx_hal_i2c.o(i.HAL_I2C_MasterTxCpltCallback) for HAL_I2C_MasterTxCpltCallback
    stm32l0xx_hal_i2c.o(i.I2C_DMAMemReceiveCplt) refers to stm32l0xx_hal_i2c.o(i.I2C_WaitOnFlagUntilTimeout) for I2C_WaitOnFlagUntilTimeout
    stm32l0xx_hal_i2c.o(i.I2C_DMAMemReceiveCplt) refers to stm32l0xx_hal_i2c.o(i.I2C_WaitOnSTOPFlagUntilTimeout) for I2C_WaitOnSTOPFlagUntilTimeout
    stm32l0xx_hal_i2c.o(i.I2C_DMAMemReceiveCplt) refers to stm32l0xx_hal_dma.o(i.HAL_DMA_Start_IT) for HAL_DMA_Start_IT
    stm32l0xx_hal_i2c.o(i.I2C_DMAMemReceiveCplt) refers to stm32l0xx_hal_i2c.o(i.I2C_TransferConfig) for I2C_TransferConfig
    stm32l0xx_hal_i2c.o(i.I2C_DMAMemReceiveCplt) refers to stm32l0xx_hal_i2c.o(i.HAL_I2C_ErrorCallback) for HAL_I2C_ErrorCallback
    stm32l0xx_hal_i2c.o(i.I2C_DMAMemReceiveCplt) refers to stm32l0xx_hal_i2c.o(i.HAL_I2C_MemRxCpltCallback) for HAL_I2C_MemRxCpltCallback
    stm32l0xx_hal_i2c.o(i.I2C_DMAMemTransmitCplt) refers to stm32l0xx_hal_i2c.o(i.I2C_WaitOnFlagUntilTimeout) for I2C_WaitOnFlagUntilTimeout
    stm32l0xx_hal_i2c.o(i.I2C_DMAMemTransmitCplt) refers to stm32l0xx_hal_i2c.o(i.I2C_WaitOnSTOPFlagUntilTimeout) for I2C_WaitOnSTOPFlagUntilTimeout
    stm32l0xx_hal_i2c.o(i.I2C_DMAMemTransmitCplt) refers to stm32l0xx_hal_dma.o(i.HAL_DMA_Start_IT) for HAL_DMA_Start_IT
    stm32l0xx_hal_i2c.o(i.I2C_DMAMemTransmitCplt) refers to stm32l0xx_hal_i2c.o(i.I2C_TransferConfig) for I2C_TransferConfig
    stm32l0xx_hal_i2c.o(i.I2C_DMAMemTransmitCplt) refers to stm32l0xx_hal_i2c.o(i.I2C_WaitOnTXISFlagUntilTimeout) for I2C_WaitOnTXISFlagUntilTimeout
    stm32l0xx_hal_i2c.o(i.I2C_DMAMemTransmitCplt) refers to stm32l0xx_hal_i2c.o(i.HAL_I2C_ErrorCallback) for HAL_I2C_ErrorCallback
    stm32l0xx_hal_i2c.o(i.I2C_DMAMemTransmitCplt) refers to stm32l0xx_hal_i2c.o(i.HAL_I2C_MemTxCpltCallback) for HAL_I2C_MemTxCpltCallback
    stm32l0xx_hal_i2c.o(i.I2C_DMASlaveReceiveCplt) refers to stm32l0xx_hal_i2c.o(i.I2C_WaitOnSTOPFlagUntilTimeout) for I2C_WaitOnSTOPFlagUntilTimeout
    stm32l0xx_hal_i2c.o(i.I2C_DMASlaveReceiveCplt) refers to stm32l0xx_hal_i2c.o(i.I2C_WaitOnFlagUntilTimeout) for I2C_WaitOnFlagUntilTimeout
    stm32l0xx_hal_i2c.o(i.I2C_DMASlaveReceiveCplt) refers to stm32l0xx_hal_i2c.o(i.HAL_I2C_ErrorCallback) for HAL_I2C_ErrorCallback
    stm32l0xx_hal_i2c.o(i.I2C_DMASlaveReceiveCplt) refers to stm32l0xx_hal_i2c.o(i.HAL_I2C_SlaveRxCpltCallback) for HAL_I2C_SlaveRxCpltCallback
    stm32l0xx_hal_i2c.o(i.I2C_DMASlaveTransmitCplt) refers to stm32l0xx_hal_i2c.o(i.I2C_WaitOnSTOPFlagUntilTimeout) for I2C_WaitOnSTOPFlagUntilTimeout
    stm32l0xx_hal_i2c.o(i.I2C_DMASlaveTransmitCplt) refers to stm32l0xx_hal_i2c.o(i.I2C_WaitOnFlagUntilTimeout) for I2C_WaitOnFlagUntilTimeout
    stm32l0xx_hal_i2c.o(i.I2C_DMASlaveTransmitCplt) refers to stm32l0xx_hal_i2c.o(i.HAL_I2C_ErrorCallback) for HAL_I2C_ErrorCallback
    stm32l0xx_hal_i2c.o(i.I2C_DMASlaveTransmitCplt) refers to stm32l0xx_hal_i2c.o(i.HAL_I2C_SlaveTxCpltCallback) for HAL_I2C_SlaveTxCpltCallback
    stm32l0xx_hal_i2c.o(i.I2C_IsAcknowledgeFailed) refers to stm32l0xx_hal.o(i.HAL_GetTick) for HAL_GetTick
    stm32l0xx_hal_i2c.o(i.I2C_MasterReceive_ISR) refers to stm32l0xx_hal_i2c.o(i.I2C_TransferConfig) for I2C_TransferConfig
    stm32l0xx_hal_i2c.o(i.I2C_MasterReceive_ISR) refers to stm32l0xx_hal_i2c.o(i.HAL_I2C_MasterRxCpltCallback) for HAL_I2C_MasterRxCpltCallback
    stm32l0xx_hal_i2c.o(i.I2C_MasterReceive_ISR) refers to stm32l0xx_hal_i2c.o(i.HAL_I2C_MemRxCpltCallback) for HAL_I2C_MemRxCpltCallback
    stm32l0xx_hal_i2c.o(i.I2C_MasterReceive_ISR) refers to stm32l0xx_hal_i2c.o(i.HAL_I2C_ErrorCallback) for HAL_I2C_ErrorCallback
    stm32l0xx_hal_i2c.o(i.I2C_MasterTransmit_ISR) refers to stm32l0xx_hal_i2c.o(i.I2C_TransferConfig) for I2C_TransferConfig
    stm32l0xx_hal_i2c.o(i.I2C_MasterTransmit_ISR) refers to stm32l0xx_hal_i2c.o(i.HAL_I2C_MasterTxCpltCallback) for HAL_I2C_MasterTxCpltCallback
    stm32l0xx_hal_i2c.o(i.I2C_MasterTransmit_ISR) refers to stm32l0xx_hal_i2c.o(i.HAL_I2C_MemTxCpltCallback) for HAL_I2C_MemTxCpltCallback
    stm32l0xx_hal_i2c.o(i.I2C_MasterTransmit_ISR) refers to stm32l0xx_hal_i2c.o(i.HAL_I2C_ErrorCallback) for HAL_I2C_ErrorCallback
    stm32l0xx_hal_i2c.o(i.I2C_RequestMemoryRead) refers to stm32l0xx_hal_i2c.o(i.I2C_TransferConfig) for I2C_TransferConfig
    stm32l0xx_hal_i2c.o(i.I2C_RequestMemoryRead) refers to stm32l0xx_hal_i2c.o(i.I2C_WaitOnTXISFlagUntilTimeout) for I2C_WaitOnTXISFlagUntilTimeout
    stm32l0xx_hal_i2c.o(i.I2C_RequestMemoryRead) refers to stm32l0xx_hal_i2c.o(i.I2C_WaitOnFlagUntilTimeout) for I2C_WaitOnFlagUntilTimeout
    stm32l0xx_hal_i2c.o(i.I2C_RequestMemoryWrite) refers to stm32l0xx_hal_i2c.o(i.I2C_TransferConfig) for I2C_TransferConfig
    stm32l0xx_hal_i2c.o(i.I2C_RequestMemoryWrite) refers to stm32l0xx_hal_i2c.o(i.I2C_WaitOnTXISFlagUntilTimeout) for I2C_WaitOnTXISFlagUntilTimeout
    stm32l0xx_hal_i2c.o(i.I2C_RequestMemoryWrite) refers to stm32l0xx_hal_i2c.o(i.I2C_WaitOnFlagUntilTimeout) for I2C_WaitOnFlagUntilTimeout
    stm32l0xx_hal_i2c.o(i.I2C_SlaveReceive_ISR) refers to stm32l0xx_hal_i2c.o(i.HAL_I2C_ErrorCallback) for HAL_I2C_ErrorCallback
    stm32l0xx_hal_i2c.o(i.I2C_SlaveReceive_ISR) refers to stm32l0xx_hal_i2c.o(i.HAL_I2C_SlaveRxCpltCallback) for HAL_I2C_SlaveRxCpltCallback
    stm32l0xx_hal_i2c.o(i.I2C_SlaveTransmit_ISR) refers to stm32l0xx_hal_i2c.o(i.HAL_I2C_ErrorCallback) for HAL_I2C_ErrorCallback
    stm32l0xx_hal_i2c.o(i.I2C_SlaveTransmit_ISR) refers to stm32l0xx_hal_i2c.o(i.HAL_I2C_SlaveTxCpltCallback) for HAL_I2C_SlaveTxCpltCallback
    stm32l0xx_hal_i2c.o(i.I2C_WaitOnFlagUntilTimeout) refers to stm32l0xx_hal.o(i.HAL_GetTick) for HAL_GetTick
    stm32l0xx_hal_i2c.o(i.I2C_WaitOnRXNEFlagUntilTimeout) refers to stm32l0xx_hal.o(i.HAL_GetTick) for HAL_GetTick
    stm32l0xx_hal_i2c.o(i.I2C_WaitOnSTOPFlagUntilTimeout) refers to stm32l0xx_hal.o(i.HAL_GetTick) for HAL_GetTick
    stm32l0xx_hal_i2c.o(i.I2C_WaitOnSTOPFlagUntilTimeout) refers to stm32l0xx_hal_i2c.o(i.I2C_IsAcknowledgeFailed) for I2C_IsAcknowledgeFailed
    stm32l0xx_hal_i2c.o(i.I2C_WaitOnTXISFlagUntilTimeout) refers to stm32l0xx_hal.o(i.HAL_GetTick) for HAL_GetTick
    stm32l0xx_hal_i2c.o(i.I2C_WaitOnTXISFlagUntilTimeout) refers to stm32l0xx_hal_i2c.o(i.I2C_IsAcknowledgeFailed) for I2C_IsAcknowledgeFailed
    stm32l0xx_hal_pcd.o(i.HAL_PCD_DeInit) refers to stm32l0xx_hal_pcd.o(i.HAL_PCD_Stop) for HAL_PCD_Stop
    stm32l0xx_hal_pcd.o(i.HAL_PCD_DeInit) refers to usbd_conf.o(i.HAL_PCD_MspDeInit) for HAL_PCD_MspDeInit
    stm32l0xx_hal_pcd.o(i.HAL_PCD_EP_Transmit) refers to stm32l0xx_hal_pcd.o(i.PCD_WritePMA) for PCD_WritePMA
    stm32l0xx_hal_pcd.o(i.HAL_PCD_IRQHandler) refers to stm32l0xx_hal_pcd.o(i.PCD_EP_ISR_Handler) for PCD_EP_ISR_Handler
    stm32l0xx_hal_pcd.o(i.HAL_PCD_IRQHandler) refers to usbd_conf.o(i.HAL_PCD_ResetCallback) for HAL_PCD_ResetCallback
    stm32l0xx_hal_pcd.o(i.HAL_PCD_IRQHandler) refers to stm32l0xx_hal_pcd.o(i.HAL_PCD_SetAddress) for HAL_PCD_SetAddress
    stm32l0xx_hal_pcd.o(i.HAL_PCD_IRQHandler) refers to usbd_conf.o(i.HAL_PCD_ResumeCallback) for HAL_PCD_ResumeCallback
    stm32l0xx_hal_pcd.o(i.HAL_PCD_IRQHandler) refers to usbd_conf.o(i.HAL_PCD_SuspendCallback) for HAL_PCD_SuspendCallback
    stm32l0xx_hal_pcd.o(i.HAL_PCD_IRQHandler) refers to usbd_conf.o(i.HAL_PCD_SOFCallback) for HAL_PCD_SOFCallback
    stm32l0xx_hal_pcd.o(i.HAL_PCD_Init) refers to usbd_conf.o(i.HAL_PCD_MspInit) for HAL_PCD_MspInit
    stm32l0xx_hal_pcd.o(i.PCD_EP_ISR_Handler) refers to usbd_conf.o(i.HAL_PCD_DataInStageCallback) for HAL_PCD_DataInStageCallback
    stm32l0xx_hal_pcd.o(i.PCD_EP_ISR_Handler) refers to stm32l0xx_hal_pcd.o(i.PCD_ReadPMA) for PCD_ReadPMA
    stm32l0xx_hal_pcd.o(i.PCD_EP_ISR_Handler) refers to usbd_conf.o(i.HAL_PCD_SetupStageCallback) for HAL_PCD_SetupStageCallback
    stm32l0xx_hal_pcd.o(i.PCD_EP_ISR_Handler) refers to usbd_conf.o(i.HAL_PCD_DataOutStageCallback) for HAL_PCD_DataOutStageCallback
    stm32l0xx_hal_pcd.o(i.PCD_EP_ISR_Handler) refers to stm32l0xx_hal_pcd.o(i.HAL_PCD_EP_Receive) for HAL_PCD_EP_Receive
    stm32l0xx_hal_pcd.o(i.PCD_EP_ISR_Handler) refers to stm32l0xx_hal_pcd.o(i.PCD_WritePMA) for PCD_WritePMA
    stm32l0xx_hal_pcd.o(i.PCD_EP_ISR_Handler) refers to stm32l0xx_hal_pcd.o(i.HAL_PCD_EP_Transmit) for HAL_PCD_EP_Transmit
    stm32l0xx_hal_pwr.o(i.HAL_PWR_PVD_IRQHandler) refers to stm32l0xx_hal_pwr.o(i.HAL_PWR_PVDCallback) for HAL_PWR_PVDCallback
    stm32l0xx_hal_rcc.o(i.HAL_RCC_ClockConfig) refers to stm32l0xx_hal.o(i.HAL_GetTick) for HAL_GetTick
    stm32l0xx_hal_rcc.o(i.HAL_RCC_ClockConfig) refers to stm32l0xx_hal.o(i.HAL_InitTick) for HAL_InitTick
    stm32l0xx_hal_rcc.o(i.HAL_RCC_GetHCLKFreq) refers to stm32l0xx_hal_rcc.o(i.HAL_RCC_GetSysClockFreq) for HAL_RCC_GetSysClockFreq
    stm32l0xx_hal_rcc.o(i.HAL_RCC_GetHCLKFreq) refers to stm32l0xx_hal_rcc.o(.data) for .data
    stm32l0xx_hal_rcc.o(i.HAL_RCC_GetHCLKFreq) refers to system_stm32l0xx.o(.data) for SystemCoreClock
    stm32l0xx_hal_rcc.o(i.HAL_RCC_GetPCLK1Freq) refers to stm32l0xx_hal_rcc.o(i.HAL_RCC_GetHCLKFreq) for HAL_RCC_GetHCLKFreq
    stm32l0xx_hal_rcc.o(i.HAL_RCC_GetPCLK1Freq) refers to stm32l0xx_hal_rcc.o(.data) for .data
    stm32l0xx_hal_rcc.o(i.HAL_RCC_GetPCLK2Freq) refers to stm32l0xx_hal_rcc.o(i.HAL_RCC_GetHCLKFreq) for HAL_RCC_GetHCLKFreq
    stm32l0xx_hal_rcc.o(i.HAL_RCC_GetPCLK2Freq) refers to stm32l0xx_hal_rcc.o(.data) for .data
    stm32l0xx_hal_rcc.o(i.HAL_RCC_GetSysClockFreq) refers to uidiv.o(.text) for __aeabi_uidivmod
    stm32l0xx_hal_rcc.o(i.HAL_RCC_GetSysClockFreq) refers to stm32l0xx_hal_rcc.o(.constdata) for .constdata
    stm32l0xx_hal_rcc.o(i.HAL_RCC_GetSysClockFreq) refers to stm32l0xx_hal_rcc.o(.data) for .data
    stm32l0xx_hal_rcc.o(i.HAL_RCC_MCOConfig) refers to stm32l0xx_hal_gpio.o(i.HAL_GPIO_Init) for HAL_GPIO_Init
    stm32l0xx_hal_rcc.o(i.HAL_RCC_NMI_IRQHandler) refers to stm32l0xx_hal_rcc.o(i.HAL_RCC_CCSCallback) for HAL_RCC_CCSCallback
    stm32l0xx_hal_rcc.o(i.HAL_RCC_OscConfig) refers to stm32l0xx_hal.o(i.HAL_GetTick) for HAL_GetTick
    stm32l0xx_hal_rcc_ex.o(i.HAL_RCCEx_CRSWaitSynchronization) refers to stm32l0xx_hal.o(i.HAL_GetTick) for HAL_GetTick
    stm32l0xx_hal_rcc_ex.o(i.HAL_RCCEx_PeriphCLKConfig) refers to stm32l0xx_hal.o(i.HAL_GetTick) for HAL_GetTick
    stm32l0xx_hal_spi.o(i.HAL_SPI_DMAStop) refers to stm32l0xx_hal_dma.o(i.HAL_DMA_Abort) for HAL_DMA_Abort
    stm32l0xx_hal_spi.o(i.HAL_SPI_DeInit) refers to stm32l0xx_hal_spi.o(i.HAL_SPI_MspDeInit) for HAL_SPI_MspDeInit
    stm32l0xx_hal_spi.o(i.HAL_SPI_IRQHandler) refers to stm32l0xx_hal_spi.o(i.HAL_SPI_ErrorCallback) for HAL_SPI_ErrorCallback
    stm32l0xx_hal_spi.o(i.HAL_SPI_Init) refers to stm32l0xx_hal_spi.o(i.HAL_SPI_MspInit) for HAL_SPI_MspInit
    stm32l0xx_hal_spi.o(i.HAL_SPI_Receive) refers to stm32l0xx_hal_spi.o(i.HAL_SPI_TransmitReceive) for HAL_SPI_TransmitReceive
    stm32l0xx_hal_spi.o(i.HAL_SPI_Receive) refers to stm32l0xx_hal_spi.o(i.SPI_WaitOnFlagUntilTimeout) for SPI_WaitOnFlagUntilTimeout
    stm32l0xx_hal_spi.o(i.HAL_SPI_Receive_DMA) refers to stm32l0xx_hal_dma.o(i.HAL_DMA_Start_IT) for HAL_DMA_Start_IT
    stm32l0xx_hal_spi.o(i.HAL_SPI_Receive_DMA) refers to stm32l0xx_hal_spi.o(i.HAL_SPI_TransmitReceive_DMA) for HAL_SPI_TransmitReceive_DMA
    stm32l0xx_hal_spi.o(i.HAL_SPI_Receive_DMA) refers to stm32l0xx_hal_spi.o(i.SPI_DMAHalfReceiveCplt) for SPI_DMAHalfReceiveCplt
    stm32l0xx_hal_spi.o(i.HAL_SPI_Receive_DMA) refers to stm32l0xx_hal_spi.o(i.SPI_DMAReceiveCplt) for SPI_DMAReceiveCplt
    stm32l0xx_hal_spi.o(i.HAL_SPI_Receive_DMA) refers to stm32l0xx_hal_spi.o(i.SPI_DMAError) for SPI_DMAError
    stm32l0xx_hal_spi.o(i.HAL_SPI_Receive_IT) refers to stm32l0xx_hal_spi.o(i.HAL_SPI_TransmitReceive_IT) for HAL_SPI_TransmitReceive_IT
    stm32l0xx_hal_spi.o(i.HAL_SPI_Receive_IT) refers to stm32l0xx_hal_spi.o(i.SPI_RxISR) for SPI_RxISR
    stm32l0xx_hal_spi.o(i.HAL_SPI_Transmit) refers to stm32l0xx_hal_spi.o(i.SPI_WaitOnFlagUntilTimeout) for SPI_WaitOnFlagUntilTimeout
    stm32l0xx_hal_spi.o(i.HAL_SPI_TransmitReceive) refers to stm32l0xx_hal_spi.o(i.SPI_WaitOnFlagUntilTimeout) for SPI_WaitOnFlagUntilTimeout
    stm32l0xx_hal_spi.o(i.HAL_SPI_TransmitReceive_DMA) refers to stm32l0xx_hal_dma.o(i.HAL_DMA_Start_IT) for HAL_DMA_Start_IT
    stm32l0xx_hal_spi.o(i.HAL_SPI_TransmitReceive_DMA) refers to stm32l0xx_hal_spi.o(i.SPI_DMAHalfTransmitReceiveCplt) for SPI_DMAHalfTransmitReceiveCplt
    stm32l0xx_hal_spi.o(i.HAL_SPI_TransmitReceive_DMA) refers to stm32l0xx_hal_spi.o(i.SPI_DMATransmitReceiveCplt) for SPI_DMATransmitReceiveCplt
    stm32l0xx_hal_spi.o(i.HAL_SPI_TransmitReceive_DMA) refers to stm32l0xx_hal_spi.o(i.SPI_DMAError) for SPI_DMAError
    stm32l0xx_hal_spi.o(i.HAL_SPI_TransmitReceive_DMA) refers to stm32l0xx_hal_spi.o(i.SPI_DMAHalfReceiveCplt) for SPI_DMAHalfReceiveCplt
    stm32l0xx_hal_spi.o(i.HAL_SPI_TransmitReceive_DMA) refers to stm32l0xx_hal_spi.o(i.SPI_DMAReceiveCplt) for SPI_DMAReceiveCplt
    stm32l0xx_hal_spi.o(i.HAL_SPI_TransmitReceive_IT) refers to stm32l0xx_hal_spi.o(i.SPI_TxISR) for SPI_TxISR
    stm32l0xx_hal_spi.o(i.HAL_SPI_TransmitReceive_IT) refers to stm32l0xx_hal_spi.o(i.SPI_2LinesRxISR) for SPI_2LinesRxISR
    stm32l0xx_hal_spi.o(i.HAL_SPI_Transmit_DMA) refers to stm32l0xx_hal_dma.o(i.HAL_DMA_Start_IT) for HAL_DMA_Start_IT
    stm32l0xx_hal_spi.o(i.HAL_SPI_Transmit_DMA) refers to stm32l0xx_hal_spi.o(i.SPI_DMAHalfTransmitCplt) for SPI_DMAHalfTransmitCplt
    stm32l0xx_hal_spi.o(i.HAL_SPI_Transmit_DMA) refers to stm32l0xx_hal_spi.o(i.SPI_DMATransmitCplt) for SPI_DMATransmitCplt
    stm32l0xx_hal_spi.o(i.HAL_SPI_Transmit_DMA) refers to stm32l0xx_hal_spi.o(i.SPI_DMAError) for SPI_DMAError
    stm32l0xx_hal_spi.o(i.HAL_SPI_Transmit_IT) refers to stm32l0xx_hal_spi.o(i.SPI_TxISR) for SPI_TxISR
    stm32l0xx_hal_spi.o(i.SPI_2LinesRxISR) refers to stm32l0xx_hal_spi.o(i.SPI_RxCloseIRQHandler) for SPI_RxCloseIRQHandler
    stm32l0xx_hal_spi.o(i.SPI_DMAError) refers to stm32l0xx_hal_spi.o(i.HAL_SPI_ErrorCallback) for HAL_SPI_ErrorCallback
    stm32l0xx_hal_spi.o(i.SPI_DMAHalfReceiveCplt) refers to stm32l0xx_hal_spi.o(i.HAL_SPI_RxHalfCpltCallback) for HAL_SPI_RxHalfCpltCallback
    stm32l0xx_hal_spi.o(i.SPI_DMAHalfTransmitCplt) refers to stm32l0xx_hal_spi.o(i.HAL_SPI_TxHalfCpltCallback) for HAL_SPI_TxHalfCpltCallback
    stm32l0xx_hal_spi.o(i.SPI_DMAHalfTransmitReceiveCplt) refers to stm32l0xx_hal_spi.o(i.HAL_SPI_TxRxHalfCpltCallback) for HAL_SPI_TxRxHalfCpltCallback
    stm32l0xx_hal_spi.o(i.SPI_DMAReceiveCplt) refers to stm32l0xx_hal_spi.o(i.SPI_WaitOnFlagUntilTimeout) for SPI_WaitOnFlagUntilTimeout
    stm32l0xx_hal_spi.o(i.SPI_DMAReceiveCplt) refers to stm32l0xx_hal_spi.o(i.HAL_SPI_ErrorCallback) for HAL_SPI_ErrorCallback
    stm32l0xx_hal_spi.o(i.SPI_DMAReceiveCplt) refers to stm32l0xx_hal_spi.o(i.HAL_SPI_RxCpltCallback) for HAL_SPI_RxCpltCallback
    stm32l0xx_hal_spi.o(i.SPI_DMATransmitCplt) refers to stm32l0xx_hal_spi.o(i.SPI_WaitOnFlagUntilTimeout) for SPI_WaitOnFlagUntilTimeout
    stm32l0xx_hal_spi.o(i.SPI_DMATransmitCplt) refers to stm32l0xx_hal_spi.o(i.HAL_SPI_ErrorCallback) for HAL_SPI_ErrorCallback
    stm32l0xx_hal_spi.o(i.SPI_DMATransmitCplt) refers to stm32l0xx_hal_spi.o(i.HAL_SPI_TxCpltCallback) for HAL_SPI_TxCpltCallback
    stm32l0xx_hal_spi.o(i.SPI_DMATransmitReceiveCplt) refers to stm32l0xx_hal_spi.o(i.SPI_WaitOnFlagUntilTimeout) for SPI_WaitOnFlagUntilTimeout
    stm32l0xx_hal_spi.o(i.SPI_DMATransmitReceiveCplt) refers to stm32l0xx_hal_spi.o(i.HAL_SPI_ErrorCallback) for HAL_SPI_ErrorCallback
    stm32l0xx_hal_spi.o(i.SPI_DMATransmitReceiveCplt) refers to stm32l0xx_hal_spi.o(i.HAL_SPI_TxRxCpltCallback) for HAL_SPI_TxRxCpltCallback
    stm32l0xx_hal_spi.o(i.SPI_RxCloseIRQHandler) refers to stm32l0xx_hal_spi.o(i.SPI_WaitOnFlagUntilTimeout) for SPI_WaitOnFlagUntilTimeout
    stm32l0xx_hal_spi.o(i.SPI_RxCloseIRQHandler) refers to stm32l0xx_hal_spi.o(i.HAL_SPI_ErrorCallback) for HAL_SPI_ErrorCallback
    stm32l0xx_hal_spi.o(i.SPI_RxCloseIRQHandler) refers to stm32l0xx_hal_spi.o(i.HAL_SPI_RxCpltCallback) for HAL_SPI_RxCpltCallback
    stm32l0xx_hal_spi.o(i.SPI_RxCloseIRQHandler) refers to stm32l0xx_hal_spi.o(i.HAL_SPI_TxRxCpltCallback) for HAL_SPI_TxRxCpltCallback
    stm32l0xx_hal_spi.o(i.SPI_RxISR) refers to stm32l0xx_hal_spi.o(i.SPI_RxCloseIRQHandler) for SPI_RxCloseIRQHandler
    stm32l0xx_hal_spi.o(i.SPI_TxCloseIRQHandler) refers to stm32l0xx_hal_spi.o(i.SPI_WaitOnFlagUntilTimeout) for SPI_WaitOnFlagUntilTimeout
    stm32l0xx_hal_spi.o(i.SPI_TxCloseIRQHandler) refers to stm32l0xx_hal_spi.o(i.HAL_SPI_ErrorCallback) for HAL_SPI_ErrorCallback
    stm32l0xx_hal_spi.o(i.SPI_TxCloseIRQHandler) refers to stm32l0xx_hal_spi.o(i.HAL_SPI_TxCpltCallback) for HAL_SPI_TxCpltCallback
    stm32l0xx_hal_spi.o(i.SPI_TxCloseIRQHandler) refers to stm32l0xx_hal_spi.o(i.HAL_SPI_TxRxCpltCallback) for HAL_SPI_TxRxCpltCallback
    stm32l0xx_hal_spi.o(i.SPI_TxISR) refers to stm32l0xx_hal_spi.o(i.SPI_TxCloseIRQHandler) for SPI_TxCloseIRQHandler
    stm32l0xx_hal_spi.o(i.SPI_WaitOnFlagUntilTimeout) refers to stm32l0xx_hal.o(i.HAL_GetTick) for HAL_GetTick
    stm32l0xx_hal_tsc.o(i.HAL_TSC_DeInit) refers to stm32l0xx_hal_msp.o(i.HAL_TSC_MspDeInit) for HAL_TSC_MspDeInit
    stm32l0xx_hal_tsc.o(i.HAL_TSC_IOConfig) refers to stm32l0xx_hal_tsc.o(i.TSC_extract_groups) for TSC_extract_groups
    stm32l0xx_hal_tsc.o(i.HAL_TSC_IRQHandler) refers to stm32l0xx_hal_tsc.o(i.HAL_TSC_ErrorCallback) for HAL_TSC_ErrorCallback
    stm32l0xx_hal_tsc.o(i.HAL_TSC_IRQHandler) refers to stm32l0xx_hal_tsc.o(i.HAL_TSC_ConvCpltCallback) for HAL_TSC_ConvCpltCallback
    stm32l0xx_hal_tsc.o(i.HAL_TSC_Init) refers to stm32l0xx_hal_msp.o(i.HAL_TSC_MspInit) for HAL_TSC_MspInit
    stm32l0xx_hal_tsc.o(i.HAL_TSC_Init) refers to stm32l0xx_hal_tsc.o(i.TSC_extract_groups) for TSC_extract_groups
    stm32l0xx_hal_tsc.o(i.HAL_TSC_PollForAcquisition) refers to stm32l0xx_hal_tsc.o(i.HAL_TSC_GetState) for HAL_TSC_GetState
    tsl.o(i.TSL_Init) refers to uidiv.o(.text) for __aeabi_uidivmod
    tsl.o(i.TSL_Init) refers to tsl_globals.o(.bss) for TSL_Globals
    tsl.o(i.TSL_Init) refers to system_stm32l0xx.o(.data) for SystemCoreClock
    tsl_acq.o(i.TSL_acq_BankCalibrate) refers to tsl_acq_tsc.o(i.TSL_acq_BankWaitEOC) for TSL_acq_BankWaitEOC
    tsl_acq.o(i.TSL_acq_BankCalibrate) refers to tsl_acq.o(i.TSL_acq_BankClearData) for TSL_acq_BankClearData
    tsl_acq.o(i.TSL_acq_BankCalibrate) refers to tsl_acq_tsc.o(i.TSL_acq_BankConfig) for TSL_acq_BankConfig
    tsl_acq.o(i.TSL_acq_BankCalibrate) refers to tsl_acq_tsc.o(i.TSL_acq_BankStartAcq) for TSL_acq_BankStartAcq
    tsl_acq.o(i.TSL_acq_BankCalibrate) refers to tsl_acq_tsc.o(i.TSL_acq_GetMeas) for TSL_acq_GetMeas
    tsl_acq.o(i.TSL_acq_BankCalibrate) refers to tsl_globals.o(.bss) for TSL_Globals
    tsl_acq.o(i.TSL_acq_BankCalibrate) refers to tsl_acq.o(.data) for .data
    tsl_acq.o(i.TSL_acq_BankCalibrate) refers to tsl_user.o(.data) for TSL_Params
    tsl_acq.o(i.TSL_acq_BankClearData) refers to tsl_globals.o(.bss) for TSL_Globals
    tsl_acq.o(i.TSL_acq_BankGetResult) refers to tsl_acq_tsc.o(i.TSL_acq_GetMeas) for TSL_acq_GetMeas
    tsl_acq.o(i.TSL_acq_BankGetResult) refers to tsl_acq_tsc.o(i.TSL_acq_UseFilter) for TSL_acq_UseFilter
    tsl_acq.o(i.TSL_acq_BankGetResult) refers to tsl_acq_tsc.o(i.TSL_acq_ComputeDelta) for TSL_acq_ComputeDelta
    tsl_acq.o(i.TSL_acq_BankGetResult) refers to tsl_acq_tsc.o(i.TSL_acq_CheckNoise) for TSL_acq_CheckNoise
    tsl_acq.o(i.TSL_acq_BankGetResult) refers to tsl_globals.o(.bss) for TSL_Globals
    tsl_acq.o(i.TSL_acq_BankGetResult) refers to tsl_user.o(.data) for TSL_Params
    tsl_acq_tsc.o(i.TSL_acq_BankConfig) refers to tsl_globals.o(.bss) for TSL_Globals
    tsl_acq_tsc.o(i.TSL_acq_BankStartAcq) refers to tsl_acq_tsc.o(i.SoftDelay) for SoftDelay
    tsl_acq_tsc.o(i.TSL_acq_BankStartAcq) refers to tsl_globals.o(.bss) for TSL_Globals
    tsl_ecs.o(i.TSL_ecs_CalcK) refers to tsl_object.o(i.TSL_obj_SetGlobalObj) for TSL_obj_SetGlobalObj
    tsl_ecs.o(i.TSL_ecs_CalcK) refers to tsl_globals.o(.bss) for TSL_Globals
    tsl_ecs.o(i.TSL_ecs_Process) refers to tsl_time.o(i.TSL_tim_CheckDelay_ms) for TSL_tim_CheckDelay_ms
    tsl_ecs.o(i.TSL_ecs_Process) refers to tsl_ecs.o(i.TSL_ecs_CalcK) for TSL_ecs_CalcK
    tsl_ecs.o(i.TSL_ecs_Process) refers to tsl_ecs.o(i.TSL_ecs_ProcessK) for TSL_ecs_ProcessK
    tsl_ecs.o(i.TSL_ecs_Process) refers to tsl_globals.o(.bss) for TSL_Globals
    tsl_ecs.o(i.TSL_ecs_ProcessK) refers to tsl_object.o(i.TSL_obj_SetGlobalObj) for TSL_obj_SetGlobalObj
    tsl_ecs.o(i.TSL_ecs_ProcessK) refers to tsl_acq_tsc.o(i.TSL_acq_ComputeMeas) for TSL_acq_ComputeMeas
    tsl_ecs.o(i.TSL_ecs_ProcessK) refers to tsl_acq_tsc.o(i.TSL_acq_TestReferenceOutOfRange) for TSL_acq_TestReferenceOutOfRange
    tsl_ecs.o(i.TSL_ecs_ProcessK) refers to tsl_globals.o(.bss) for TSL_Globals
    tsl_ecs.o(i.TSL_ecs_ProcessK) refers to tsl_linrot.o(i.TSL_linrot_SetStateCalibration) for TSL_linrot_SetStateCalibration
    tsl_linrot.o(i.TSL_linrot_CalcPos) refers to uidiv.o(.text) for __aeabi_uidivmod
    tsl_linrot.o(i.TSL_linrot_CalcPos) refers to tsl_globals.o(.bss) for TSL_Globals
    tsl_linrot.o(i.TSL_linrot_CalcPos) refers to tsl_linrot.o(.data) for .data
    tsl_linrot.o(i.TSL_linrot_CalibrationStateProcess) refers to tsl_linrot.o(i.TSL_linrot_ProcessCh_One_AcqStatusError) for TSL_linrot_ProcessCh_One_AcqStatusError
    tsl_linrot.o(i.TSL_linrot_CalibrationStateProcess) refers to tsl_acq_tsc.o(i.TSL_acq_TestFirstReferenceIsValid) for TSL_acq_TestFirstReferenceIsValid
    tsl_linrot.o(i.TSL_linrot_CalibrationStateProcess) refers to tsl_globals.o(.bss) for TSL_Globals
    tsl_linrot.o(i.TSL_linrot_CalibrationStateProcess) refers to tsl_user.o(.data) for TSL_Params
    tsl_linrot.o(i.TSL_linrot_CalibrationStateProcess) refers to tsl_linrot.o(.data) for .data
    tsl_linrot.o(i.TSL_linrot_DTOGetTime) refers to tsl_globals.o(.bss) for TSL_Globals
    tsl_linrot.o(i.TSL_linrot_DebCalibrationStateProcess) refers to tsl_linrot.o(i.TSL_linrot_ProcessCh_One_AcqStatusError) for TSL_linrot_ProcessCh_One_AcqStatusError
    tsl_linrot.o(i.TSL_linrot_DebCalibrationStateProcess) refers to tsl_linrot.o(i.TSL_linrot_ProcessCh_One_DeltaBelowEquMinus) for TSL_linrot_ProcessCh_One_DeltaBelowEquMinus
    tsl_linrot.o(i.TSL_linrot_DebCalibrationStateProcess) refers to tsl_linrot.o(i.TSL_linrot_SetStateCalibration) for TSL_linrot_SetStateCalibration
    tsl_linrot.o(i.TSL_linrot_DebCalibrationStateProcess) refers to tsl_globals.o(.bss) for TSL_Globals
    tsl_linrot.o(i.TSL_linrot_DebDetectStateProcess) refers to tsl_linrot.o(i.TSL_linrot_ProcessCh_One_AcqStatusError) for TSL_linrot_ProcessCh_One_AcqStatusError
    tsl_linrot.o(i.TSL_linrot_DebDetectStateProcess) refers to tsl_linrot.o(i.TSL_linrot_ProcessCh_One_DeltaAboveEqu) for TSL_linrot_ProcessCh_One_DeltaAboveEqu
    tsl_linrot.o(i.TSL_linrot_DebDetectStateProcess) refers to tsl_linrot.o(i.TSL_linrot_DTOGetTime) for TSL_linrot_DTOGetTime
    tsl_linrot.o(i.TSL_linrot_DebDetectStateProcess) refers to tsl_globals.o(.bss) for TSL_Globals
    tsl_linrot.o(i.TSL_linrot_DebErrorStateProcess) refers to tsl_linrot.o(i.TSL_linrot_ProcessCh_One_AcqStatusError) for TSL_linrot_ProcessCh_One_AcqStatusError
    tsl_linrot.o(i.TSL_linrot_DebErrorStateProcess) refers to tsl_linrot.o(i.TSL_linrot_GetStateMask) for TSL_linrot_GetStateMask
    tsl_linrot.o(i.TSL_linrot_DebErrorStateProcess) refers to tsl_linrot.o(i.TSL_linrot_SetStateCalibration) for TSL_linrot_SetStateCalibration
    tsl_linrot.o(i.TSL_linrot_DebErrorStateProcess) refers to tsl_globals.o(.bss) for TSL_Globals
    tsl_linrot.o(i.TSL_linrot_DebProxDetectStateProcess) refers to tsl_linrot.o(i.TSL_linrot_ProcessCh_One_AcqStatusError) for TSL_linrot_ProcessCh_One_AcqStatusError
    tsl_linrot.o(i.TSL_linrot_DebProxDetectStateProcess) refers to tsl_linrot.o(i.TSL_linrot_ProcessCh_One_DeltaAbove) for TSL_linrot_ProcessCh_One_DeltaAbove
    tsl_linrot.o(i.TSL_linrot_DebProxDetectStateProcess) refers to tsl_linrot.o(i.TSL_linrot_DTOGetTime) for TSL_linrot_DTOGetTime
    tsl_linrot.o(i.TSL_linrot_DebProxDetectStateProcess) refers to tsl_globals.o(.bss) for TSL_Globals
    tsl_linrot.o(i.TSL_linrot_DebProxStateProcess) refers to tsl_linrot.o(i.TSL_linrot_ProcessCh_One_AcqStatusError) for TSL_linrot_ProcessCh_One_AcqStatusError
    tsl_linrot.o(i.TSL_linrot_DebProxStateProcess) refers to tsl_linrot.o(i.TSL_linrot_ProcessCh_One_DeltaAboveEqu) for TSL_linrot_ProcessCh_One_DeltaAboveEqu
    tsl_linrot.o(i.TSL_linrot_DebProxStateProcess) refers to tsl_linrot.o(i.TSL_linrot_DTOGetTime) for TSL_linrot_DTOGetTime
    tsl_linrot.o(i.TSL_linrot_DebProxStateProcess) refers to tsl_globals.o(.bss) for TSL_Globals
    tsl_linrot.o(i.TSL_linrot_DebProxTouchStateProcess) refers to tsl_linrot.o(i.TSL_linrot_ProcessCh_One_AcqStatusError) for TSL_linrot_ProcessCh_One_AcqStatusError
    tsl_linrot.o(i.TSL_linrot_DebProxTouchStateProcess) refers to tsl_linrot.o(i.TSL_linrot_ProcessCh_One_DeltaAbove) for TSL_linrot_ProcessCh_One_DeltaAbove
    tsl_linrot.o(i.TSL_linrot_DebProxTouchStateProcess) refers to tsl_linrot.o(i.TSL_linrot_DTOGetTime) for TSL_linrot_DTOGetTime
    tsl_linrot.o(i.TSL_linrot_DebProxTouchStateProcess) refers to tsl_globals.o(.bss) for TSL_Globals
    tsl_linrot.o(i.TSL_linrot_DebReleaseDetectStateProcess) refers to tsl_linrot.o(i.TSL_linrot_ProcessCh_One_AcqStatusError) for TSL_linrot_ProcessCh_One_AcqStatusError
    tsl_linrot.o(i.TSL_linrot_DebReleaseDetectStateProcess) refers to tsl_linrot.o(i.TSL_linrot_ProcessCh_One_DeltaAbove) for TSL_linrot_ProcessCh_One_DeltaAbove
    tsl_linrot.o(i.TSL_linrot_DebReleaseDetectStateProcess) refers to tsl_globals.o(.bss) for TSL_Globals
    tsl_linrot.o(i.TSL_linrot_DebReleaseProxStateProcess) refers to tsl_linrot.o(i.TSL_linrot_ProcessCh_One_AcqStatusError) for TSL_linrot_ProcessCh_One_AcqStatusError
    tsl_linrot.o(i.TSL_linrot_DebReleaseProxStateProcess) refers to tsl_linrot.o(i.TSL_linrot_ProcessCh_One_DeltaAbove) for TSL_linrot_ProcessCh_One_DeltaAbove
    tsl_linrot.o(i.TSL_linrot_DebReleaseProxStateProcess) refers to tsl_globals.o(.bss) for TSL_Globals
    tsl_linrot.o(i.TSL_linrot_DebReleaseTouchStateProcess) refers to tsl_linrot.o(i.TSL_linrot_ProcessCh_One_AcqStatusError) for TSL_linrot_ProcessCh_One_AcqStatusError
    tsl_linrot.o(i.TSL_linrot_DebReleaseTouchStateProcess) refers to tsl_linrot.o(i.TSL_linrot_ProcessCh_One_DeltaAbove) for TSL_linrot_ProcessCh_One_DeltaAbove
    tsl_linrot.o(i.TSL_linrot_DebReleaseTouchStateProcess) refers to tsl_globals.o(.bss) for TSL_Globals
    tsl_linrot.o(i.TSL_linrot_DetectStateProcess) refers to tsl_linrot.o(i.TSL_linrot_ProcessCh_One_AcqStatusError) for TSL_linrot_ProcessCh_One_AcqStatusError
    tsl_linrot.o(i.TSL_linrot_DetectStateProcess) refers to tsl_linrot.o(i.TSL_linrot_ProcessCh_One_DeltaAbove) for TSL_linrot_ProcessCh_One_DeltaAbove
    tsl_linrot.o(i.TSL_linrot_DetectStateProcess) refers to tsl_time.o(i.TSL_tim_CheckDelay_sec) for TSL_tim_CheckDelay_sec
    tsl_linrot.o(i.TSL_linrot_DetectStateProcess) refers to tsl_linrot.o(i.TSL_linrot_SetStateCalibration) for TSL_linrot_SetStateCalibration
    tsl_linrot.o(i.TSL_linrot_DetectStateProcess) refers to tsl_linrot.o(i.TSL_linrot_DTOGetTime) for TSL_linrot_DTOGetTime
    tsl_linrot.o(i.TSL_linrot_DetectStateProcess) refers to tsl_globals.o(.bss) for TSL_Globals
    tsl_linrot.o(i.TSL_linrot_DetectStateProcess) refers to tsl_user.o(.data) for TSL_Params
    tsl_linrot.o(i.TSL_linrot_GetStateId) refers to tsl_globals.o(.bss) for TSL_Globals
    tsl_linrot.o(i.TSL_linrot_GetStateMask) refers to tsl_globals.o(.bss) for TSL_Globals
    tsl_linrot.o(i.TSL_linrot_Init) refers to tsl_linrot.o(i.TSL_linrot_SetStateCalibration) for TSL_linrot_SetStateCalibration
    tsl_linrot.o(i.TSL_linrot_Init) refers to tsl_globals.o(.bss) for TSL_Globals
    tsl_linrot.o(i.TSL_linrot_IsChanged) refers to tsl_globals.o(.bss) for TSL_Globals
    tsl_linrot.o(i.TSL_linrot_NormDelta) refers to tsl_globals.o(.bss) for TSL_Globals
    tsl_linrot.o(i.TSL_linrot_Process) refers to tsl_linrot.o(i.TSL_linrot_ProcessCh_One_DataReady) for TSL_linrot_ProcessCh_One_DataReady
    tsl_linrot.o(i.TSL_linrot_Process) refers to tsl_globals.o(.bss) for TSL_Globals
    tsl_linrot.o(i.TSL_linrot_ProcessCh_All_AcqStatus) refers to tsl_globals.o(.bss) for TSL_Globals
    tsl_linrot.o(i.TSL_linrot_ProcessCh_All_ClearRef) refers to tsl_globals.o(.bss) for TSL_Globals
    tsl_linrot.o(i.TSL_linrot_ProcessCh_All_DeltaBelowEqu) refers to tsl_globals.o(.bss) for TSL_Globals
    tsl_linrot.o(i.TSL_linrot_ProcessCh_All_SetStatus) refers to tsl_globals.o(.bss) for TSL_Globals
    tsl_linrot.o(i.TSL_linrot_ProcessCh_One_AcqStatusError) refers to tsl_globals.o(.bss) for TSL_Globals
    tsl_linrot.o(i.TSL_linrot_ProcessCh_One_DataReady) refers to tsl_globals.o(.bss) for TSL_Globals
    tsl_linrot.o(i.TSL_linrot_ProcessCh_One_DeltaAbove) refers to tsl_globals.o(.bss) for TSL_Globals
    tsl_linrot.o(i.TSL_linrot_ProcessCh_One_DeltaAboveEqu) refers to tsl_globals.o(.bss) for TSL_Globals
    tsl_linrot.o(i.TSL_linrot_ProcessCh_One_DeltaBelowEquMinus) refers to tsl_globals.o(.bss) for TSL_Globals
    tsl_linrot.o(i.TSL_linrot_ProxStateProcess) refers to tsl_linrot.o(i.TSL_linrot_ProcessCh_One_AcqStatusError) for TSL_linrot_ProcessCh_One_AcqStatusError
    tsl_linrot.o(i.TSL_linrot_ProxStateProcess) refers to tsl_linrot.o(i.TSL_linrot_ProcessCh_One_DeltaAboveEqu) for TSL_linrot_ProcessCh_One_DeltaAboveEqu
    tsl_linrot.o(i.TSL_linrot_ProxStateProcess) refers to tsl_linrot.o(i.TSL_linrot_ProcessCh_All_DeltaBelowEqu) for TSL_linrot_ProcessCh_All_DeltaBelowEqu
    tsl_linrot.o(i.TSL_linrot_ProxStateProcess) refers to tsl_time.o(i.TSL_tim_CheckDelay_sec) for TSL_tim_CheckDelay_sec
    tsl_linrot.o(i.TSL_linrot_ProxStateProcess) refers to tsl_linrot.o(i.TSL_linrot_SetStateCalibration) for TSL_linrot_SetStateCalibration
    tsl_linrot.o(i.TSL_linrot_ProxStateProcess) refers to tsl_linrot.o(i.TSL_linrot_DTOGetTime) for TSL_linrot_DTOGetTime
    tsl_linrot.o(i.TSL_linrot_ProxStateProcess) refers to tsl_globals.o(.bss) for TSL_Globals
    tsl_linrot.o(i.TSL_linrot_ProxStateProcess) refers to tsl_user.o(.data) for TSL_Params
    tsl_linrot.o(i.TSL_linrot_ReleaseStateProcess) refers to tsl_linrot.o(i.TSL_linrot_ProcessCh_One_AcqStatusError) for TSL_linrot_ProcessCh_One_AcqStatusError
    tsl_linrot.o(i.TSL_linrot_ReleaseStateProcess) refers to tsl_linrot.o(i.TSL_linrot_ProcessCh_One_DeltaAboveEqu) for TSL_linrot_ProcessCh_One_DeltaAboveEqu
    tsl_linrot.o(i.TSL_linrot_ReleaseStateProcess) refers to tsl_linrot.o(i.TSL_linrot_ProcessCh_One_DeltaBelowEquMinus) for TSL_linrot_ProcessCh_One_DeltaBelowEquMinus
    tsl_linrot.o(i.TSL_linrot_ReleaseStateProcess) refers to tsl_linrot.o(i.TSL_linrot_DTOGetTime) for TSL_linrot_DTOGetTime
    tsl_linrot.o(i.TSL_linrot_ReleaseStateProcess) refers to tsl_linrot.o(i.TSL_linrot_SetStateCalibration) for TSL_linrot_SetStateCalibration
    tsl_linrot.o(i.TSL_linrot_ReleaseStateProcess) refers to tsl_globals.o(.bss) for TSL_Globals
    tsl_linrot.o(i.TSL_linrot_SetStateBurstOnly) refers to tsl_linrot.o(i.TSL_linrot_ProcessCh_All_SetStatus) for TSL_linrot_ProcessCh_All_SetStatus
    tsl_linrot.o(i.TSL_linrot_SetStateBurstOnly) refers to tsl_globals.o(.bss) for TSL_Globals
    tsl_linrot.o(i.TSL_linrot_SetStateCalibration) refers to tsl_linrot.o(i.TSL_linrot_ProcessCh_All_SetStatus) for TSL_linrot_ProcessCh_All_SetStatus
    tsl_linrot.o(i.TSL_linrot_SetStateCalibration) refers to tsl_linrot.o(i.TSL_linrot_ProcessCh_All_ClearRef) for TSL_linrot_ProcessCh_All_ClearRef
    tsl_linrot.o(i.TSL_linrot_SetStateCalibration) refers to tsl_globals.o(.bss) for TSL_Globals
    tsl_linrot.o(i.TSL_linrot_SetStateCalibration) refers to tsl_user.o(.data) for TSL_Params
    tsl_linrot.o(i.TSL_linrot_SetStateCalibration) refers to tsl_linrot.o(.data) for .data
    tsl_linrot.o(i.TSL_linrot_SetStateOff) refers to tsl_linrot.o(i.TSL_linrot_ProcessCh_All_SetStatus) for TSL_linrot_ProcessCh_All_SetStatus
    tsl_linrot.o(i.TSL_linrot_SetStateOff) refers to tsl_globals.o(.bss) for TSL_Globals
    tsl_linrot.o(i.TSL_linrot_TouchStateProcess) refers to tsl_linrot.o(i.TSL_linrot_ProcessCh_One_AcqStatusError) for TSL_linrot_ProcessCh_One_AcqStatusError
    tsl_linrot.o(i.TSL_linrot_TouchStateProcess) refers to tsl_linrot.o(i.TSL_linrot_ProcessCh_One_DeltaAbove) for TSL_linrot_ProcessCh_One_DeltaAbove
    tsl_linrot.o(i.TSL_linrot_TouchStateProcess) refers to tsl_time.o(i.TSL_tim_CheckDelay_sec) for TSL_tim_CheckDelay_sec
    tsl_linrot.o(i.TSL_linrot_TouchStateProcess) refers to tsl_linrot.o(i.TSL_linrot_SetStateCalibration) for TSL_linrot_SetStateCalibration
    tsl_linrot.o(i.TSL_linrot_TouchStateProcess) refers to tsl_linrot.o(i.TSL_linrot_DTOGetTime) for TSL_linrot_DTOGetTime
    tsl_linrot.o(i.TSL_linrot_TouchStateProcess) refers to tsl_globals.o(.bss) for TSL_Globals
    tsl_linrot.o(i.TSL_linrot_TouchStateProcess) refers to tsl_user.o(.data) for TSL_Params
    tsl_object.o(i.TSL_obj_GroupInit) refers to tsl_object.o(i.TSL_obj_SetGlobalObj) for TSL_obj_SetGlobalObj
    tsl_object.o(i.TSL_obj_GroupInit) refers to tsl_globals.o(.bss) for TSL_Globals
    tsl_object.o(i.TSL_obj_GroupProcess) refers to tsl_object.o(i.TSL_obj_SetGlobalObj) for TSL_obj_SetGlobalObj
    tsl_object.o(i.TSL_obj_GroupProcess) refers to tsl_globals.o(.bss) for TSL_Globals
    tsl_object.o(i.TSL_obj_SetGlobalObj) refers to tsl_globals.o(.bss) for TSL_Globals
    tsl_time.o(i.TSL_tim_CheckDelay_ms) refers to tsl_globals.o(.bss) for TSL_Globals
    tsl_time.o(i.TSL_tim_CheckDelay_sec) refers to tsl_globals.o(.bss) for TSL_Globals
    tsl_time.o(i.TSL_tim_ProcessIT) refers to tsl_globals.o(.bss) for TSL_Globals
    tsl_time.o(i.TSL_tim_ProcessIT) refers to tsl_time.o(.data) for .data
    usbd_hid.o(i.USBD_HID_DeInit) refers to usbd_conf.o(i.USBD_LL_CloseEP) for USBD_LL_CloseEP
    usbd_hid.o(i.USBD_HID_DeInit) refers to usbd_conf.o(i.USBD_static_free) for USBD_static_free
    usbd_hid.o(i.USBD_HID_GetCfgDesc) refers to usbd_hid.o(.data) for .data
    usbd_hid.o(i.USBD_HID_GetDeviceQualifierDesc) refers to usbd_hid.o(.data) for .data
    usbd_hid.o(i.USBD_HID_Init) refers to usbd_conf.o(i.USBD_LL_OpenEP) for USBD_LL_OpenEP
    usbd_hid.o(i.USBD_HID_Init) refers to usbd_conf.o(i.USBD_static_malloc) for USBD_static_malloc
    usbd_hid.o(i.USBD_HID_SendReport) refers to usbd_conf.o(i.USBD_LL_Transmit) for USBD_LL_Transmit
    usbd_hid.o(i.USBD_HID_Setup) refers to usbd_ctlreq.o(i.USBD_CtlError) for USBD_CtlError
    usbd_hid.o(i.USBD_HID_Setup) refers to usbd_ioreq.o(i.USBD_CtlSendData) for USBD_CtlSendData
    usbd_hid.o(i.USBD_HID_Setup) refers to usbd_hid.o(.data) for .data
    usbd_hid.o(.data) refers to usbd_hid.o(i.USBD_HID_Init) for USBD_HID_Init
    usbd_hid.o(.data) refers to usbd_hid.o(i.USBD_HID_DeInit) for USBD_HID_DeInit
    usbd_hid.o(.data) refers to usbd_hid.o(i.USBD_HID_Setup) for USBD_HID_Setup
    usbd_hid.o(.data) refers to usbd_hid.o(i.USBD_HID_DataIn) for USBD_HID_DataIn
    usbd_hid.o(.data) refers to usbd_hid.o(i.USBD_HID_GetCfgDesc) for USBD_HID_GetCfgDesc
    usbd_hid.o(.data) refers to usbd_hid.o(i.USBD_HID_GetDeviceQualifierDesc) for USBD_HID_GetDeviceQualifierDesc
    usbd_core.o(i.USBD_DeInit) refers to usbd_conf.o(i.USBD_LL_Stop) for USBD_LL_Stop
    usbd_core.o(i.USBD_DeInit) refers to usbd_conf.o(i.USBD_LL_DeInit) for USBD_LL_DeInit
    usbd_core.o(i.USBD_Init) refers to usbd_conf.o(i.USBD_LL_Init) for USBD_LL_Init
    usbd_core.o(i.USBD_LL_DataInStage) refers to usbd_ioreq.o(i.USBD_CtlContinueSendData) for USBD_CtlContinueSendData
    usbd_core.o(i.USBD_LL_DataInStage) refers to uidiv.o(.text) for __aeabi_uidivmod
    usbd_core.o(i.USBD_LL_DataInStage) refers to usbd_ioreq.o(i.USBD_CtlReceiveStatus) for USBD_CtlReceiveStatus
    usbd_core.o(i.USBD_LL_DataOutStage) refers to usbd_ioreq.o(i.USBD_CtlContinueRx) for USBD_CtlContinueRx
    usbd_core.o(i.USBD_LL_DataOutStage) refers to usbd_ioreq.o(i.USBD_CtlSendStatus) for USBD_CtlSendStatus
    usbd_core.o(i.USBD_LL_Reset) refers to usbd_conf.o(i.USBD_LL_OpenEP) for USBD_LL_OpenEP
    usbd_core.o(i.USBD_LL_SetupStage) refers to usbd_ctlreq.o(i.USBD_ParseSetupRequest) for USBD_ParseSetupRequest
    usbd_core.o(i.USBD_LL_SetupStage) refers to usbd_conf.o(i.USBD_LL_StallEP) for USBD_LL_StallEP
    usbd_core.o(i.USBD_LL_SetupStage) refers to usbd_ctlreq.o(i.USBD_StdDevReq) for USBD_StdDevReq
    usbd_core.o(i.USBD_LL_SetupStage) refers to usbd_ctlreq.o(i.USBD_StdItfReq) for USBD_StdItfReq
    usbd_core.o(i.USBD_LL_SetupStage) refers to usbd_ctlreq.o(i.USBD_StdEPReq) for USBD_StdEPReq
    usbd_core.o(i.USBD_Start) refers to usbd_conf.o(i.USBD_LL_Start) for USBD_LL_Start
    usbd_core.o(i.USBD_Stop) refers to usbd_conf.o(i.USBD_LL_Stop) for USBD_LL_Stop
    usbd_ctlreq.o(i.USBD_CtlError) refers to usbd_conf.o(i.USBD_LL_StallEP) for USBD_LL_StallEP
    usbd_ctlreq.o(i.USBD_GetDescriptor) refers to menu.o(i.__ARM_common_switch8) for __ARM_common_switch8
    usbd_ctlreq.o(i.USBD_GetDescriptor) refers to usbd_ctlreq.o(i.USBD_CtlError) for USBD_CtlError
    usbd_ctlreq.o(i.USBD_GetDescriptor) refers to usbd_ioreq.o(i.USBD_CtlSendData) for USBD_CtlSendData
    usbd_ctlreq.o(i.USBD_SetConfig) refers to usbd_ctlreq.o(i.USBD_CtlError) for USBD_CtlError
    usbd_ctlreq.o(i.USBD_SetConfig) refers to usbd_core.o(i.USBD_ClrClassConfig) for USBD_ClrClassConfig
    usbd_ctlreq.o(i.USBD_SetConfig) refers to usbd_core.o(i.USBD_SetClassConfig) for USBD_SetClassConfig
    usbd_ctlreq.o(i.USBD_SetConfig) refers to usbd_ioreq.o(i.USBD_CtlSendStatus) for USBD_CtlSendStatus
    usbd_ctlreq.o(i.USBD_SetConfig) refers to usbd_ctlreq.o(.data) for .data
    usbd_ctlreq.o(i.USBD_StdDevReq) refers to menu.o(i.__ARM_common_switch8) for __ARM_common_switch8
    usbd_ctlreq.o(i.USBD_StdDevReq) refers to usbd_ctlreq.o(i.USBD_GetDescriptor) for USBD_GetDescriptor
    usbd_ctlreq.o(i.USBD_StdDevReq) refers to usbd_conf.o(i.USBD_LL_SetUSBAddress) for USBD_LL_SetUSBAddress
    usbd_ctlreq.o(i.USBD_StdDevReq) refers to usbd_ioreq.o(i.USBD_CtlSendStatus) for USBD_CtlSendStatus
    usbd_ctlreq.o(i.USBD_StdDevReq) refers to usbd_ctlreq.o(i.USBD_SetConfig) for USBD_SetConfig
    usbd_ctlreq.o(i.USBD_StdDevReq) refers to usbd_ctlreq.o(i.USBD_CtlError) for USBD_CtlError
    usbd_ctlreq.o(i.USBD_StdDevReq) refers to usbd_ioreq.o(i.USBD_CtlSendData) for USBD_CtlSendData
    usbd_ctlreq.o(i.USBD_StdEPReq) refers to usbd_conf.o(i.USBD_LL_StallEP) for USBD_LL_StallEP
    usbd_ctlreq.o(i.USBD_StdEPReq) refers to usbd_conf.o(i.USBD_LL_ClearStallEP) for USBD_LL_ClearStallEP
    usbd_ctlreq.o(i.USBD_StdEPReq) refers to usbd_ioreq.o(i.USBD_CtlSendStatus) for USBD_CtlSendStatus
    usbd_ctlreq.o(i.USBD_StdEPReq) refers to usbd_ctlreq.o(i.USBD_CtlError) for USBD_CtlError
    usbd_ctlreq.o(i.USBD_StdEPReq) refers to usbd_conf.o(i.USBD_LL_IsStallEP) for USBD_LL_IsStallEP
    usbd_ctlreq.o(i.USBD_StdEPReq) refers to usbd_ioreq.o(i.USBD_CtlSendData) for USBD_CtlSendData
    usbd_ctlreq.o(i.USBD_StdItfReq) refers to usbd_ioreq.o(i.USBD_CtlSendStatus) for USBD_CtlSendStatus
    usbd_ctlreq.o(i.USBD_StdItfReq) refers to usbd_ctlreq.o(i.USBD_CtlError) for USBD_CtlError
    usbd_ioreq.o(i.USBD_CtlContinueRx) refers to usbd_conf.o(i.USBD_LL_PrepareReceive) for USBD_LL_PrepareReceive
    usbd_ioreq.o(i.USBD_CtlContinueSendData) refers to usbd_conf.o(i.USBD_LL_Transmit) for USBD_LL_Transmit
    usbd_ioreq.o(i.USBD_CtlPrepareRx) refers to usbd_conf.o(i.USBD_LL_PrepareReceive) for USBD_LL_PrepareReceive
    usbd_ioreq.o(i.USBD_CtlReceiveStatus) refers to usbd_conf.o(i.USBD_LL_PrepareReceive) for USBD_LL_PrepareReceive
    usbd_ioreq.o(i.USBD_CtlSendData) refers to usbd_conf.o(i.USBD_LL_Transmit) for USBD_LL_Transmit
    usbd_ioreq.o(i.USBD_CtlSendStatus) refers to usbd_conf.o(i.USBD_LL_Transmit) for USBD_LL_Transmit
    usbd_ioreq.o(i.USBD_GetRxCount) refers to usbd_conf.o(i.USBD_LL_GetRxDataSize) for USBD_LL_GetRxDataSize
    entry.o(.ARM.Collect$$$$00000000) refers (Special) to entry10a.o(.ARM.Collect$$$$0000000D) for __rt_final_cpp
    entry.o(.ARM.Collect$$$$00000000) refers (Special) to entry11a.o(.ARM.Collect$$$$0000000F) for __rt_final_exit
    entry.o(.ARM.Collect$$$$00000000) refers (Special) to entry7b.o(.ARM.Collect$$$$00000008) for _main_clock
    entry.o(.ARM.Collect$$$$00000000) refers (Special) to entry8b.o(.ARM.Collect$$$$0000000A) for _main_cpp_init
    entry.o(.ARM.Collect$$$$00000000) refers (Special) to entry9a.o(.ARM.Collect$$$$0000000B) for _main_init
    entry.o(.ARM.Collect$$$$00000000) refers (Special) to entry5.o(.ARM.Collect$$$$00000004) for _main_scatterload
    entry.o(.ARM.Collect$$$$00000000) refers (Special) to entry2.o(.ARM.Collect$$$$00000001) for _main_stk
    idiv.o(.text) refers to uidiv.o(.text) for __aeabi_uidivmod
    printfb.o(i.__0fprintf$bare) refers to printfb.o(i._printf_core) for _printf_core
    printfb.o(i.__0fprintf$bare) refers to fputc.o(i.fputc) for fputc
    printfb.o(i.__0printf$bare) refers to printfb.o(i._printf_core) for _printf_core
    printfb.o(i.__0printf$bare) refers to fputc.o(i.fputc) for fputc
    printfb.o(i.__0printf$bare) refers to stdout.o(.data) for __stdout
    printfb.o(i.__0snprintf$bare) refers to printfb.o(i._printf_core) for _printf_core
    printfb.o(i.__0snprintf$bare) refers to printfb.o(i._snputc) for _snputc
    printfb.o(i.__0sprintf$bare) refers to printfb.o(i._printf_core) for _printf_core
    printfb.o(i.__0sprintf$bare) refers to printfb.o(i._sputc) for _sputc
    printfb.o(i.__0vfprintf$bare) refers to printfb.o(i._printf_core) for _printf_core
    printfb.o(i.__0vfprintf$bare) refers to fputc.o(i.fputc) for fputc
    printfb.o(i.__0vprintf$bare) refers to printfb.o(i._printf_core) for _printf_core
    printfb.o(i.__0vprintf$bare) refers to fputc.o(i.fputc) for fputc
    printfb.o(i.__0vprintf$bare) refers to stdout.o(.data) for __stdout
    printfb.o(i.__0vsnprintf$bare) refers to printfb.o(i._printf_core) for _printf_core
    printfb.o(i.__0vsnprintf$bare) refers to printfb.o(i._snputc) for _snputc
    printfb.o(i.__0vsprintf$bare) refers to printfb.o(i._printf_core) for _printf_core
    printfb.o(i.__0vsprintf$bare) refers to printfb.o(i._sputc) for _sputc
    printf0.o(i.__0fprintf$0) refers to printf0.o(i._printf_core) for _printf_core
    printf0.o(i.__0fprintf$0) refers to fputc.o(i.fputc) for fputc
    printf0.o(i.__0printf$0) refers to printf0.o(i._printf_core) for _printf_core
    printf0.o(i.__0printf$0) refers to fputc.o(i.fputc) for fputc
    printf0.o(i.__0printf$0) refers to stdout.o(.data) for __stdout
    printf0.o(i.__0snprintf$0) refers to printf0.o(i._printf_core) for _printf_core
    printf0.o(i.__0snprintf$0) refers to printf0.o(i._snputc) for _snputc
    printf0.o(i.__0sprintf$0) refers to printf0.o(i._printf_core) for _printf_core
    printf0.o(i.__0sprintf$0) refers to printf0.o(i._sputc) for _sputc
    printf0.o(i.__0vfprintf$0) refers to printf0.o(i._printf_core) for _printf_core
    printf0.o(i.__0vfprintf$0) refers to fputc.o(i.fputc) for fputc
    printf0.o(i.__0vprintf$0) refers to printf0.o(i._printf_core) for _printf_core
    printf0.o(i.__0vprintf$0) refers to fputc.o(i.fputc) for fputc
    printf0.o(i.__0vprintf$0) refers to stdout.o(.data) for __stdout
    printf0.o(i.__0vsnprintf$0) refers to printf0.o(i._printf_core) for _printf_core
    printf0.o(i.__0vsnprintf$0) refers to printf0.o(i._snputc) for _snputc
    printf0.o(i.__0vsprintf$0) refers to printf0.o(i._printf_core) for _printf_core
    printf0.o(i.__0vsprintf$0) refers to printf0.o(i._sputc) for _sputc
    printf1.o(i.__0fprintf$1) refers to printf1.o(i._printf_core) for _printf_core
    printf1.o(i.__0fprintf$1) refers to fputc.o(i.fputc) for fputc
    printf1.o(i.__0printf$1) refers to printf1.o(i._printf_core) for _printf_core
    printf1.o(i.__0printf$1) refers to fputc.o(i.fputc) for fputc
    printf1.o(i.__0printf$1) refers to stdout.o(.data) for __stdout
    printf1.o(i.__0snprintf$1) refers to printf1.o(i._printf_core) for _printf_core
    printf1.o(i.__0snprintf$1) refers to printf1.o(i._snputc) for _snputc
    printf1.o(i.__0sprintf$1) refers to printf1.o(i._printf_core) for _printf_core
    printf1.o(i.__0sprintf$1) refers to printf1.o(i._sputc) for _sputc
    printf1.o(i.__0vfprintf$1) refers to printf1.o(i._printf_core) for _printf_core
    printf1.o(i.__0vfprintf$1) refers to fputc.o(i.fputc) for fputc
    printf1.o(i.__0vprintf$1) refers to printf1.o(i._printf_core) for _printf_core
    printf1.o(i.__0vprintf$1) refers to fputc.o(i.fputc) for fputc
    printf1.o(i.__0vprintf$1) refers to stdout.o(.data) for __stdout
    printf1.o(i.__0vsnprintf$1) refers to printf1.o(i._printf_core) for _printf_core
    printf1.o(i.__0vsnprintf$1) refers to printf1.o(i._snputc) for _snputc
    printf1.o(i.__0vsprintf$1) refers to printf1.o(i._printf_core) for _printf_core
    printf1.o(i.__0vsprintf$1) refers to printf1.o(i._sputc) for _sputc
    printf1.o(i._printf_core) refers to uidiv.o(.text) for __aeabi_uidivmod
    printf2.o(i.__0fprintf$2) refers to printf2.o(i._printf_core) for _printf_core
    printf2.o(i.__0fprintf$2) refers to fputc.o(i.fputc) for fputc
    printf2.o(i.__0printf$2) refers to printf2.o(i._printf_core) for _printf_core
    printf2.o(i.__0printf$2) refers to fputc.o(i.fputc) for fputc
    printf2.o(i.__0printf$2) refers to stdout.o(.data) for __stdout
    printf2.o(i.__0snprintf$2) refers to printf2.o(i._printf_core) for _printf_core
    printf2.o(i.__0snprintf$2) refers to printf2.o(i._snputc) for _snputc
    printf2.o(i.__0sprintf$2) refers to printf2.o(i._printf_core) for _printf_core
    printf2.o(i.__0sprintf$2) refers to printf2.o(i._sputc) for _sputc
    printf2.o(i.__0vfprintf$2) refers to printf2.o(i._printf_core) for _printf_core
    printf2.o(i.__0vfprintf$2) refers to fputc.o(i.fputc) for fputc
    printf2.o(i.__0vprintf$2) refers to printf2.o(i._printf_core) for _printf_core
    printf2.o(i.__0vprintf$2) refers to fputc.o(i.fputc) for fputc
    printf2.o(i.__0vprintf$2) refers to stdout.o(.data) for __stdout
    printf2.o(i.__0vsnprintf$2) refers to printf2.o(i._printf_core) for _printf_core
    printf2.o(i.__0vsnprintf$2) refers to printf2.o(i._snputc) for _snputc
    printf2.o(i.__0vsprintf$2) refers to printf2.o(i._printf_core) for _printf_core
    printf2.o(i.__0vsprintf$2) refers to printf2.o(i._sputc) for _sputc
    printf3.o(i.__0fprintf$3) refers to printf3.o(i._printf_core) for _printf_core
    printf3.o(i.__0fprintf$3) refers to fputc.o(i.fputc) for fputc
    printf3.o(i.__0printf$3) refers to printf3.o(i._printf_core) for _printf_core
    printf3.o(i.__0printf$3) refers to fputc.o(i.fputc) for fputc
    printf3.o(i.__0printf$3) refers to stdout.o(.data) for __stdout
    printf3.o(i.__0snprintf$3) refers to printf3.o(i._printf_core) for _printf_core
    printf3.o(i.__0snprintf$3) refers to printf3.o(i._snputc) for _snputc
    printf3.o(i.__0sprintf$3) refers to printf3.o(i._printf_core) for _printf_core
    printf3.o(i.__0sprintf$3) refers to printf3.o(i._sputc) for _sputc
    printf3.o(i.__0vfprintf$3) refers to printf3.o(i._printf_core) for _printf_core
    printf3.o(i.__0vfprintf$3) refers to fputc.o(i.fputc) for fputc
    printf3.o(i.__0vprintf$3) refers to printf3.o(i._printf_core) for _printf_core
    printf3.o(i.__0vprintf$3) refers to fputc.o(i.fputc) for fputc
    printf3.o(i.__0vprintf$3) refers to stdout.o(.data) for __stdout
    printf3.o(i.__0vsnprintf$3) refers to printf3.o(i._printf_core) for _printf_core
    printf3.o(i.__0vsnprintf$3) refers to printf3.o(i._snputc) for _snputc
    printf3.o(i.__0vsprintf$3) refers to printf3.o(i._printf_core) for _printf_core
    printf3.o(i.__0vsprintf$3) refers to printf3.o(i._sputc) for _sputc
    printf3.o(i._printf_core) refers to uidiv.o(.text) for __aeabi_uidivmod
    printf4.o(i.__0fprintf$4) refers to printf4.o(i._printf_core) for _printf_core
    printf4.o(i.__0fprintf$4) refers to fputc.o(i.fputc) for fputc
    printf4.o(i.__0printf$4) refers to printf4.o(i._printf_core) for _printf_core
    printf4.o(i.__0printf$4) refers to fputc.o(i.fputc) for fputc
    printf4.o(i.__0printf$4) refers to stdout.o(.data) for __stdout
    printf4.o(i.__0snprintf$4) refers to printf4.o(i._printf_core) for _printf_core
    printf4.o(i.__0snprintf$4) refers to printf4.o(i._snputc) for _snputc
    printf4.o(i.__0sprintf$4) refers to printf4.o(i._printf_core) for _printf_core
    printf4.o(i.__0sprintf$4) refers to printf4.o(i._sputc) for _sputc
    printf4.o(i.__0vfprintf$4) refers to printf4.o(i._printf_core) for _printf_core
    printf4.o(i.__0vfprintf$4) refers to fputc.o(i.fputc) for fputc
    printf4.o(i.__0vprintf$4) refers to printf4.o(i._printf_core) for _printf_core
    printf4.o(i.__0vprintf$4) refers to fputc.o(i.fputc) for fputc
    printf4.o(i.__0vprintf$4) refers to stdout.o(.data) for __stdout
    printf4.o(i.__0vsnprintf$4) refers to printf4.o(i._printf_core) for _printf_core
    printf4.o(i.__0vsnprintf$4) refers to printf4.o(i._snputc) for _snputc
    printf4.o(i.__0vsprintf$4) refers to printf4.o(i._printf_core) for _printf_core
    printf4.o(i.__0vsprintf$4) refers to printf4.o(i._sputc) for _sputc
    printf4.o(i._printf_core) refers to uldiv.o(.text) for __aeabi_uldivmod
    printf5.o(i.__0fprintf$5) refers to printf5.o(i._printf_core) for _printf_core
    printf5.o(i.__0fprintf$5) refers to fputc.o(i.fputc) for fputc
    printf5.o(i.__0printf$5) refers to printf5.o(i._printf_core) for _printf_core
    printf5.o(i.__0printf$5) refers to fputc.o(i.fputc) for fputc
    printf5.o(i.__0printf$5) refers to stdout.o(.data) for __stdout
    printf5.o(i.__0snprintf$5) refers to printf5.o(i._printf_core) for _printf_core
    printf5.o(i.__0snprintf$5) refers to printf5.o(i._snputc) for _snputc
    printf5.o(i.__0sprintf$5) refers to printf5.o(i._printf_core) for _printf_core
    printf5.o(i.__0sprintf$5) refers to printf5.o(i._sputc) for _sputc
    printf5.o(i.__0vfprintf$5) refers to printf5.o(i._printf_core) for _printf_core
    printf5.o(i.__0vfprintf$5) refers to fputc.o(i.fputc) for fputc
    printf5.o(i.__0vprintf$5) refers to printf5.o(i._printf_core) for _printf_core
    printf5.o(i.__0vprintf$5) refers to fputc.o(i.fputc) for fputc
    printf5.o(i.__0vprintf$5) refers to stdout.o(.data) for __stdout
    printf5.o(i.__0vsnprintf$5) refers to printf5.o(i._printf_core) for _printf_core
    printf5.o(i.__0vsnprintf$5) refers to printf5.o(i._snputc) for _snputc
    printf5.o(i.__0vsprintf$5) refers to printf5.o(i._printf_core) for _printf_core
    printf5.o(i.__0vsprintf$5) refers to printf5.o(i._sputc) for _sputc
    printf5.o(i._printf_core) refers to uldiv.o(.text) for __aeabi_uldivmod
    printf6.o(i.__0fprintf$6) refers to printf6.o(i._printf_core) for _printf_core
    printf6.o(i.__0fprintf$6) refers to fputc.o(i.fputc) for fputc
    printf6.o(i.__0printf$6) refers to printf6.o(i._printf_core) for _printf_core
    printf6.o(i.__0printf$6) refers to fputc.o(i.fputc) for fputc
    printf6.o(i.__0printf$6) refers to stdout.o(.data) for __stdout
    printf6.o(i.__0snprintf$6) refers to printf6.o(i._printf_core) for _printf_core
    printf6.o(i.__0snprintf$6) refers to printf6.o(i._snputc) for _snputc
    printf6.o(i.__0sprintf$6) refers to printf6.o(i._printf_core) for _printf_core
    printf6.o(i.__0sprintf$6) refers to printf6.o(i._sputc) for _sputc
    printf6.o(i.__0vfprintf$6) refers to printf6.o(i._printf_core) for _printf_core
    printf6.o(i.__0vfprintf$6) refers to fputc.o(i.fputc) for fputc
    printf6.o(i.__0vprintf$6) refers to printf6.o(i._printf_core) for _printf_core
    printf6.o(i.__0vprintf$6) refers to fputc.o(i.fputc) for fputc
    printf6.o(i.__0vprintf$6) refers to stdout.o(.data) for __stdout
    printf6.o(i.__0vsnprintf$6) refers to printf6.o(i._printf_core) for _printf_core
    printf6.o(i.__0vsnprintf$6) refers to printf6.o(i._snputc) for _snputc
    printf6.o(i.__0vsprintf$6) refers to printf6.o(i._printf_core) for _printf_core
    printf6.o(i.__0vsprintf$6) refers to printf6.o(i._sputc) for _sputc
    printf6.o(i._printf_core) refers to printf6.o(i._printf_pre_padding) for _printf_pre_padding
    printf6.o(i._printf_core) refers to printf6.o(i._printf_post_padding) for _printf_post_padding
    printf6.o(i._printf_core) refers to uidiv.o(.text) for __aeabi_uidivmod
    printf7.o(i.__0fprintf$7) refers to printf7.o(i._printf_core) for _printf_core
    printf7.o(i.__0fprintf$7) refers to fputc.o(i.fputc) for fputc
    printf7.o(i.__0printf$7) refers to printf7.o(i._printf_core) for _printf_core
    printf7.o(i.__0printf$7) refers to fputc.o(i.fputc) for fputc
    printf7.o(i.__0printf$7) refers to stdout.o(.data) for __stdout
    printf7.o(i.__0snprintf$7) refers to printf7.o(i._printf_core) for _printf_core
    printf7.o(i.__0snprintf$7) refers to printf7.o(i._snputc) for _snputc
    printf7.o(i.__0sprintf$7) refers to printf7.o(i._printf_core) for _printf_core
    printf7.o(i.__0sprintf$7) refers to printf7.o(i._sputc) for _sputc
    printf7.o(i.__0vfprintf$7) refers to printf7.o(i._printf_core) for _printf_core
    printf7.o(i.__0vfprintf$7) refers to fputc.o(i.fputc) for fputc
    printf7.o(i.__0vprintf$7) refers to printf7.o(i._printf_core) for _printf_core
    printf7.o(i.__0vprintf$7) refers to fputc.o(i.fputc) for fputc
    printf7.o(i.__0vprintf$7) refers to stdout.o(.data) for __stdout
    printf7.o(i.__0vsnprintf$7) refers to printf7.o(i._printf_core) for _printf_core
    printf7.o(i.__0vsnprintf$7) refers to printf7.o(i._snputc) for _snputc
    printf7.o(i.__0vsprintf$7) refers to printf7.o(i._printf_core) for _printf_core
    printf7.o(i.__0vsprintf$7) refers to printf7.o(i._sputc) for _sputc
    printf7.o(i._printf_core) refers to printf7.o(i._printf_pre_padding) for _printf_pre_padding
    printf7.o(i._printf_core) refers to printf7.o(i._printf_post_padding) for _printf_post_padding
    printf7.o(i._printf_core) refers to uldiv.o(.text) for __aeabi_uldivmod
    printf8.o(i.__0fprintf$8) refers to printf8.o(i._printf_core) for _printf_core
    printf8.o(i.__0fprintf$8) refers to fputc.o(i.fputc) for fputc
    printf8.o(i.__0printf$8) refers to printf8.o(i._printf_core) for _printf_core
    printf8.o(i.__0printf$8) refers to fputc.o(i.fputc) for fputc
    printf8.o(i.__0printf$8) refers to stdout.o(.data) for __stdout
    printf8.o(i.__0snprintf$8) refers to printf8.o(i._printf_core) for _printf_core
    printf8.o(i.__0snprintf$8) refers to printf8.o(i._snputc) for _snputc
    printf8.o(i.__0sprintf$8) refers to printf8.o(i._printf_core) for _printf_core
    printf8.o(i.__0sprintf$8) refers to printf8.o(i._sputc) for _sputc
    printf8.o(i.__0vfprintf$8) refers to printf8.o(i._printf_core) for _printf_core
    printf8.o(i.__0vfprintf$8) refers to fputc.o(i.fputc) for fputc
    printf8.o(i.__0vprintf$8) refers to printf8.o(i._printf_core) for _printf_core
    printf8.o(i.__0vprintf$8) refers to fputc.o(i.fputc) for fputc
    printf8.o(i.__0vprintf$8) refers to stdout.o(.data) for __stdout
    printf8.o(i.__0vsnprintf$8) refers to printf8.o(i._printf_core) for _printf_core
    printf8.o(i.__0vsnprintf$8) refers to printf8.o(i._snputc) for _snputc
    printf8.o(i.__0vsprintf$8) refers to printf8.o(i._printf_core) for _printf_core
    printf8.o(i.__0vsprintf$8) refers to printf8.o(i._sputc) for _sputc
    printf8.o(i._printf_core) refers to printf8.o(i._printf_pre_padding) for _printf_pre_padding
    printf8.o(i._printf_core) refers to printf8.o(i._printf_post_padding) for _printf_post_padding
    printf8.o(i._printf_core) refers to uldiv.o(.text) for __aeabi_uldivmod
    printfa.o(i.__0fprintf) refers (Special) to iusefp.o(.text) for __I$use$fp
    printfa.o(i.__0fprintf) refers to printfa.o(i._printf_core) for _printf_core
    printfa.o(i.__0fprintf) refers to fputc.o(i.fputc) for fputc
    printfa.o(i.__0printf) refers (Special) to iusefp.o(.text) for __I$use$fp
    printfa.o(i.__0printf) refers to printfa.o(i._printf_core) for _printf_core
    printfa.o(i.__0printf) refers to fputc.o(i.fputc) for fputc
    printfa.o(i.__0printf) refers to stdout.o(.data) for __stdout
    printfa.o(i.__0snprintf) refers (Special) to iusefp.o(.text) for __I$use$fp
    printfa.o(i.__0snprintf) refers to printfa.o(i._printf_core) for _printf_core
    printfa.o(i.__0snprintf) refers to printfa.o(i._snputc) for _snputc
    printfa.o(i.__0sprintf) refers (Special) to iusefp.o(.text) for __I$use$fp
    printfa.o(i.__0sprintf) refers to printfa.o(i._printf_core) for _printf_core
    printfa.o(i.__0sprintf) refers to printfa.o(i._sputc) for _sputc
    printfa.o(i.__0vfprintf) refers (Special) to iusefp.o(.text) for __I$use$fp
    printfa.o(i.__0vfprintf) refers to printfa.o(i._printf_core) for _printf_core
    printfa.o(i.__0vfprintf) refers to fputc.o(i.fputc) for fputc
    printfa.o(i.__0vprintf) refers (Special) to iusefp.o(.text) for __I$use$fp
    printfa.o(i.__0vprintf) refers to printfa.o(i._printf_core) for _printf_core
    printfa.o(i.__0vprintf) refers to fputc.o(i.fputc) for fputc
    printfa.o(i.__0vprintf) refers to stdout.o(.data) for __stdout
    printfa.o(i.__0vsnprintf) refers (Special) to iusefp.o(.text) for __I$use$fp
    printfa.o(i.__0vsnprintf) refers to printfa.o(i._printf_core) for _printf_core
    printfa.o(i.__0vsnprintf) refers to printfa.o(i._snputc) for _snputc
    printfa.o(i.__0vsprintf) refers (Special) to iusefp.o(.text) for __I$use$fp
    printfa.o(i.__0vsprintf) refers to printfa.o(i._printf_core) for _printf_core
    printfa.o(i.__0vsprintf) refers to printfa.o(i._sputc) for _sputc
    printfa.o(i._fp_digits) refers (Special) to iusefp.o(.text) for __I$use$fp
    printfa.o(i._fp_digits) refers to dmul.o(.text) for __aeabi_dmul
    printfa.o(i._fp_digits) refers to ddiv.o(.text) for __aeabi_ddiv
    printfa.o(i._fp_digits) refers to cdrcmple.o(.text) for __aeabi_cdrcmple
    printfa.o(i._fp_digits) refers to dadd.o(.text) for __aeabi_dadd
    printfa.o(i._fp_digits) refers to dfixul.o(.text) for __aeabi_d2ulz
    printfa.o(i._fp_digits) refers to uldiv.o(.text) for __aeabi_uldivmod
    printfa.o(i._printf_core) refers (Special) to iusefp.o(.text) for __I$use$fp
    printfa.o(i._printf_core) refers to printfa.o(i._printf_pre_padding) for _printf_pre_padding
    printfa.o(i._printf_core) refers to uldiv.o(.text) for __aeabi_uldivmod
    printfa.o(i._printf_core) refers to printfa.o(i._printf_post_padding) for _printf_post_padding
    printfa.o(i._printf_core) refers to printfa.o(i._fp_digits) for _fp_digits
    printfa.o(i._printf_core) refers to uidiv.o(.text) for __aeabi_uidivmod
    printfa.o(i._printf_post_padding) refers (Special) to iusefp.o(.text) for __I$use$fp
    printfa.o(i._printf_pre_padding) refers (Special) to iusefp.o(.text) for __I$use$fp
    printfa.o(i._snputc) refers (Special) to iusefp.o(.text) for __I$use$fp
    printfa.o(i._sputc) refers (Special) to iusefp.o(.text) for __I$use$fp
    entry2.o(.ARM.Collect$$$$00000001) refers to entry2.o(.ARM.Collect$$$$00002712) for __lit__00000000
    entry2.o(.ARM.Collect$$$$00002712) refers to startup_stm32l053xx.o(STACK) for __initial_sp
    entry2.o(__vectab_stack_and_reset_area) refers to startup_stm32l053xx.o(STACK) for __initial_sp
    entry2.o(__vectab_stack_and_reset_area) refers to entry.o(.ARM.Collect$$$$00000000) for __main
    entry5.o(.ARM.Collect$$$$00000004) refers to init.o(.text) for __scatterload
    entry9a.o(.ARM.Collect$$$$0000000B) refers to main.o(i.main) for main
    entry9b.o(.ARM.Collect$$$$0000000C) refers to main.o(i.main) for main
    fputc.o(i.fputc) refers (Special) to iusesemip.o(.text) for __I$use$semihosting$fputc
    fputc.o(i.fputc) refers (Special) to semi.o(.text) for __semihosting_library_function
    uldiv.o(.text) refers to llushr.o(.text) for __aeabi_llsr
    uldiv.o(.text) refers to llshl.o(.text) for __aeabi_llsl
    dadd.o(.text) refers to llshl.o(.text) for __aeabi_llsl
    dadd.o(.text) refers to llsshr.o(.text) for __aeabi_lasr
    dadd.o(.text) refers to depilogue.o(.text) for _double_epilogue
    dmul.o(.text) refers to depilogue.o(.text) for _double_epilogue
    ddiv.o(.text) refers to depilogue.o(.text) for _double_round
    dfixul.o(.text) refers to llushr.o(.text) for __aeabi_llsr
    dfixul.o(.text) refers to llshl.o(.text) for __aeabi_llsl
    init.o(.text) refers to entry5.o(.ARM.Collect$$$$00000004) for __main_after_scatterload
    depilogue.o(.text) refers to depilogue.o(i.__ARM_clz) for __ARM_clz
    depilogue.o(.text) refers to llshl.o(.text) for __aeabi_llsl
    depilogue.o(.text) refers to llushr.o(.text) for __aeabi_llsr


==============================================================================

Removing Unused input sections from the image.

    Removing startup_stm32l053xx.o(HEAP), (2048 bytes).
    Removing bsp.o(.rev16_text), (4 bytes).
    Removing bsp.o(.revsh_text), (4 bytes).
    Removing main.o(.rev16_text), (4 bytes).
    Removing main.o(.revsh_text), (4 bytes).
    Removing menu.o(.rev16_text), (4 bytes).
    Removing menu.o(.revsh_text), (4 bytes).
    Removing stm32l0xx_hal_msp.o(.rev16_text), (4 bytes).
    Removing stm32l0xx_hal_msp.o(.revsh_text), (4 bytes).
    Removing stm32l0xx_hal_msp.o(i.HAL_MspDeInit), (2 bytes).
    Removing stm32l0xx_it.o(.rev16_text), (4 bytes).
    Removing stm32l0xx_it.o(.revsh_text), (4 bytes).
    Removing tsl_user.o(.rev16_text), (4 bytes).
    Removing tsl_user.o(.revsh_text), (4 bytes).
    Removing tsl_user.o(i.tsl_user_SetThresholds), (2 bytes).
    Removing power.o(.rev16_text), (4 bytes).
    Removing power.o(.revsh_text), (4 bytes).
    Removing power.o(i.Idd_Stop_process), (524 bytes).
    Removing usbd_conf.o(.rev16_text), (4 bytes).
    Removing usbd_conf.o(.revsh_text), (4 bytes).
    Removing usbd_conf.o(i.HAL_PCD_ConnectCallback), (14 bytes).
    Removing usbd_conf.o(i.HAL_PCD_DisconnectCallback), (14 bytes).
    Removing usbd_conf.o(i.HAL_PCD_ISOINIncompleteCallback), (14 bytes).
    Removing usbd_conf.o(i.HAL_PCD_ISOOUTIncompleteCallback), (14 bytes).
    Removing usbd_conf.o(i.USBD_LL_Delay), (8 bytes).
    Removing usbd_conf.o(i.USBD_LL_FlushEP), (18 bytes).
    Removing usbd_conf.o(i.USBD_LL_GetRxDataSize), (16 bytes).
    Removing usbd_desc.o(.rev16_text), (4 bytes).
    Removing usbd_desc.o(.revsh_text), (4 bytes).
    Removing usbdapp.o(.rev16_text), (4 bytes).
    Removing usbdapp.o(.revsh_text), (4 bytes).
    Removing gde021a1.o(i.gde021a1_ReadReg), (14 bytes).
    Removing gde021a1.o(i.gde021a1_WriteReg), (16 bytes).
    Removing stm32l0538_discovery.o(.rev16_text), (4 bytes).
    Removing stm32l0538_discovery.o(.revsh_text), (4 bytes).
    Removing stm32l0538_discovery.o(i.BSP_GetVersion), (6 bytes).
    Removing stm32l0538_discovery.o(i.BSP_LED_On), (32 bytes).
    Removing stm32l0538_discovery.o(i.BSP_PB_GetState), (28 bytes).
    Removing stm32l0538_discovery.o(i.EPD_IO_ReadData), (72 bytes).
    Removing stm32l0538_discovery_epd.o(.rev16_text), (4 bytes).
    Removing stm32l0538_discovery_epd.o(.revsh_text), (4 bytes).
    Removing stm32l0538_discovery_epd.o(i.BSP_EPD_CloseChargePump), (24 bytes).
    Removing stm32l0538_discovery_epd.o(i.BSP_EPD_DisplayStringAtLine), (28 bytes).
    Removing stm32l0538_discovery_epd.o(i.BSP_EPD_FillRect), (48 bytes).
    Removing stm32l0538_discovery_epd.o(i.BSP_EPD_GetFont), (12 bytes).
    Removing stm32l0538_discovery_epd.o(.constdata), (6650 bytes).
    Removing stm32l0538_discovery_epd.o(.data), (8 bytes).
    Removing system_stm32l0xx.o(.rev16_text), (4 bytes).
    Removing system_stm32l0xx.o(.revsh_text), (4 bytes).
    Removing system_stm32l0xx.o(i.SystemCoreClockUpdate), (148 bytes).
    Removing stm32l0xx_hal.o(.rev16_text), (4 bytes).
    Removing stm32l0xx_hal.o(.revsh_text), (4 bytes).
    Removing stm32l0xx_hal.o(i.HAL_ADC_EnableBufferSensor_Cmd), (32 bytes).
    Removing stm32l0xx_hal.o(i.HAL_ADC_EnableBuffer_Cmd), (28 bytes).
    Removing stm32l0xx_hal.o(i.HAL_COMP_EnableBuffer_Cmd), (32 bytes).
    Removing stm32l0xx_hal.o(i.HAL_DBG_LowPowerConfig), (24 bytes).
    Removing stm32l0xx_hal.o(i.HAL_DeInit), (40 bytes).
    Removing stm32l0xx_hal.o(i.HAL_DisableDBGSleepMode), (16 bytes).
    Removing stm32l0xx_hal.o(i.HAL_DisableDBGStandbyMode), (16 bytes).
    Removing stm32l0xx_hal.o(i.HAL_DisableDBGStopMode), (16 bytes).
    Removing stm32l0xx_hal.o(i.HAL_EnableDBGSleepMode), (16 bytes).
    Removing stm32l0xx_hal.o(i.HAL_EnableDBGStandbyMode), (16 bytes).
    Removing stm32l0xx_hal.o(i.HAL_EnableDBGStopMode), (16 bytes).
    Removing stm32l0xx_hal.o(i.HAL_GetBootMode), (16 bytes).
    Removing stm32l0xx_hal.o(i.HAL_GetDEVID), (16 bytes).
    Removing stm32l0xx_hal.o(i.HAL_GetHalVersion), (8 bytes).
    Removing stm32l0xx_hal.o(i.HAL_GetREVID), (12 bytes).
    Removing stm32l0xx_hal.o(i.HAL_I2CFastModePlusConfig), (24 bytes).
    Removing stm32l0xx_hal.o(i.HAL_Lock_Cmd), (28 bytes).
    Removing stm32l0xx_hal.o(i.HAL_MspDeInit), (2 bytes).
    Removing stm32l0xx_hal.o(i.HAL_MspInit), (2 bytes).
    Removing stm32l0xx_hal.o(i.HAL_RC48_EnableBuffer_Cmd), (32 bytes).
    Removing stm32l0xx_hal.o(i.HAL_VREFINT_Cmd), (28 bytes).
    Removing stm32l0xx_hal.o(i.HAL_VREFINT_OutputSelect), (24 bytes).
    Removing stm32l0xx_hal_cortex.o(.rev16_text), (4 bytes).
    Removing stm32l0xx_hal_cortex.o(.revsh_text), (4 bytes).
    Removing stm32l0xx_hal_cortex.o(i.HAL_NVIC_ClearPendingIRQ), (20 bytes).
    Removing stm32l0xx_hal_cortex.o(i.HAL_NVIC_GetPendingIRQ), (28 bytes).
    Removing stm32l0xx_hal_cortex.o(i.HAL_NVIC_SetPendingIRQ), (20 bytes).
    Removing stm32l0xx_hal_cortex.o(i.HAL_NVIC_SystemReset), (24 bytes).
    Removing stm32l0xx_hal_cortex.o(i.HAL_SYSTICK_CLKSourceConfig), (24 bytes).
    Removing stm32l0xx_hal_cortex.o(i.HAL_SYSTICK_Callback), (2 bytes).
    Removing stm32l0xx_hal_cortex.o(i.HAL_SYSTICK_IRQHandler), (8 bytes).
    Removing stm32l0xx_hal_dma.o(.rev16_text), (4 bytes).
    Removing stm32l0xx_hal_dma.o(.revsh_text), (4 bytes).
    Removing stm32l0xx_hal_dma.o(i.DMA_SetConfig), (30 bytes).
    Removing stm32l0xx_hal_dma.o(i.HAL_DMA_Abort), (76 bytes).
    Removing stm32l0xx_hal_dma.o(i.HAL_DMA_DeInit), (468 bytes).
    Removing stm32l0xx_hal_dma.o(i.HAL_DMA_GetError), (4 bytes).
    Removing stm32l0xx_hal_dma.o(i.HAL_DMA_GetState), (6 bytes).
    Removing stm32l0xx_hal_dma.o(i.HAL_DMA_IRQHandler), (640 bytes).
    Removing stm32l0xx_hal_dma.o(i.HAL_DMA_Init), (252 bytes).
    Removing stm32l0xx_hal_dma.o(i.HAL_DMA_PollForTransfer), (616 bytes).
    Removing stm32l0xx_hal_dma.o(i.HAL_DMA_Start), (50 bytes).
    Removing stm32l0xx_hal_dma.o(i.HAL_DMA_Start_IT), (78 bytes).
    Removing stm32l0xx_hal_flash.o(.rev16_text), (4 bytes).
    Removing stm32l0xx_hal_flash.o(.revsh_text), (4 bytes).
    Removing stm32l0xx_hal_flash.o(i.FLASH_Erase_Page), (28 bytes).
    Removing stm32l0xx_hal_flash.o(i.FLASH_Program_Word), (20 bytes).
    Removing stm32l0xx_hal_flash.o(i.FLASH_SetErrorCode), (84 bytes).
    Removing stm32l0xx_hal_flash.o(i.FLASH_WaitForLastOperation), (108 bytes).
    Removing stm32l0xx_hal_flash.o(i.HAL_FLASH_EndOfOperationCallback), (2 bytes).
    Removing stm32l0xx_hal_flash.o(i.HAL_FLASH_GetError), (12 bytes).
    Removing stm32l0xx_hal_flash.o(i.HAL_FLASH_IRQHandler), (248 bytes).
    Removing stm32l0xx_hal_flash.o(i.HAL_FLASH_Lock), (20 bytes).
    Removing stm32l0xx_hal_flash.o(i.HAL_FLASH_OB_Launch), (32 bytes).
    Removing stm32l0xx_hal_flash.o(i.HAL_FLASH_OB_Lock), (20 bytes).
    Removing stm32l0xx_hal_flash.o(i.HAL_FLASH_OB_Unlock), (60 bytes).
    Removing stm32l0xx_hal_flash.o(i.HAL_FLASH_OperationErrorCallback), (2 bytes).
    Removing stm32l0xx_hal_flash.o(i.HAL_FLASH_Program), (84 bytes).
    Removing stm32l0xx_hal_flash.o(i.HAL_FLASH_Program_IT), (84 bytes).
    Removing stm32l0xx_hal_flash.o(i.HAL_FLASH_Unlock), (60 bytes).
    Removing stm32l0xx_hal_flash.o(.bss), (20 bytes).
    Removing stm32l0xx_hal_flash_ex.o(.rev16_text), (4 bytes).
    Removing stm32l0xx_hal_flash_ex.o(.revsh_text), (4 bytes).
    Removing stm32l0xx_hal_flash_ex.o(i.FLASH_OB_PCROPConfig), (64 bytes).
    Removing stm32l0xx_hal_flash_ex.o(i.FLASH_OB_PCROPSelectionConfig), (44 bytes).
    Removing stm32l0xx_hal_flash_ex.o(i.FLASH_OB_WRPConfig), (64 bytes).
    Removing stm32l0xx_hal_flash_ex.o(i.HAL_FLASHEx_AdvOBGetConfig), (36 bytes).
    Removing stm32l0xx_hal_flash_ex.o(i.HAL_FLASHEx_AdvOBProgram), (104 bytes).
    Removing stm32l0xx_hal_flash_ex.o(i.HAL_FLASHEx_DATAEEPROM_Erase), (22 bytes).
    Removing stm32l0xx_hal_flash_ex.o(i.HAL_FLASHEx_DATAEEPROM_Lock), (20 bytes).
    Removing stm32l0xx_hal_flash_ex.o(i.HAL_FLASHEx_DATAEEPROM_Program), (264 bytes).
    Removing stm32l0xx_hal_flash_ex.o(i.HAL_FLASHEx_DATAEEPROM_Unlock), (36 bytes).
    Removing stm32l0xx_hal_flash_ex.o(i.HAL_FLASHEx_Erase), (120 bytes).
    Removing stm32l0xx_hal_flash_ex.o(i.HAL_FLASHEx_Erase_IT), (84 bytes).
    Removing stm32l0xx_hal_flash_ex.o(i.HAL_FLASHEx_OBGetConfig), (44 bytes).
    Removing stm32l0xx_hal_flash_ex.o(i.HAL_FLASHEx_OBProgram), (228 bytes).
    Removing stm32l0xx_hal_flash_ex.o(i.HAL_FLASHEx_OB_DeSelectPCROP), (40 bytes).
    Removing stm32l0xx_hal_flash_ex.o(i.HAL_FLASHEx_OB_SelectPCROP), (44 bytes).
    Removing stm32l0xx_hal_gpio.o(.rev16_text), (4 bytes).
    Removing stm32l0xx_hal_gpio.o(.revsh_text), (4 bytes).
    Removing stm32l0xx_hal_gpio.o(i.HAL_GPIO_EXTI_Callback), (2 bytes).
    Removing stm32l0xx_hal_gpio.o(i.HAL_GPIO_LockPin), (36 bytes).
    Removing stm32l0xx_hal_i2c.o(.rev16_text), (4 bytes).
    Removing stm32l0xx_hal_i2c.o(.revsh_text), (4 bytes).
    Removing stm32l0xx_hal_i2c.o(i.HAL_I2C_ER_IRQHandler), (112 bytes).
    Removing stm32l0xx_hal_i2c.o(i.HAL_I2C_EV_IRQHandler), (290 bytes).
    Removing stm32l0xx_hal_i2c.o(i.HAL_I2C_ErrorCallback), (2 bytes).
    Removing stm32l0xx_hal_i2c.o(i.HAL_I2C_GetError), (6 bytes).
    Removing stm32l0xx_hal_i2c.o(i.HAL_I2C_GetState), (6 bytes).
    Removing stm32l0xx_hal_i2c.o(i.HAL_I2C_IsDeviceReady), (284 bytes).
    Removing stm32l0xx_hal_i2c.o(i.HAL_I2C_MasterRxCpltCallback), (2 bytes).
    Removing stm32l0xx_hal_i2c.o(i.HAL_I2C_MasterTxCpltCallback), (2 bytes).
    Removing stm32l0xx_hal_i2c.o(i.HAL_I2C_Master_Receive), (240 bytes).
    Removing stm32l0xx_hal_i2c.o(i.HAL_I2C_Master_Receive_DMA), (188 bytes).
    Removing stm32l0xx_hal_i2c.o(i.HAL_I2C_Master_Receive_IT), (132 bytes).
    Removing stm32l0xx_hal_i2c.o(i.HAL_I2C_Master_Transmit), (236 bytes).
    Removing stm32l0xx_hal_i2c.o(i.HAL_I2C_Master_Transmit_DMA), (204 bytes).
    Removing stm32l0xx_hal_i2c.o(i.HAL_I2C_Master_Transmit_IT), (132 bytes).
    Removing stm32l0xx_hal_i2c.o(i.HAL_I2C_MemRxCpltCallback), (2 bytes).
    Removing stm32l0xx_hal_i2c.o(i.HAL_I2C_MemTxCpltCallback), (2 bytes).
    Removing stm32l0xx_hal_i2c.o(i.HAL_I2C_Mem_Read_DMA), (220 bytes).
    Removing stm32l0xx_hal_i2c.o(i.HAL_I2C_Mem_Read_IT), (160 bytes).
    Removing stm32l0xx_hal_i2c.o(i.HAL_I2C_Mem_Write_DMA), (220 bytes).
    Removing stm32l0xx_hal_i2c.o(i.HAL_I2C_Mem_Write_IT), (158 bytes).
    Removing stm32l0xx_hal_i2c.o(i.HAL_I2C_MspDeInit), (2 bytes).
    Removing stm32l0xx_hal_i2c.o(i.HAL_I2C_MspInit), (2 bytes).
    Removing stm32l0xx_hal_i2c.o(i.HAL_I2C_SlaveRxCpltCallback), (2 bytes).
    Removing stm32l0xx_hal_i2c.o(i.HAL_I2C_SlaveTxCpltCallback), (2 bytes).
    Removing stm32l0xx_hal_i2c.o(i.HAL_I2C_Slave_Receive), (248 bytes).
    Removing stm32l0xx_hal_i2c.o(i.HAL_I2C_Slave_Receive_DMA), (172 bytes).
    Removing stm32l0xx_hal_i2c.o(i.HAL_I2C_Slave_Receive_IT), (80 bytes).
    Removing stm32l0xx_hal_i2c.o(i.HAL_I2C_Slave_Transmit), (270 bytes).
    Removing stm32l0xx_hal_i2c.o(i.HAL_I2C_Slave_Transmit_DMA), (204 bytes).
    Removing stm32l0xx_hal_i2c.o(i.HAL_I2C_Slave_Transmit_IT), (80 bytes).
    Removing stm32l0xx_hal_i2c.o(i.I2C_DMAError), (42 bytes).
    Removing stm32l0xx_hal_i2c.o(i.I2C_DMAMasterReceiveCplt), (376 bytes).
    Removing stm32l0xx_hal_i2c.o(i.I2C_DMAMasterTransmitCplt), (360 bytes).
    Removing stm32l0xx_hal_i2c.o(i.I2C_DMAMemReceiveCplt), (376 bytes).
    Removing stm32l0xx_hal_i2c.o(i.I2C_DMAMemTransmitCplt), (360 bytes).
    Removing stm32l0xx_hal_i2c.o(i.I2C_DMASlaveReceiveCplt), (118 bytes).
    Removing stm32l0xx_hal_i2c.o(i.I2C_DMASlaveTransmitCplt), (110 bytes).
    Removing stm32l0xx_hal_i2c.o(i.I2C_MasterReceive_ISR), (260 bytes).
    Removing stm32l0xx_hal_i2c.o(i.I2C_MasterTransmit_ISR), (260 bytes).
    Removing stm32l0xx_hal_i2c.o(i.I2C_SlaveReceive_ISR), (148 bytes).
    Removing stm32l0xx_hal_i2c.o(i.I2C_SlaveTransmit_ISR), (158 bytes).
    Removing stm32l0xx_hal_i2c.o(i.I2C_WaitOnRXNEFlagUntilTimeout), (108 bytes).
    Removing stm32l0xx_hal_i2c_ex.o(.rev16_text), (4 bytes).
    Removing stm32l0xx_hal_i2c_ex.o(.revsh_text), (4 bytes).
    Removing stm32l0xx_hal_i2c_ex.o(i.HAL_I2CEx_AnalogFilter_Config), (96 bytes).
    Removing stm32l0xx_hal_i2c_ex.o(i.HAL_I2CEx_DigitalFilter_Config), (94 bytes).
    Removing stm32l0xx_hal_i2c_ex.o(i.HAL_I2CEx_DisableWakeUp), (88 bytes).
    Removing stm32l0xx_hal_i2c_ex.o(i.HAL_I2CEx_EnableWakeUp), (88 bytes).
    Removing stm32l0xx_hal_pcd.o(.rev16_text), (4 bytes).
    Removing stm32l0xx_hal_pcd.o(.revsh_text), (4 bytes).
    Removing stm32l0xx_hal_pcd.o(i.HAL_PCD_ActiveRemoteWakeup), (16 bytes).
    Removing stm32l0xx_hal_pcd.o(i.HAL_PCD_ConnectCallback), (2 bytes).
    Removing stm32l0xx_hal_pcd.o(i.HAL_PCD_DataInStageCallback), (2 bytes).
    Removing stm32l0xx_hal_pcd.o(i.HAL_PCD_DataOutStageCallback), (2 bytes).
    Removing stm32l0xx_hal_pcd.o(i.HAL_PCD_DeActiveRemoteWakeup), (16 bytes).
    Removing stm32l0xx_hal_pcd.o(i.HAL_PCD_DevConnect), (40 bytes).
    Removing stm32l0xx_hal_pcd.o(i.HAL_PCD_DevDisconnect), (38 bytes).
    Removing stm32l0xx_hal_pcd.o(i.HAL_PCD_DisconnectCallback), (2 bytes).
    Removing stm32l0xx_hal_pcd.o(i.HAL_PCD_EP_Flush), (4 bytes).
    Removing stm32l0xx_hal_pcd.o(i.HAL_PCD_EP_GetRxCount), (18 bytes).
    Removing stm32l0xx_hal_pcd.o(i.HAL_PCD_GetState), (8 bytes).
    Removing stm32l0xx_hal_pcd.o(i.HAL_PCD_ISOINIncompleteCallback), (2 bytes).
    Removing stm32l0xx_hal_pcd.o(i.HAL_PCD_ISOOUTIncompleteCallback), (2 bytes).
    Removing stm32l0xx_hal_pcd.o(i.HAL_PCD_MspDeInit), (2 bytes).
    Removing stm32l0xx_hal_pcd.o(i.HAL_PCD_MspInit), (2 bytes).
    Removing stm32l0xx_hal_pcd.o(i.HAL_PCD_ResetCallback), (2 bytes).
    Removing stm32l0xx_hal_pcd.o(i.HAL_PCD_ResumeCallback), (2 bytes).
    Removing stm32l0xx_hal_pcd.o(i.HAL_PCD_SOFCallback), (2 bytes).
    Removing stm32l0xx_hal_pcd.o(i.HAL_PCD_SetupStageCallback), (2 bytes).
    Removing stm32l0xx_hal_pcd.o(i.HAL_PCD_SuspendCallback), (2 bytes).
    Removing stm32l0xx_hal_pcd_ex.o(.rev16_text), (4 bytes).
    Removing stm32l0xx_hal_pcd_ex.o(.revsh_text), (4 bytes).
    Removing stm32l0xx_hal_pwr.o(.rev16_text), (4 bytes).
    Removing stm32l0xx_hal_pwr.o(.revsh_text), (4 bytes).
    Removing stm32l0xx_hal_pwr.o(i.HAL_PWR_DeInit), (24 bytes).
    Removing stm32l0xx_hal_pwr.o(i.HAL_PWR_DisableBkUpAccess), (16 bytes).
    Removing stm32l0xx_hal_pwr.o(i.HAL_PWR_DisablePVD), (16 bytes).
    Removing stm32l0xx_hal_pwr.o(i.HAL_PWR_DisableWakeUpPin), (16 bytes).
    Removing stm32l0xx_hal_pwr.o(i.HAL_PWR_EnableBkUpAccess), (16 bytes).
    Removing stm32l0xx_hal_pwr.o(i.HAL_PWR_EnablePVD), (16 bytes).
    Removing stm32l0xx_hal_pwr.o(i.HAL_PWR_EnableWakeUpPin), (16 bytes).
    Removing stm32l0xx_hal_pwr.o(i.HAL_PWR_EnterSTANDBYMode), (32 bytes).
    Removing stm32l0xx_hal_pwr.o(i.HAL_PWR_EnterSTOPMode), (52 bytes).
    Removing stm32l0xx_hal_pwr.o(i.HAL_PWR_PVDCallback), (2 bytes).
    Removing stm32l0xx_hal_pwr.o(i.HAL_PWR_PVDConfig), (96 bytes).
    Removing stm32l0xx_hal_pwr.o(i.HAL_PWR_PVD_IRQHandler), (28 bytes).
    Removing stm32l0xx_hal_pwr_ex.o(.rev16_text), (4 bytes).
    Removing stm32l0xx_hal_pwr_ex.o(.revsh_text), (4 bytes).
    Removing stm32l0xx_hal_pwr_ex.o(i.HAL_PWREx_DisableFastWakeUp), (16 bytes).
    Removing stm32l0xx_hal_pwr_ex.o(i.HAL_PWREx_DisableLowPowerRunMode), (24 bytes).
    Removing stm32l0xx_hal_pwr_ex.o(i.HAL_PWREx_DisableUltraLowPower), (16 bytes).
    Removing stm32l0xx_hal_pwr_ex.o(i.HAL_PWREx_EnableLowPowerRunMode), (24 bytes).
    Removing stm32l0xx_hal_rcc.o(.rev16_text), (4 bytes).
    Removing stm32l0xx_hal_rcc.o(.revsh_text), (4 bytes).
    Removing stm32l0xx_hal_rcc.o(i.HAL_RCC_CCSCallback), (2 bytes).
    Removing stm32l0xx_hal_rcc.o(i.HAL_RCC_DeInit), (44 bytes).
    Removing stm32l0xx_hal_rcc.o(i.HAL_RCC_EnableCSS), (20 bytes).
    Removing stm32l0xx_hal_rcc.o(i.HAL_RCC_GetClockConfig), (64 bytes).
    Removing stm32l0xx_hal_rcc.o(i.HAL_RCC_GetOscConfig), (192 bytes).
    Removing stm32l0xx_hal_rcc.o(i.HAL_RCC_GetPCLK1Freq), (32 bytes).
    Removing stm32l0xx_hal_rcc.o(i.HAL_RCC_GetPCLK2Freq), (32 bytes).
    Removing stm32l0xx_hal_rcc.o(i.HAL_RCC_MCOConfig), (80 bytes).
    Removing stm32l0xx_hal_rcc.o(i.HAL_RCC_NMI_IRQHandler), (24 bytes).
    Removing stm32l0xx_hal_rcc_ex.o(.rev16_text), (4 bytes).
    Removing stm32l0xx_hal_rcc_ex.o(.revsh_text), (4 bytes).
    Removing stm32l0xx_hal_rcc_ex.o(i.HAL_RCCEx_CRSGetSynchronizationInfo), (40 bytes).
    Removing stm32l0xx_hal_rcc_ex.o(i.HAL_RCCEx_CRSSoftwareSynchronizationGenerate), (16 bytes).
    Removing stm32l0xx_hal_rcc_ex.o(i.HAL_RCCEx_CRSWaitSynchronization), (136 bytes).
    Removing stm32l0xx_hal_rcc_ex.o(i.HAL_RCCEx_DisableLSECSS), (20 bytes).
    Removing stm32l0xx_hal_rcc_ex.o(i.HAL_RCCEx_EnableLSECSS), (20 bytes).
    Removing stm32l0xx_hal_rcc_ex.o(i.HAL_RCCEx_GetPeriphCLKConfig), (72 bytes).
    Removing stm32l0xx_hal_spi.o(.rev16_text), (4 bytes).
    Removing stm32l0xx_hal_spi.o(.revsh_text), (4 bytes).
    Removing stm32l0xx_hal_spi.o(i.HAL_SPI_DMAPause), (46 bytes).
    Removing stm32l0xx_hal_spi.o(i.HAL_SPI_DMAResume), (44 bytes).
    Removing stm32l0xx_hal_spi.o(i.HAL_SPI_DMAStop), (54 bytes).
    Removing stm32l0xx_hal_spi.o(i.HAL_SPI_ErrorCallback), (2 bytes).
    Removing stm32l0xx_hal_spi.o(i.HAL_SPI_GetError), (6 bytes).
    Removing stm32l0xx_hal_spi.o(i.HAL_SPI_IRQHandler), (192 bytes).
    Removing stm32l0xx_hal_spi.o(i.HAL_SPI_Receive), (462 bytes).
    Removing stm32l0xx_hal_spi.o(i.HAL_SPI_Receive_DMA), (208 bytes).
    Removing stm32l0xx_hal_spi.o(i.HAL_SPI_Receive_IT), (172 bytes).
    Removing stm32l0xx_hal_spi.o(i.HAL_SPI_RxCpltCallback), (2 bytes).
    Removing stm32l0xx_hal_spi.o(i.HAL_SPI_RxHalfCpltCallback), (2 bytes).
    Removing stm32l0xx_hal_spi.o(i.HAL_SPI_TransmitReceive), (690 bytes).
    Removing stm32l0xx_hal_spi.o(i.HAL_SPI_TransmitReceive_DMA), (252 bytes).
    Removing stm32l0xx_hal_spi.o(i.HAL_SPI_TransmitReceive_IT), (160 bytes).
    Removing stm32l0xx_hal_spi.o(i.HAL_SPI_Transmit_DMA), (188 bytes).
    Removing stm32l0xx_hal_spi.o(i.HAL_SPI_Transmit_IT), (156 bytes).
    Removing stm32l0xx_hal_spi.o(i.HAL_SPI_TxCpltCallback), (2 bytes).
    Removing stm32l0xx_hal_spi.o(i.HAL_SPI_TxHalfCpltCallback), (2 bytes).
    Removing stm32l0xx_hal_spi.o(i.HAL_SPI_TxRxCpltCallback), (2 bytes).
    Removing stm32l0xx_hal_spi.o(i.HAL_SPI_TxRxHalfCpltCallback), (2 bytes).
    Removing stm32l0xx_hal_spi.o(i.SPI_2LinesRxISR), (48 bytes).
    Removing stm32l0xx_hal_spi.o(i.SPI_DMAError), (32 bytes).
    Removing stm32l0xx_hal_spi.o(i.SPI_DMAHalfReceiveCplt), (10 bytes).
    Removing stm32l0xx_hal_spi.o(i.SPI_DMAHalfTransmitCplt), (10 bytes).
    Removing stm32l0xx_hal_spi.o(i.SPI_DMAHalfTransmitReceiveCplt), (10 bytes).
    Removing stm32l0xx_hal_spi.o(i.SPI_DMAReceiveCplt), (186 bytes).
    Removing stm32l0xx_hal_spi.o(i.SPI_DMATransmitCplt), (120 bytes).
    Removing stm32l0xx_hal_spi.o(i.SPI_DMATransmitReceiveCplt), (208 bytes).
    Removing stm32l0xx_hal_spi.o(i.SPI_RxCloseIRQHandler), (200 bytes).
    Removing stm32l0xx_hal_spi.o(i.SPI_RxISR), (78 bytes).
    Removing stm32l0xx_hal_spi.o(i.SPI_TxCloseIRQHandler), (130 bytes).
    Removing stm32l0xx_hal_spi.o(i.SPI_TxISR), (72 bytes).
    Removing stm32l0xx_hal_tsc.o(.rev16_text), (4 bytes).
    Removing stm32l0xx_hal_tsc.o(.revsh_text), (4 bytes).
    Removing stm32l0xx_hal_tsc.o(i.HAL_TSC_ConvCpltCallback), (2 bytes).
    Removing stm32l0xx_hal_tsc.o(i.HAL_TSC_ErrorCallback), (2 bytes).
    Removing stm32l0xx_hal_tsc.o(i.HAL_TSC_GetState), (40 bytes).
    Removing stm32l0xx_hal_tsc.o(i.HAL_TSC_GroupGetStatus), (22 bytes).
    Removing stm32l0xx_hal_tsc.o(i.HAL_TSC_GroupGetValue), (10 bytes).
    Removing stm32l0xx_hal_tsc.o(i.HAL_TSC_IOConfig), (80 bytes).
    Removing stm32l0xx_hal_tsc.o(i.HAL_TSC_IODischarge), (42 bytes).
    Removing stm32l0xx_hal_tsc.o(i.HAL_TSC_IRQHandler), (56 bytes).
    Removing stm32l0xx_hal_tsc.o(i.HAL_TSC_MspDeInit), (2 bytes).
    Removing stm32l0xx_hal_tsc.o(i.HAL_TSC_MspInit), (2 bytes).
    Removing stm32l0xx_hal_tsc.o(i.HAL_TSC_PollForAcquisition), (38 bytes).
    Removing stm32l0xx_hal_tsc.o(i.HAL_TSC_Start), (64 bytes).
    Removing stm32l0xx_hal_tsc.o(i.HAL_TSC_Start_IT), (80 bytes).
    Removing stm32l0xx_hal_tsc.o(i.HAL_TSC_Stop), (44 bytes).
    Removing stm32l0xx_hal_tsc.o(i.HAL_TSC_Stop_IT), (54 bytes).
    Removing tsl.o(.rev16_text), (4 bytes).
    Removing tsl.o(.revsh_text), (4 bytes).
    Removing tsl_acq.o(.rev16_text), (4 bytes).
    Removing tsl_acq.o(.revsh_text), (4 bytes).
    Removing tsl_acq.o(i.TSL_acq_BankCalibrate), (268 bytes).
    Removing tsl_acq.o(i.TSL_acq_BankClearData), (60 bytes).
    Removing tsl_acq.o(.data), (6 bytes).
    Removing tsl_acq_tsc.o(.rev16_text), (4 bytes).
    Removing tsl_acq_tsc.o(.revsh_text), (4 bytes).
    Removing tsl_dxs.o(.rev16_text), (4 bytes).
    Removing tsl_dxs.o(.revsh_text), (4 bytes).
    Removing tsl_ecs.o(.rev16_text), (4 bytes).
    Removing tsl_ecs.o(.revsh_text), (4 bytes).
    Removing tsl_filter.o(.rev16_text), (4 bytes).
    Removing tsl_filter.o(.revsh_text), (4 bytes).
    Removing tsl_filter.o(i.TSL_filt_DeltaFilter), (2 bytes).
    Removing tsl_filter.o(i.TSL_filt_MeasFilter), (32 bytes).
    Removing tsl_globals.o(.rev16_text), (4 bytes).
    Removing tsl_globals.o(.revsh_text), (4 bytes).
    Removing tsl_linrot.o(.rev16_text), (4 bytes).
    Removing tsl_linrot.o(.revsh_text), (4 bytes).
    Removing tsl_linrot.o(i.TSL_linrot_GetStateId), (16 bytes).
    Removing tsl_linrot.o(i.TSL_linrot_IsChanged), (20 bytes).
    Removing tsl_linrot.o(i.TSL_linrot_NormDelta), (32 bytes).
    Removing tsl_linrot.o(i.TSL_linrot_ProcessCh_All_AcqStatus), (48 bytes).
    Removing tsl_linrot.o(i.TSL_linrot_SetStateBurstOnly), (36 bytes).
    Removing tsl_linrot.o(i.TSL_linrot_SetStateOff), (36 bytes).
    Removing tsl_object.o(.rev16_text), (4 bytes).
    Removing tsl_object.o(.revsh_text), (4 bytes).
    Removing tsl_time.o(.rev16_text), (4 bytes).
    Removing tsl_time.o(.revsh_text), (4 bytes).
    Removing tsl_time.o(i.TSL_tim_ProcessIT), (56 bytes).
    Removing tsl_time.o(.data), (2 bytes).
    Removing tsl_touchkey.o(.rev16_text), (4 bytes).
    Removing tsl_touchkey.o(.revsh_text), (4 bytes).
    Removing usbd_hid.o(.rev16_text), (4 bytes).
    Removing usbd_hid.o(.revsh_text), (4 bytes).
    Removing usbd_hid.o(i.USBD_HID_GetPollingInterval), (4 bytes).
    Removing usbd_core.o(.rev16_text), (4 bytes).
    Removing usbd_core.o(.revsh_text), (4 bytes).
    Removing usbd_core.o(i.USBD_LL_DevConnected), (4 bytes).
    Removing usbd_core.o(i.USBD_LL_DevDisconnected), (26 bytes).
    Removing usbd_core.o(i.USBD_LL_IsoINIncomplete), (4 bytes).
    Removing usbd_core.o(i.USBD_LL_IsoOUTIncomplete), (4 bytes).
    Removing usbd_core.o(i.USBD_LL_Resume), (12 bytes).
    Removing usbd_core.o(i.USBD_LL_Suspend), (16 bytes).
    Removing usbd_core.o(i.USBD_RunTestMode), (4 bytes).
    Removing usbd_core.o(i.USBD_Stop), (30 bytes).
    Removing usbd_ctlreq.o(.rev16_text), (4 bytes).
    Removing usbd_ctlreq.o(.revsh_text), (4 bytes).
    Removing usbd_ioreq.o(.rev16_text), (4 bytes).
    Removing usbd_ioreq.o(.revsh_text), (4 bytes).
    Removing usbd_ioreq.o(i.USBD_CtlPrepareRx), (32 bytes).
    Removing usbd_ioreq.o(i.USBD_GetRxCount), (10 bytes).
    Removing dadd.o(.text), (356 bytes).
    Removing dmul.o(.text), (208 bytes).
    Removing ddiv.o(.text), (240 bytes).
    Removing dfixul.o(.text), (64 bytes).
    Removing cdrcmple.o(.text), (40 bytes).
    Removing depilogue.o(.text), (190 bytes).
    Removing depilogue.o(i.__ARM_clz), (46 bytes).

359 unused section(s) (total 29300 bytes) removed from the image.

==============================================================================

Image Symbol Table

    Local Symbols

    Symbol Name                              Value     Ov Type        Size  Object(Section)

    ../clib/../cmprslib/zerorunl2.c          0x00000000   Number         0  __dczerorl2.o ABSOLUTE
    ../clib/microlib/division.c              0x00000000   Number         0  idiv.o ABSOLUTE
    ../clib/microlib/division.c              0x00000000   Number         0  uldiv.o ABSOLUTE
    ../clib/microlib/division.c              0x00000000   Number         0  uidiv.o ABSOLUTE
    ../clib/microlib/init/entry.s            0x00000000   Number         0  entry10a.o ABSOLUTE
    ../clib/microlib/init/entry.s            0x00000000   Number         0  entry.o ABSOLUTE
    ../clib/microlib/init/entry.s            0x00000000   Number         0  entry9a.o ABSOLUTE
    ../clib/microlib/init/entry.s            0x00000000   Number         0  entry2.o ABSOLUTE
    ../clib/microlib/init/entry.s            0x00000000   Number         0  entry11a.o ABSOLUTE
    ../clib/microlib/init/entry.s            0x00000000   Number         0  entry8b.o ABSOLUTE
    ../clib/microlib/init/entry.s            0x00000000   Number         0  entry8a.o ABSOLUTE
    ../clib/microlib/init/entry.s            0x00000000   Number         0  entry9b.o ABSOLUTE
    ../clib/microlib/init/entry.s            0x00000000   Number         0  entry11b.o ABSOLUTE
    ../clib/microlib/init/entry.s            0x00000000   Number         0  entry7a.o ABSOLUTE
    ../clib/microlib/init/entry.s            0x00000000   Number         0  entry7b.o ABSOLUTE
    ../clib/microlib/init/entry.s            0x00000000   Number         0  entry5.o ABSOLUTE
    ../clib/microlib/init/entry.s            0x00000000   Number         0  entry10b.o ABSOLUTE
    ../clib/microlib/longlong.c              0x00000000   Number         0  llushr.o ABSOLUTE
    ../clib/microlib/longlong.c              0x00000000   Number         0  llsshr.o ABSOLUTE
    ../clib/microlib/longlong.c              0x00000000   Number         0  llshl.o ABSOLUTE
    ../clib/microlib/printf/printf.c         0x00000000   Number         0  printfb.o ABSOLUTE
    ../clib/microlib/printf/printf.c         0x00000000   Number         0  printf1.o ABSOLUTE
    ../clib/microlib/printf/printf.c         0x00000000   Number         0  printf2.o ABSOLUTE
    ../clib/microlib/printf/printf.c         0x00000000   Number         0  printf3.o ABSOLUTE
    ../clib/microlib/printf/printf.c         0x00000000   Number         0  printf4.o ABSOLUTE
    ../clib/microlib/printf/printf.c         0x00000000   Number         0  printf5.o ABSOLUTE
    ../clib/microlib/printf/printf.c         0x00000000   Number         0  printf7.o ABSOLUTE
    ../clib/microlib/printf/printf.c         0x00000000   Number         0  printf8.o ABSOLUTE
    ../clib/microlib/printf/printf.c         0x00000000   Number         0  printf0.o ABSOLUTE
    ../clib/microlib/printf/printf.c         0x00000000   Number         0  printfa.o ABSOLUTE
    ../clib/microlib/printf/printf.c         0x00000000   Number         0  printf6.o ABSOLUTE
    ../clib/microlib/printf/stubs.s          0x00000000   Number         0  stubs.o ABSOLUTE
    ../clib/microlib/stdio/fputc.c           0x00000000   Number         0  fputc.o ABSOLUTE
    ../clib/microlib/stdio/semi.s            0x00000000   Number         0  semi.o ABSOLUTE
    ../clib/microlib/stdio/streams.c         0x00000000   Number         0  stdout.o ABSOLUTE
    ../clib/microlib/stubs.s                 0x00000000   Number         0  iusefp.o ABSOLUTE
    ../clib/microlib/stubs.s                 0x00000000   Number         0  iusesemip.o ABSOLUTE
    ../fplib/microlib/fpadd.c                0x00000000   Number         0  dadd.o ABSOLUTE
    ../fplib/microlib/fpdiv.c                0x00000000   Number         0  ddiv.o ABSOLUTE
    ../fplib/microlib/fpepilogue.c           0x00000000   Number         0  depilogue.o ABSOLUTE
    ../fplib/microlib/fpfix.c                0x00000000   Number         0  dfixul.o ABSOLUTE
    ../fplib/microlib/fpmul.c                0x00000000   Number         0  dmul.o ABSOLUTE
    ..\..\..\..\Drivers\BSP\Components\gde021a1\gde021a1.c 0x00000000   Number         0  gde021a1.o ABSOLUTE
    ..\..\..\..\Drivers\BSP\STM32L0538-Discovery\stm32l0538_discovery.c 0x00000000   Number         0  stm32l0538_discovery.o ABSOLUTE
    ..\..\..\..\Drivers\BSP\STM32L0538-Discovery\stm32l0538_discovery_epd.c 0x00000000   Number         0  stm32l0538_discovery_epd.o ABSOLUTE
    ..\..\..\..\Drivers\STM32L0xx_HAL_Driver\Src\stm32l0xx_hal.c 0x00000000   Number         0  stm32l0xx_hal.o ABSOLUTE
    ..\..\..\..\Drivers\STM32L0xx_HAL_Driver\Src\stm32l0xx_hal_cortex.c 0x00000000   Number         0  stm32l0xx_hal_cortex.o ABSOLUTE
    ..\..\..\..\Drivers\STM32L0xx_HAL_Driver\Src\stm32l0xx_hal_dma.c 0x00000000   Number         0  stm32l0xx_hal_dma.o ABSOLUTE
    ..\..\..\..\Drivers\STM32L0xx_HAL_Driver\Src\stm32l0xx_hal_flash.c 0x00000000   Number         0  stm32l0xx_hal_flash.o ABSOLUTE
    ..\..\..\..\Drivers\STM32L0xx_HAL_Driver\Src\stm32l0xx_hal_flash_ex.c 0x00000000   Number         0  stm32l0xx_hal_flash_ex.o ABSOLUTE
    ..\..\..\..\Drivers\STM32L0xx_HAL_Driver\Src\stm32l0xx_hal_gpio.c 0x00000000   Number         0  stm32l0xx_hal_gpio.o ABSOLUTE
    ..\..\..\..\Drivers\STM32L0xx_HAL_Driver\Src\stm32l0xx_hal_i2c.c 0x00000000   Number         0  stm32l0xx_hal_i2c.o ABSOLUTE
    ..\..\..\..\Drivers\STM32L0xx_HAL_Driver\Src\stm32l0xx_hal_i2c_ex.c 0x00000000   Number         0  stm32l0xx_hal_i2c_ex.o ABSOLUTE
    ..\..\..\..\Drivers\STM32L0xx_HAL_Driver\Src\stm32l0xx_hal_pcd.c 0x00000000   Number         0  stm32l0xx_hal_pcd.o ABSOLUTE
    ..\..\..\..\Drivers\STM32L0xx_HAL_Driver\Src\stm32l0xx_hal_pcd_ex.c 0x00000000   Number         0  stm32l0xx_hal_pcd_ex.o ABSOLUTE
    ..\..\..\..\Drivers\STM32L0xx_HAL_Driver\Src\stm32l0xx_hal_pwr.c 0x00000000   Number         0  stm32l0xx_hal_pwr.o ABSOLUTE
    ..\..\..\..\Drivers\STM32L0xx_HAL_Driver\Src\stm32l0xx_hal_pwr_ex.c 0x00000000   Number         0  stm32l0xx_hal_pwr_ex.o ABSOLUTE
    ..\..\..\..\Drivers\STM32L0xx_HAL_Driver\Src\stm32l0xx_hal_rcc.c 0x00000000   Number         0  stm32l0xx_hal_rcc.o ABSOLUTE
    ..\..\..\..\Drivers\STM32L0xx_HAL_Driver\Src\stm32l0xx_hal_rcc_ex.c 0x00000000   Number         0  stm32l0xx_hal_rcc_ex.o ABSOLUTE
    ..\..\..\..\Drivers\STM32L0xx_HAL_Driver\Src\stm32l0xx_hal_spi.c 0x00000000   Number         0  stm32l0xx_hal_spi.o ABSOLUTE
    ..\..\..\..\Drivers\STM32L0xx_HAL_Driver\Src\stm32l0xx_hal_tsc.c 0x00000000   Number         0  stm32l0xx_hal_tsc.o ABSOLUTE
    ..\..\..\..\Middlewares\ST\STM32_TouchSensing_Library\src\tsl.c 0x00000000   Number         0  tsl.o ABSOLUTE
    ..\..\..\..\Middlewares\ST\STM32_TouchSensing_Library\src\tsl_acq.c 0x00000000   Number         0  tsl_acq.o ABSOLUTE
    ..\..\..\..\Middlewares\ST\STM32_TouchSensing_Library\src\tsl_acq_tsc.c 0x00000000   Number         0  tsl_acq_tsc.o ABSOLUTE
    ..\..\..\..\Middlewares\ST\STM32_TouchSensing_Library\src\tsl_dxs.c 0x00000000   Number         0  tsl_dxs.o ABSOLUTE
    ..\..\..\..\Middlewares\ST\STM32_TouchSensing_Library\src\tsl_ecs.c 0x00000000   Number         0  tsl_ecs.o ABSOLUTE
    ..\..\..\..\Middlewares\ST\STM32_TouchSensing_Library\src\tsl_filter.c 0x00000000   Number         0  tsl_filter.o ABSOLUTE
    ..\..\..\..\Middlewares\ST\STM32_TouchSensing_Library\src\tsl_globals.c 0x00000000   Number         0  tsl_globals.o ABSOLUTE
    ..\..\..\..\Middlewares\ST\STM32_TouchSensing_Library\src\tsl_linrot.c 0x00000000   Number         0  tsl_linrot.o ABSOLUTE
    ..\..\..\..\Middlewares\ST\STM32_TouchSensing_Library\src\tsl_object.c 0x00000000   Number         0  tsl_object.o ABSOLUTE
    ..\..\..\..\Middlewares\ST\STM32_TouchSensing_Library\src\tsl_time.c 0x00000000   Number         0  tsl_time.o ABSOLUTE
    ..\..\..\..\Middlewares\ST\STM32_TouchSensing_Library\src\tsl_touchkey.c 0x00000000   Number         0  tsl_touchkey.o ABSOLUTE
    ..\..\..\..\Middlewares\ST\STM32_USB_Device_Library\Class\HID\Src\usbd_hid.c 0x00000000   Number         0  usbd_hid.o ABSOLUTE
    ..\..\..\..\Middlewares\ST\STM32_USB_Device_Library\Core\Src\usbd_core.c 0x00000000   Number         0  usbd_core.o ABSOLUTE
    ..\..\..\..\Middlewares\ST\STM32_USB_Device_Library\Core\Src\usbd_ctlreq.c 0x00000000   Number         0  usbd_ctlreq.o ABSOLUTE
    ..\..\..\..\Middlewares\ST\STM32_USB_Device_Library\Core\Src\usbd_ioreq.c 0x00000000   Number         0  usbd_ioreq.o ABSOLUTE
    ..\Core\Src\bsp.c                        0x00000000   Number         0  bsp.o ABSOLUTE
    ..\Core\Src\main.c                       0x00000000   Number         0  main.o ABSOLUTE
    ..\Core\Src\menu.c                       0x00000000   Number         0  menu.o ABSOLUTE
    ..\Core\Src\stm32l0xx_hal_msp.c          0x00000000   Number         0  stm32l0xx_hal_msp.o ABSOLUTE
    ..\Core\Src\stm32l0xx_it.c               0x00000000   Number         0  stm32l0xx_it.o ABSOLUTE
    ..\Core\Src\system_stm32l0xx.c           0x00000000   Number         0  system_stm32l0xx.o ABSOLUTE
    ..\Core\Src\tsl_user.c                   0x00000000   Number         0  tsl_user.o ABSOLUTE
    ..\Modules\iddmeasurement\power.c        0x00000000   Number         0  power.o ABSOLUTE
    ..\Modules\usbHID\usbd_conf.c            0x00000000   Number         0  usbd_conf.o ABSOLUTE
    ..\Modules\usbHID\usbd_desc.c            0x00000000   Number         0  usbd_desc.o ABSOLUTE
    ..\Modules\usbHID\usbdapp.c              0x00000000   Number         0  usbdapp.o ABSOLUTE
    ..\\..\\..\\..\\Drivers\\BSP\\STM32L0538-Discovery\\stm32l0538_discovery.c 0x00000000   Number         0  stm32l0538_discovery.o ABSOLUTE
    ..\\..\\..\\..\\Drivers\\BSP\\STM32L0538-Discovery\\stm32l0538_discovery_epd.c 0x00000000   Number         0  stm32l0538_discovery_epd.o ABSOLUTE
    ..\\..\\..\\..\\Drivers\\STM32L0xx_HAL_Driver\\Src\\stm32l0xx_hal.c 0x00000000   Number         0  stm32l0xx_hal.o ABSOLUTE
    ..\\..\\..\\..\\Drivers\\STM32L0xx_HAL_Driver\\Src\\stm32l0xx_hal_cortex.c 0x00000000   Number         0  stm32l0xx_hal_cortex.o ABSOLUTE
    ..\\..\\..\\..\\Drivers\\STM32L0xx_HAL_Driver\\Src\\stm32l0xx_hal_dma.c 0x00000000   Number         0  stm32l0xx_hal_dma.o ABSOLUTE
    ..\\..\\..\\..\\Drivers\\STM32L0xx_HAL_Driver\\Src\\stm32l0xx_hal_flash.c 0x00000000   Number         0  stm32l0xx_hal_flash.o ABSOLUTE
    ..\\..\\..\\..\\Drivers\\STM32L0xx_HAL_Driver\\Src\\stm32l0xx_hal_flash_ex.c 0x00000000   Number         0  stm32l0xx_hal_flash_ex.o ABSOLUTE
    ..\\..\\..\\..\\Drivers\\STM32L0xx_HAL_Driver\\Src\\stm32l0xx_hal_gpio.c 0x00000000   Number         0  stm32l0xx_hal_gpio.o ABSOLUTE
    ..\\..\\..\\..\\Drivers\\STM32L0xx_HAL_Driver\\Src\\stm32l0xx_hal_i2c.c 0x00000000   Number         0  stm32l0xx_hal_i2c.o ABSOLUTE
    ..\\..\\..\\..\\Drivers\\STM32L0xx_HAL_Driver\\Src\\stm32l0xx_hal_i2c_ex.c 0x00000000   Number         0  stm32l0xx_hal_i2c_ex.o ABSOLUTE
    ..\\..\\..\\..\\Drivers\\STM32L0xx_HAL_Driver\\Src\\stm32l0xx_hal_pcd.c 0x00000000   Number         0  stm32l0xx_hal_pcd.o ABSOLUTE
    ..\\..\\..\\..\\Drivers\\STM32L0xx_HAL_Driver\\Src\\stm32l0xx_hal_pcd_ex.c 0x00000000   Number         0  stm32l0xx_hal_pcd_ex.o ABSOLUTE
    ..\\..\\..\\..\\Drivers\\STM32L0xx_HAL_Driver\\Src\\stm32l0xx_hal_pwr.c 0x00000000   Number         0  stm32l0xx_hal_pwr.o ABSOLUTE
    ..\\..\\..\\..\\Drivers\\STM32L0xx_HAL_Driver\\Src\\stm32l0xx_hal_pwr_ex.c 0x00000000   Number         0  stm32l0xx_hal_pwr_ex.o ABSOLUTE
    ..\\..\\..\\..\\Drivers\\STM32L0xx_HAL_Driver\\Src\\stm32l0xx_hal_rcc.c 0x00000000   Number         0  stm32l0xx_hal_rcc.o ABSOLUTE
    ..\\..\\..\\..\\Drivers\\STM32L0xx_HAL_Driver\\Src\\stm32l0xx_hal_rcc_ex.c 0x00000000   Number         0  stm32l0xx_hal_rcc_ex.o ABSOLUTE
    ..\\..\\..\\..\\Drivers\\STM32L0xx_HAL_Driver\\Src\\stm32l0xx_hal_spi.c 0x00000000   Number         0  stm32l0xx_hal_spi.o ABSOLUTE
    ..\\..\\..\\..\\Drivers\\STM32L0xx_HAL_Driver\\Src\\stm32l0xx_hal_tsc.c 0x00000000   Number         0  stm32l0xx_hal_tsc.o ABSOLUTE
    ..\\..\\..\\..\\Middlewares\\ST\\STM32_TouchSensing_Library\\src\\tsl.c 0x00000000   Number         0  tsl.o ABSOLUTE
    ..\\..\\..\\..\\Middlewares\\ST\\STM32_TouchSensing_Library\\src\\tsl_acq.c 0x00000000   Number         0  tsl_acq.o ABSOLUTE
    ..\\..\\..\\..\\Middlewares\\ST\\STM32_TouchSensing_Library\\src\\tsl_acq_tsc.c 0x00000000   Number         0  tsl_acq_tsc.o ABSOLUTE
    ..\\..\\..\\..\\Middlewares\\ST\\STM32_TouchSensing_Library\\src\\tsl_dxs.c 0x00000000   Number         0  tsl_dxs.o ABSOLUTE
    ..\\..\\..\\..\\Middlewares\\ST\\STM32_TouchSensing_Library\\src\\tsl_ecs.c 0x00000000   Number         0  tsl_ecs.o ABSOLUTE
    ..\\..\\..\\..\\Middlewares\\ST\\STM32_TouchSensing_Library\\src\\tsl_filter.c 0x00000000   Number         0  tsl_filter.o ABSOLUTE
    ..\\..\\..\\..\\Middlewares\\ST\\STM32_TouchSensing_Library\\src\\tsl_globals.c 0x00000000   Number         0  tsl_globals.o ABSOLUTE
    ..\\..\\..\\..\\Middlewares\\ST\\STM32_TouchSensing_Library\\src\\tsl_linrot.c 0x00000000   Number         0  tsl_linrot.o ABSOLUTE
    ..\\..\\..\\..\\Middlewares\\ST\\STM32_TouchSensing_Library\\src\\tsl_object.c 0x00000000   Number         0  tsl_object.o ABSOLUTE
    ..\\..\\..\\..\\Middlewares\\ST\\STM32_TouchSensing_Library\\src\\tsl_time.c 0x00000000   Number         0  tsl_time.o ABSOLUTE
    ..\\..\\..\\..\\Middlewares\\ST\\STM32_TouchSensing_Library\\src\\tsl_touchkey.c 0x00000000   Number         0  tsl_touchkey.o ABSOLUTE
    ..\\..\\..\\..\\Middlewares\\ST\\STM32_USB_Device_Library\\Class\\HID\\Src\\usbd_hid.c 0x00000000   Number         0  usbd_hid.o ABSOLUTE
    ..\\..\\..\\..\\Middlewares\\ST\\STM32_USB_Device_Library\\Core\\Src\\usbd_core.c 0x00000000   Number         0  usbd_core.o ABSOLUTE
    ..\\..\\..\\..\\Middlewares\\ST\\STM32_USB_Device_Library\\Core\\Src\\usbd_ctlreq.c 0x00000000   Number         0  usbd_ctlreq.o ABSOLUTE
    ..\\..\\..\\..\\Middlewares\\ST\\STM32_USB_Device_Library\\Core\\Src\\usbd_ioreq.c 0x00000000   Number         0  usbd_ioreq.o ABSOLUTE
    ..\\Core\\Src\\bsp.c                     0x00000000   Number         0  bsp.o ABSOLUTE
    ..\\Core\\Src\\main.c                    0x00000000   Number         0  main.o ABSOLUTE
    ..\\Core\\Src\\menu.c                    0x00000000   Number         0  menu.o ABSOLUTE
    ..\\Core\\Src\\stm32l0xx_hal_msp.c       0x00000000   Number         0  stm32l0xx_hal_msp.o ABSOLUTE
    ..\\Core\\Src\\stm32l0xx_it.c            0x00000000   Number         0  stm32l0xx_it.o ABSOLUTE
    ..\\Core\\Src\\system_stm32l0xx.c        0x00000000   Number         0  system_stm32l0xx.o ABSOLUTE
    ..\\Core\\Src\\tsl_user.c                0x00000000   Number         0  tsl_user.o ABSOLUTE
    ..\\Modules\\iddmeasurement\\power.c     0x00000000   Number         0  power.o ABSOLUTE
    ..\\Modules\\usbHID\\usbd_conf.c         0x00000000   Number         0  usbd_conf.o ABSOLUTE
    ..\\Modules\\usbHID\\usbd_desc.c         0x00000000   Number         0  usbd_desc.o ABSOLUTE
    ..\\Modules\\usbHID\\usbdapp.c           0x00000000   Number         0  usbdapp.o ABSOLUTE
    cdrcmple.s                               0x00000000   Number         0  cdrcmple.o ABSOLUTE
    dc.s                                     0x00000000   Number         0  dc.o ABSOLUTE
    handlers.s                               0x00000000   Number         0  handlers.o ABSOLUTE
    init.s                                   0x00000000   Number         0  init.o ABSOLUTE
    startup_stm32l053xx.s                    0x00000000   Number         0  startup_stm32l053xx.o ABSOLUTE
    RESET                                    0x08000000   Section      192  startup_stm32l053xx.o(RESET)
    .ARM.Collect$$$$00000000                 0x080000c0   Section        0  entry.o(.ARM.Collect$$$$00000000)
    .ARM.Collect$$$$00000001                 0x080000c0   Section        4  entry2.o(.ARM.Collect$$$$00000001)
    .ARM.Collect$$$$00000004                 0x080000c4   Section        4  entry5.o(.ARM.Collect$$$$00000004)
    .ARM.Collect$$$$00000008                 0x080000c8   Section        0  entry7b.o(.ARM.Collect$$$$00000008)
    .ARM.Collect$$$$0000000A                 0x080000c8   Section        0  entry8b.o(.ARM.Collect$$$$0000000A)
    .ARM.Collect$$$$0000000B                 0x080000c8   Section        8  entry9a.o(.ARM.Collect$$$$0000000B)
    .ARM.Collect$$$$0000000D                 0x080000d0   Section        0  entry10a.o(.ARM.Collect$$$$0000000D)
    .ARM.Collect$$$$0000000F                 0x080000d0   Section        0  entry11a.o(.ARM.Collect$$$$0000000F)
    .ARM.Collect$$$$00002712                 0x080000d0   Section        4  entry2.o(.ARM.Collect$$$$00002712)
    __lit__00000000                          0x080000d0   Data           4  entry2.o(.ARM.Collect$$$$00002712)
    .text                                    0x080000d4   Section       32  startup_stm32l053xx.o(.text)
    .text                                    0x080000f4   Section        0  uidiv.o(.text)
    .text                                    0x08000120   Section        0  idiv.o(.text)
    .text                                    0x08000148   Section       36  init.o(.text)
    .text                                    0x0800016c   Section        0  __dczerorl2.o(.text)
    i.BSP_EPD_Clear                          0x080001c4   Section        0  stm32l0538_discovery_epd.o(i.BSP_EPD_Clear)
    i.BSP_EPD_DisplayChar                    0x080001f4   Section        0  stm32l0538_discovery_epd.o(i.BSP_EPD_DisplayChar)
    i.BSP_EPD_DisplayStringAt                0x08000240   Section        0  stm32l0538_discovery_epd.o(i.BSP_EPD_DisplayStringAt)
    i.BSP_EPD_DrawHLine                      0x080002dc   Section        0  stm32l0538_discovery_epd.o(i.BSP_EPD_DrawHLine)
    i.BSP_EPD_DrawImage                      0x08000308   Section        0  stm32l0538_discovery_epd.o(i.BSP_EPD_DrawImage)
    i.BSP_EPD_DrawRect                       0x08000364   Section        0  stm32l0538_discovery_epd.o(i.BSP_EPD_DrawRect)
    i.BSP_EPD_DrawVLine                      0x08000398   Section        0  stm32l0538_discovery_epd.o(i.BSP_EPD_DrawVLine)
    i.BSP_EPD_GetXSize                       0x080003c4   Section        0  stm32l0538_discovery_epd.o(i.BSP_EPD_GetXSize)
    i.BSP_EPD_GetYSize                       0x080003d0   Section        0  stm32l0538_discovery_epd.o(i.BSP_EPD_GetYSize)
    i.BSP_EPD_Init                           0x080003dc   Section        0  stm32l0538_discovery_epd.o(i.BSP_EPD_Init)
    i.BSP_EPD_RefreshDisplay                 0x08000408   Section        0  stm32l0538_discovery_epd.o(i.BSP_EPD_RefreshDisplay)
    i.BSP_EPD_SetFont                        0x08000440   Section        0  stm32l0538_discovery_epd.o(i.BSP_EPD_SetFont)
    i.BSP_LED_Init                           0x0800044c   Section        0  stm32l0538_discovery.o(i.BSP_LED_Init)
    i.BSP_LED_Off                            0x08000498   Section        0  stm32l0538_discovery.o(i.BSP_LED_Off)
    i.BSP_LED_Toggle                         0x080004b8   Section        0  stm32l0538_discovery.o(i.BSP_LED_Toggle)
    i.BSP_PB_Init                            0x080004d4   Section        0  stm32l0538_discovery.o(i.BSP_PB_Init)
    i.BSP_TSL_Init                           0x08000544   Section        0  bsp.o(i.BSP_TSL_Init)
    i.BSP_USB_Init                           0x08000590   Section        0  bsp.o(i.BSP_USB_Init)
    i.Bsp_Init                               0x080005b8   Section        0  bsp.o(i.Bsp_Init)
    i.DebugMon_Handler                       0x080005d8   Section        0  stm32l0xx_it.o(i.DebugMon_Handler)
    i.EPD_Delay                              0x080005da   Section        0  stm32l0538_discovery.o(i.EPD_Delay)
    i.EPD_IO_Init                            0x080005e4   Section        0  stm32l0538_discovery.o(i.EPD_IO_Init)
    i.EPD_IO_WriteData                       0x0800069c   Section        0  stm32l0538_discovery.o(i.EPD_IO_WriteData)
    i.EPD_IO_WriteReg                        0x080006d4   Section        0  stm32l0538_discovery.o(i.EPD_IO_WriteReg)
    i.EXTI0_1_IRQHandler                     0x0800070c   Section        0  stm32l0xx_it.o(i.EXTI0_1_IRQHandler)
    i.EXTI4_15_IRQHandler                    0x08000716   Section        0  stm32l0xx_it.o(i.EXTI4_15_IRQHandler)
    i.GetPointerData                         0x08000724   Section        0  usbdapp.o(i.GetPointerData)
    i.HAL_Delay                              0x0800075c   Section        0  stm32l0xx_hal.o(i.HAL_Delay)
    i.HAL_GPIO_DeInit                        0x08000774   Section        0  stm32l0xx_hal_gpio.o(i.HAL_GPIO_DeInit)
    i.HAL_GPIO_EXTI_Callback                 0x080007fc   Section        0  menu.o(i.HAL_GPIO_EXTI_Callback)
    i.HAL_GPIO_EXTI_IRQHandler               0x0800080c   Section        0  stm32l0xx_hal_gpio.o(i.HAL_GPIO_EXTI_IRQHandler)
    i.HAL_GPIO_Init                          0x08000824   Section        0  stm32l0xx_hal_gpio.o(i.HAL_GPIO_Init)
    i.HAL_GPIO_ReadPin                       0x08000998   Section        0  stm32l0xx_hal_gpio.o(i.HAL_GPIO_ReadPin)
    i.HAL_GPIO_TogglePin                     0x080009a2   Section        0  stm32l0xx_hal_gpio.o(i.HAL_GPIO_TogglePin)
    i.HAL_GPIO_WritePin                      0x080009aa   Section        0  stm32l0xx_hal_gpio.o(i.HAL_GPIO_WritePin)
    i.HAL_GetTick                            0x080009b8   Section        0  stm32l0xx_hal.o(i.HAL_GetTick)
    i.HAL_I2C_DeInit                         0x080009c4   Section        0  stm32l0xx_hal_i2c.o(i.HAL_I2C_DeInit)
    i.HAL_I2C_Init                           0x080009f0   Section        0  stm32l0xx_hal_i2c.o(i.HAL_I2C_Init)
    i.HAL_I2C_Mem_Read                       0x08000a90   Section        0  stm32l0xx_hal_i2c.o(i.HAL_I2C_Mem_Read)
    i.HAL_I2C_Mem_Write                      0x08000ba4   Section        0  stm32l0xx_hal_i2c.o(i.HAL_I2C_Mem_Write)
    i.HAL_I2C_MspDeInit                      0x08000cac   Section        0  stm32l0xx_hal_msp.o(i.HAL_I2C_MspDeInit)
    i.HAL_I2C_MspInit                        0x08000ce4   Section        0  stm32l0xx_hal_msp.o(i.HAL_I2C_MspInit)
    i.HAL_IncTick                            0x08000d44   Section        0  stm32l0xx_hal.o(i.HAL_IncTick)
    i.HAL_Init                               0x08000d54   Section        0  stm32l0xx_hal.o(i.HAL_Init)
    i.HAL_InitTick                           0x08000d7c   Section        0  stm32l0xx_hal.o(i.HAL_InitTick)
    i.HAL_MspInit                            0x08000d9e   Section        0  stm32l0xx_hal_msp.o(i.HAL_MspInit)
    i.HAL_NVIC_DisableIRQ                    0x08000da0   Section        0  stm32l0xx_hal_cortex.o(i.HAL_NVIC_DisableIRQ)
    i.HAL_NVIC_EnableIRQ                     0x08000db4   Section        0  stm32l0xx_hal_cortex.o(i.HAL_NVIC_EnableIRQ)
    i.HAL_NVIC_SetPriority                   0x08000dc8   Section        0  stm32l0xx_hal_cortex.o(i.HAL_NVIC_SetPriority)
    i.HAL_PCDEx_PMAConfig                    0x08000dd0   Section        0  stm32l0xx_hal_pcd_ex.o(i.HAL_PCDEx_PMAConfig)
    i.HAL_PCD_DataInStageCallback            0x08000e08   Section        0  usbd_conf.o(i.HAL_PCD_DataInStageCallback)
    i.HAL_PCD_DataOutStageCallback           0x08000e1e   Section        0  usbd_conf.o(i.HAL_PCD_DataOutStageCallback)
    i.HAL_PCD_DeInit                         0x08000e36   Section        0  stm32l0xx_hal_pcd.o(i.HAL_PCD_DeInit)
    i.HAL_PCD_EP_Close                       0x08000e60   Section        0  stm32l0xx_hal_pcd.o(i.HAL_PCD_EP_Close)
    i.HAL_PCD_EP_ClrStall                    0x08000fd0   Section        0  stm32l0xx_hal_pcd.o(i.HAL_PCD_EP_ClrStall)
    i.HAL_PCD_EP_Open                        0x08001084   Section        0  stm32l0xx_hal_pcd.o(i.HAL_PCD_EP_Open)
    i.HAL_PCD_EP_Receive                     0x08001344   Section        0  stm32l0xx_hal_pcd.o(i.HAL_PCD_EP_Receive)
    i.HAL_PCD_EP_SetStall                    0x08001418   Section        0  stm32l0xx_hal_pcd.o(i.HAL_PCD_EP_SetStall)
    i.HAL_PCD_EP_Transmit                    0x080014ac   Section        0  stm32l0xx_hal_pcd.o(i.HAL_PCD_EP_Transmit)
    i.HAL_PCD_IRQHandler                     0x080015f0   Section        0  stm32l0xx_hal_pcd.o(i.HAL_PCD_IRQHandler)
    i.HAL_PCD_Init                           0x080016e0   Section        0  stm32l0xx_hal_pcd.o(i.HAL_PCD_Init)
    i.HAL_PCD_MspDeInit                      0x08001774   Section        0  usbd_conf.o(i.HAL_PCD_MspDeInit)
    i.HAL_PCD_MspInit                        0x080017b0   Section        0  usbd_conf.o(i.HAL_PCD_MspInit)
    i.HAL_PCD_ResetCallback                  0x08001800   Section        0  usbd_conf.o(i.HAL_PCD_ResetCallback)
    i.HAL_PCD_ResumeCallback                 0x08001816   Section        0  usbd_conf.o(i.HAL_PCD_ResumeCallback)
    i.HAL_PCD_SOFCallback                    0x08001818   Section        0  usbd_conf.o(i.HAL_PCD_SOFCallback)
    i.HAL_PCD_SetAddress                     0x08001826   Section        0  stm32l0xx_hal_pcd.o(i.HAL_PCD_SetAddress)
    i.HAL_PCD_SetupStageCallback             0x08001852   Section        0  usbd_conf.o(i.HAL_PCD_SetupStageCallback)
    i.HAL_PCD_Start                          0x08001868   Section        0  stm32l0xx_hal_pcd.o(i.HAL_PCD_Start)
    i.HAL_PCD_Stop                           0x0800187a   Section        0  stm32l0xx_hal_pcd.o(i.HAL_PCD_Stop)
    i.HAL_PCD_SuspendCallback                0x080018aa   Section        0  usbd_conf.o(i.HAL_PCD_SuspendCallback)
    i.HAL_PWREx_EnableFastWakeUp             0x080018ac   Section        0  stm32l0xx_hal_pwr_ex.o(i.HAL_PWREx_EnableFastWakeUp)
    i.HAL_PWREx_EnableUltraLowPower          0x080018bc   Section        0  stm32l0xx_hal_pwr_ex.o(i.HAL_PWREx_EnableUltraLowPower)
    i.HAL_PWR_EnterSLEEPMode                 0x080018cc   Section        0  stm32l0xx_hal_pwr.o(i.HAL_PWR_EnterSLEEPMode)
    i.HAL_RCCEx_CRSConfig                    0x080018fc   Section        0  stm32l0xx_hal_rcc_ex.o(i.HAL_RCCEx_CRSConfig)
    i.HAL_RCCEx_PeriphCLKConfig              0x08001978   Section        0  stm32l0xx_hal_rcc_ex.o(i.HAL_RCCEx_PeriphCLKConfig)
    i.HAL_RCC_ClockConfig                    0x08001ab4   Section        0  stm32l0xx_hal_rcc.o(i.HAL_RCC_ClockConfig)
    i.HAL_RCC_GetHCLKFreq                    0x08001cb8   Section        0  stm32l0xx_hal_rcc.o(i.HAL_RCC_GetHCLKFreq)
    i.HAL_RCC_GetSysClockFreq                0x08001ce0   Section        0  stm32l0xx_hal_rcc.o(i.HAL_RCC_GetSysClockFreq)
    i.HAL_RCC_OscConfig                      0x08001d58   Section        0  stm32l0xx_hal_rcc.o(i.HAL_RCC_OscConfig)
    i.HAL_ResumeTick                         0x0800211c   Section        0  stm32l0xx_hal.o(i.HAL_ResumeTick)
    i.HAL_SPI_DeInit                         0x0800212c   Section        0  stm32l0xx_hal_spi.o(i.HAL_SPI_DeInit)
    i.HAL_SPI_GetState                       0x08002158   Section        0  stm32l0xx_hal_spi.o(i.HAL_SPI_GetState)
    i.HAL_SPI_Init                           0x0800215e   Section        0  stm32l0xx_hal_spi.o(i.HAL_SPI_Init)
    i.HAL_SPI_MspDeInit                      0x080021e0   Section        0  stm32l0xx_hal_spi.o(i.HAL_SPI_MspDeInit)
    i.HAL_SPI_MspInit                        0x080021e2   Section        0  stm32l0xx_hal_spi.o(i.HAL_SPI_MspInit)
    i.HAL_SPI_Transmit                       0x080021e4   Section        0  stm32l0xx_hal_spi.o(i.HAL_SPI_Transmit)
    i.HAL_SYSTICK_Config                     0x08002330   Section        0  stm32l0xx_hal_cortex.o(i.HAL_SYSTICK_Config)
    i.HAL_SuspendTick                        0x08002360   Section        0  stm32l0xx_hal.o(i.HAL_SuspendTick)
    i.HAL_TSC_DeInit                         0x08002370   Section        0  stm32l0xx_hal_tsc.o(i.HAL_TSC_DeInit)
    i.HAL_TSC_Init                           0x08002390   Section        0  stm32l0xx_hal_tsc.o(i.HAL_TSC_Init)
    i.HAL_TSC_MspDeInit                      0x08002434   Section        0  stm32l0xx_hal_msp.o(i.HAL_TSC_MspDeInit)
    i.HAL_TSC_MspInit                        0x08002498   Section        0  stm32l0xx_hal_msp.o(i.HAL_TSC_MspInit)
    i.HardFault_Handler                      0x0800250c   Section        0  stm32l0xx_it.o(i.HardFault_Handler)
    i.I2C_Config                             0x08002510   Section        0  power.o(i.I2C_Config)
    I2C_Config                               0x08002511   Thumb Code    48  power.o(i.I2C_Config)
    i.I2C_IsAcknowledgeFailed                0x0800254c   Section        0  stm32l0xx_hal_i2c.o(i.I2C_IsAcknowledgeFailed)
    I2C_IsAcknowledgeFailed                  0x0800254d   Thumb Code   142  stm32l0xx_hal_i2c.o(i.I2C_IsAcknowledgeFailed)
    i.I2C_RequestMemoryRead                  0x080025e0   Section        0  stm32l0xx_hal_i2c.o(i.I2C_RequestMemoryRead)
    I2C_RequestMemoryRead                    0x080025e1   Thumb Code   102  stm32l0xx_hal_i2c.o(i.I2C_RequestMemoryRead)
    i.I2C_RequestMemoryWrite                 0x08002646   Section        0  stm32l0xx_hal_i2c.o(i.I2C_RequestMemoryWrite)
    I2C_RequestMemoryWrite                   0x08002647   Thumb Code   102  stm32l0xx_hal_i2c.o(i.I2C_RequestMemoryWrite)
    i.I2C_TransferConfig                     0x080026ac   Section        0  stm32l0xx_hal_i2c.o(i.I2C_TransferConfig)
    I2C_TransferConfig                       0x080026ad   Thumb Code    30  stm32l0xx_hal_i2c.o(i.I2C_TransferConfig)
    i.I2C_WaitOnFlagUntilTimeout             0x080026d0   Section        0  stm32l0xx_hal_i2c.o(i.I2C_WaitOnFlagUntilTimeout)
    I2C_WaitOnFlagUntilTimeout               0x080026d1   Thumb Code   112  stm32l0xx_hal_i2c.o(i.I2C_WaitOnFlagUntilTimeout)
    i.I2C_WaitOnSTOPFlagUntilTimeout         0x08002740   Section        0  stm32l0xx_hal_i2c.o(i.I2C_WaitOnSTOPFlagUntilTimeout)
    I2C_WaitOnSTOPFlagUntilTimeout           0x08002741   Thumb Code    80  stm32l0xx_hal_i2c.o(i.I2C_WaitOnSTOPFlagUntilTimeout)
    i.I2C_WaitOnTXISFlagUntilTimeout         0x08002790   Section        0  stm32l0xx_hal_i2c.o(i.I2C_WaitOnTXISFlagUntilTimeout)
    I2C_WaitOnTXISFlagUntilTimeout           0x08002791   Thumb Code    84  stm32l0xx_hal_i2c.o(i.I2C_WaitOnTXISFlagUntilTimeout)
    i.IDD_RestoreContext                     0x080027e4   Section        0  menu.o(i.IDD_RestoreContext)
    i.IDD_SaveContext                        0x080028c0   Section        0  menu.o(i.IDD_SaveContext)
    i.Idd_LPSleep_process                    0x08002a0c   Section        0  power.o(i.Idd_LPSleep_process)
    i.Idd_Run_process                        0x08002cb8   Section        0  power.o(i.Idd_Run_process)
    i.Idd_Sleep_process                      0x08002e74   Section        0  power.o(i.Idd_Sleep_process)
    i.IntToUnicode                           0x08003094   Section        0  usbd_desc.o(i.IntToUnicode)
    IntToUnicode                             0x08003095   Thumb Code    44  usbd_desc.o(i.IntToUnicode)
    i.Menu_Process                           0x080030c0   Section        0  menu.o(i.Menu_Process)
    i.MyLinRots_ErrorStateProcess            0x0800359c   Section        0  tsl_user.o(i.MyLinRots_ErrorStateProcess)
    i.MyLinRots_OffStateProcess              0x0800359e   Section        0  tsl_user.o(i.MyLinRots_OffStateProcess)
    i.NMI_Handler                            0x080035a0   Section        0  stm32l0xx_it.o(i.NMI_Handler)
    i.NVIC_SetPriority                       0x080035a4   Section        0  stm32l0xx_hal_cortex.o(i.NVIC_SetPriority)
    NVIC_SetPriority                         0x080035a5   Thumb Code    60  stm32l0xx_hal_cortex.o(i.NVIC_SetPriority)
    i.PCD_EP_ISR_Handler                     0x080035e8   Section        0  stm32l0xx_hal_pcd.o(i.PCD_EP_ISR_Handler)
    PCD_EP_ISR_Handler                       0x080035e9   Thumb Code   804  stm32l0xx_hal_pcd.o(i.PCD_EP_ISR_Handler)
    i.PCD_ReadPMA                            0x08003920   Section        0  stm32l0xx_hal_pcd.o(i.PCD_ReadPMA)
    i.PCD_WritePMA                           0x0800393e   Section        0  stm32l0xx_hal_pcd.o(i.PCD_WritePMA)
    i.PendSV_Handler                         0x08003964   Section        0  stm32l0xx_it.o(i.PendSV_Handler)
    i.SPI_WaitOnFlagUntilTimeout             0x08003966   Section        0  stm32l0xx_hal_spi.o(i.SPI_WaitOnFlagUntilTimeout)
    SPI_WaitOnFlagUntilTimeout               0x08003967   Thumb Code   178  stm32l0xx_hal_spi.o(i.SPI_WaitOnFlagUntilTimeout)
    i.SPIx_Error                             0x08003a18   Section        0  stm32l0538_discovery.o(i.SPIx_Error)
    SPIx_Error                               0x08003a19   Thumb Code    14  stm32l0538_discovery.o(i.SPIx_Error)
    i.SPIx_Init                              0x08003a2c   Section        0  stm32l0538_discovery.o(i.SPIx_Init)
    SPIx_Init                                0x08003a2d   Thumb Code   124  stm32l0538_discovery.o(i.SPIx_Init)
    i.SPIx_Write                             0x08003ab8   Section        0  stm32l0538_discovery.o(i.SPIx_Write)
    SPIx_Write                               0x08003ab9   Thumb Code    26  stm32l0538_discovery.o(i.SPIx_Write)
    i.SVC_Handler                            0x08003ad8   Section        0  stm32l0xx_it.o(i.SVC_Handler)
    i.SoftDelay                              0x08003ada   Section        0  tsl_acq_tsc.o(i.SoftDelay)
    SoftDelay                                0x08003adb   Thumb Code    10  tsl_acq_tsc.o(i.SoftDelay)
    i.SysTick_Handler                        0x08003ae4   Section        0  stm32l0xx_it.o(i.SysTick_Handler)
    i.SystemClock_Config                     0x08003b18   Section        0  menu.o(i.SystemClock_Config)
    i.SystemInit                             0x08003b70   Section        0  system_stm32l0xx.o(i.SystemInit)
    i.TSC_extract_groups                     0x08003bc4   Section        0  stm32l0xx_hal_tsc.o(i.TSC_extract_groups)
    TSC_extract_groups                       0x08003bc5   Thumb Code    36  stm32l0xx_hal_tsc.o(i.TSC_extract_groups)
    i.TSL_Init                               0x08003be8   Section        0  tsl.o(i.TSL_Init)
    i.TSL_acq_BankConfig                     0x08003c18   Section        0  tsl_acq_tsc.o(i.TSL_acq_BankConfig)
    i.TSL_acq_BankGetResult                  0x08003c7c   Section        0  tsl_acq.o(i.TSL_acq_BankGetResult)
    i.TSL_acq_BankStartAcq                   0x08003da8   Section        0  tsl_acq_tsc.o(i.TSL_acq_BankStartAcq)
    i.TSL_acq_BankWaitEOC                    0x08003dd8   Section        0  tsl_acq_tsc.o(i.TSL_acq_BankWaitEOC)
    i.TSL_acq_CheckNoise                     0x08003dfc   Section        0  tsl_acq_tsc.o(i.TSL_acq_CheckNoise)
    i.TSL_acq_ComputeDelta                   0x08003e00   Section        0  tsl_acq_tsc.o(i.TSL_acq_ComputeDelta)
    i.TSL_acq_ComputeMeas                    0x08003e06   Section        0  tsl_acq_tsc.o(i.TSL_acq_ComputeMeas)
    i.TSL_acq_GetMeas                        0x08003e0c   Section        0  tsl_acq_tsc.o(i.TSL_acq_GetMeas)
    i.TSL_acq_TestFirstReferenceIsValid      0x08003e24   Section        0  tsl_acq_tsc.o(i.TSL_acq_TestFirstReferenceIsValid)
    i.TSL_acq_TestReferenceOutOfRange        0x08003e28   Section        0  tsl_acq_tsc.o(i.TSL_acq_TestReferenceOutOfRange)
    i.TSL_acq_UseFilter                      0x08003e2c   Section        0  tsl_acq_tsc.o(i.TSL_acq_UseFilter)
    i.TSL_dxs_FirstObj                       0x08003e30   Section        0  tsl_dxs.o(i.TSL_dxs_FirstObj)
    i.TSL_ecs_CalcK                          0x08003e34   Section        0  tsl_ecs.o(i.TSL_ecs_CalcK)
    i.TSL_ecs_Process                        0x08003ee0   Section        0  tsl_ecs.o(i.TSL_ecs_Process)
    i.TSL_ecs_ProcessK                       0x08003f60   Section        0  tsl_ecs.o(i.TSL_ecs_ProcessK)
    i.TSL_linrot_CalcPos                     0x08004020   Section        0  tsl_linrot.o(i.TSL_linrot_CalcPos)
    i.TSL_linrot_CalibrationStateProcess     0x080042b4   Section        0  tsl_linrot.o(i.TSL_linrot_CalibrationStateProcess)
    i.TSL_linrot_DTOGetTime                  0x0800437c   Section        0  tsl_linrot.o(i.TSL_linrot_DTOGetTime)
    i.TSL_linrot_DebCalibrationStateProcess  0x080043b0   Section        0  tsl_linrot.o(i.TSL_linrot_DebCalibrationStateProcess)
    i.TSL_linrot_DebDetectStateProcess       0x080043f8   Section        0  tsl_linrot.o(i.TSL_linrot_DebDetectStateProcess)
    i.TSL_linrot_DebErrorStateProcess        0x08004470   Section        0  tsl_linrot.o(i.TSL_linrot_DebErrorStateProcess)
    i.TSL_linrot_DebProxDetectStateProcess   0x080044dc   Section        0  tsl_linrot.o(i.TSL_linrot_DebProxDetectStateProcess)
    i.TSL_linrot_DebProxStateProcess         0x08004554   Section        0  tsl_linrot.o(i.TSL_linrot_DebProxStateProcess)
    i.TSL_linrot_DebProxTouchStateProcess    0x080045cc   Section        0  tsl_linrot.o(i.TSL_linrot_DebProxTouchStateProcess)
    i.TSL_linrot_DebReleaseDetectStateProcess 0x08004644   Section        0  tsl_linrot.o(i.TSL_linrot_DebReleaseDetectStateProcess)
    i.TSL_linrot_DebReleaseProxStateProcess  0x080046a0   Section        0  tsl_linrot.o(i.TSL_linrot_DebReleaseProxStateProcess)
    i.TSL_linrot_DebReleaseTouchStateProcess 0x080046e8   Section        0  tsl_linrot.o(i.TSL_linrot_DebReleaseTouchStateProcess)
    i.TSL_linrot_DetectStateProcess          0x08004744   Section        0  tsl_linrot.o(i.TSL_linrot_DetectStateProcess)
    i.TSL_linrot_GetStateMask                0x08004814   Section        0  tsl_linrot.o(i.TSL_linrot_GetStateMask)
    i.TSL_linrot_Init                        0x08004838   Section        0  tsl_linrot.o(i.TSL_linrot_Init)
    i.TSL_linrot_Process                     0x080048a8   Section        0  tsl_linrot.o(i.TSL_linrot_Process)
    i.TSL_linrot_ProcessCh_All_ClearRef      0x080048f8   Section        0  tsl_linrot.o(i.TSL_linrot_ProcessCh_All_ClearRef)
    i.TSL_linrot_ProcessCh_All_DeltaBelowEqu 0x08004920   Section        0  tsl_linrot.o(i.TSL_linrot_ProcessCh_All_DeltaBelowEqu)
    i.TSL_linrot_ProcessCh_All_SetStatus     0x0800494c   Section        0  tsl_linrot.o(i.TSL_linrot_ProcessCh_All_SetStatus)
    i.TSL_linrot_ProcessCh_One_AcqStatusError 0x0800497c   Section        0  tsl_linrot.o(i.TSL_linrot_ProcessCh_One_AcqStatusError)
    i.TSL_linrot_ProcessCh_One_DataReady     0x080049a8   Section        0  tsl_linrot.o(i.TSL_linrot_ProcessCh_One_DataReady)
    i.TSL_linrot_ProcessCh_One_DeltaAbove    0x080049d8   Section        0  tsl_linrot.o(i.TSL_linrot_ProcessCh_One_DeltaAbove)
    i.TSL_linrot_ProcessCh_One_DeltaAboveEqu 0x08004a04   Section        0  tsl_linrot.o(i.TSL_linrot_ProcessCh_One_DeltaAboveEqu)
    i.TSL_linrot_ProcessCh_One_DeltaBelowEquMinus 0x08004a30   Section        0  tsl_linrot.o(i.TSL_linrot_ProcessCh_One_DeltaBelowEquMinus)
    i.TSL_linrot_ProxStateProcess            0x08004a60   Section        0  tsl_linrot.o(i.TSL_linrot_ProxStateProcess)
    i.TSL_linrot_ReleaseStateProcess         0x08004b10   Section        0  tsl_linrot.o(i.TSL_linrot_ReleaseStateProcess)
    i.TSL_linrot_SetStateCalibration         0x08004bc0   Section        0  tsl_linrot.o(i.TSL_linrot_SetStateCalibration)
    i.TSL_linrot_TouchStateProcess           0x08004c1c   Section        0  tsl_linrot.o(i.TSL_linrot_TouchStateProcess)
    i.TSL_obj_GroupInit                      0x08004cec   Section        0  tsl_object.o(i.TSL_obj_GroupInit)
    i.TSL_obj_GroupProcess                   0x08004d48   Section        0  tsl_object.o(i.TSL_obj_GroupProcess)
    i.TSL_obj_SetGlobalObj                   0x08004da4   Section        0  tsl_object.o(i.TSL_obj_SetGlobalObj)
    i.TSL_tim_CheckDelay_ms                  0x08004dc4   Section        0  tsl_time.o(i.TSL_tim_CheckDelay_ms)
    i.TSL_tim_CheckDelay_sec                 0x08004e1c   Section        0  tsl_time.o(i.TSL_tim_CheckDelay_sec)
    i.USBClock_Disable                       0x08004e74   Section        0  menu.o(i.USBClock_Disable)
    i.USBClock_Enable                        0x08004e98   Section        0  menu.o(i.USBClock_Enable)
    i.USBD_ClrClassConfig                    0x08004eec   Section        0  usbd_core.o(i.USBD_ClrClassConfig)
    i.USBD_CtlContinueRx                     0x08004efc   Section        0  usbd_ioreq.o(i.USBD_CtlContinueRx)
    i.USBD_CtlContinueSendData               0x08004f0c   Section        0  usbd_ioreq.o(i.USBD_CtlContinueSendData)
    i.USBD_CtlError                          0x08004f1c   Section        0  usbd_ctlreq.o(i.USBD_CtlError)
    i.USBD_CtlReceiveStatus                  0x08004f30   Section        0  usbd_ioreq.o(i.USBD_CtlReceiveStatus)
    i.USBD_CtlSendData                       0x08004f48   Section        0  usbd_ioreq.o(i.USBD_CtlSendData)
    i.USBD_CtlSendStatus                     0x08004f64   Section        0  usbd_ioreq.o(i.USBD_CtlSendStatus)
    i.USBD_DeInit                            0x08004f7c   Section        0  usbd_core.o(i.USBD_DeInit)
    i.USBD_GetDescriptor                     0x08004fa6   Section        0  usbd_ctlreq.o(i.USBD_GetDescriptor)
    USBD_GetDescriptor                       0x08004fa7   Thumb Code   224  usbd_ctlreq.o(i.USBD_GetDescriptor)
    i.USBD_GetString                         0x08005086   Section        0  usbd_ctlreq.o(i.USBD_GetString)
    i.USBD_HID_ConfigStrDescriptor           0x080050cc   Section        0  usbd_desc.o(i.USBD_HID_ConfigStrDescriptor)
    i.USBD_HID_DataIn                        0x080050ec   Section        0  usbd_hid.o(i.USBD_HID_DataIn)
    USBD_HID_DataIn                          0x080050ed   Thumb Code    16  usbd_hid.o(i.USBD_HID_DataIn)
    i.USBD_HID_DeInit                        0x080050fc   Section        0  usbd_hid.o(i.USBD_HID_DeInit)
    USBD_HID_DeInit                          0x080050fd   Thumb Code    34  usbd_hid.o(i.USBD_HID_DeInit)
    i.USBD_HID_DeviceDescriptor              0x08005120   Section        0  usbd_desc.o(i.USBD_HID_DeviceDescriptor)
    i.USBD_HID_GetCfgDesc                    0x0800512c   Section        0  usbd_hid.o(i.USBD_HID_GetCfgDesc)
    USBD_HID_GetCfgDesc                      0x0800512d   Thumb Code     8  usbd_hid.o(i.USBD_HID_GetCfgDesc)
    i.USBD_HID_GetDeviceQualifierDesc        0x08005138   Section        0  usbd_hid.o(i.USBD_HID_GetDeviceQualifierDesc)
    USBD_HID_GetDeviceQualifierDesc          0x08005139   Thumb Code     8  usbd_hid.o(i.USBD_HID_GetDeviceQualifierDesc)
    i.USBD_HID_Init                          0x08005144   Section        0  usbd_hid.o(i.USBD_HID_Init)
    USBD_HID_Init                            0x08005145   Thumb Code    46  usbd_hid.o(i.USBD_HID_Init)
    i.USBD_HID_InterfaceStrDescriptor        0x08005174   Section        0  usbd_desc.o(i.USBD_HID_InterfaceStrDescriptor)
    i.USBD_HID_LangIDStrDescriptor           0x08005198   Section        0  usbd_desc.o(i.USBD_HID_LangIDStrDescriptor)
    i.USBD_HID_ManufacturerStrDescriptor     0x080051a4   Section        0  usbd_desc.o(i.USBD_HID_ManufacturerStrDescriptor)
    i.USBD_HID_ProductStrDescriptor          0x080051cc   Section        0  usbd_desc.o(i.USBD_HID_ProductStrDescriptor)
    i.USBD_HID_SendReport                    0x080051f8   Section        0  usbd_hid.o(i.USBD_HID_SendReport)
    i.USBD_HID_SerialStrDescriptor           0x08005224   Section        0  usbd_desc.o(i.USBD_HID_SerialStrDescriptor)
    i.USBD_HID_Setup                         0x08005258   Section        0  usbd_hid.o(i.USBD_HID_Setup)
    USBD_HID_Setup                           0x08005259   Thumb Code   154  usbd_hid.o(i.USBD_HID_Setup)
    i.USBD_Init                              0x080052f8   Section        0  usbd_core.o(i.USBD_Init)
    i.USBD_LL_ClearStallEP                   0x0800532a   Section        0  usbd_conf.o(i.USBD_LL_ClearStallEP)
    i.USBD_LL_CloseEP                        0x0800533c   Section        0  usbd_conf.o(i.USBD_LL_CloseEP)
    i.USBD_LL_DataInStage                    0x0800534e   Section        0  usbd_core.o(i.USBD_LL_DataInStage)
    i.USBD_LL_DataOutStage                   0x080053f8   Section        0  usbd_core.o(i.USBD_LL_DataOutStage)
    i.USBD_LL_DeInit                         0x0800546c   Section        0  usbd_conf.o(i.USBD_LL_DeInit)
    i.USBD_LL_Init                           0x08005480   Section        0  usbd_conf.o(i.USBD_LL_Init)
    i.USBD_LL_IsStallEP                      0x080054dc   Section        0  usbd_conf.o(i.USBD_LL_IsStallEP)
    i.USBD_LL_OpenEP                         0x08005500   Section        0  usbd_conf.o(i.USBD_LL_OpenEP)
    i.USBD_LL_PrepareReceive                 0x08005518   Section        0  usbd_conf.o(i.USBD_LL_PrepareReceive)
    i.USBD_LL_Reset                          0x0800552a   Section        0  usbd_core.o(i.USBD_LL_Reset)
    i.USBD_LL_SOF                            0x08005570   Section        0  usbd_core.o(i.USBD_LL_SOF)
    i.USBD_LL_SetSpeed                       0x0800558e   Section        0  usbd_core.o(i.USBD_LL_SetSpeed)
    i.USBD_LL_SetUSBAddress                  0x08005594   Section        0  usbd_conf.o(i.USBD_LL_SetUSBAddress)
    i.USBD_LL_SetupStage                     0x080055a6   Section        0  usbd_core.o(i.USBD_LL_SetupStage)
    i.USBD_LL_StallEP                        0x08005604   Section        0  usbd_conf.o(i.USBD_LL_StallEP)
    i.USBD_LL_Start                          0x08005616   Section        0  usbd_conf.o(i.USBD_LL_Start)
    i.USBD_LL_Stop                           0x08005628   Section        0  usbd_conf.o(i.USBD_LL_Stop)
    i.USBD_LL_Transmit                       0x0800563a   Section        0  usbd_conf.o(i.USBD_LL_Transmit)
    i.USBD_ParseSetupRequest                 0x0800564c   Section        0  usbd_ctlreq.o(i.USBD_ParseSetupRequest)
    i.USBD_RegisterClass                     0x08005674   Section        0  usbd_core.o(i.USBD_RegisterClass)
    i.USBD_SetClassConfig                    0x0800568a   Section        0  usbd_core.o(i.USBD_SetClassConfig)
    i.USBD_SetConfig                         0x080056a8   Section        0  usbd_ctlreq.o(i.USBD_SetConfig)
    USBD_SetConfig                           0x080056a9   Thumb Code   108  usbd_ctlreq.o(i.USBD_SetConfig)
    i.USBD_Start                             0x08005718   Section        0  usbd_core.o(i.USBD_Start)
    i.USBD_StdDevReq                         0x08005722   Section        0  usbd_ctlreq.o(i.USBD_StdDevReq)
    i.USBD_StdEPReq                          0x08005810   Section        0  usbd_ctlreq.o(i.USBD_StdEPReq)
    i.USBD_StdItfReq                         0x080058e0   Section        0  usbd_ctlreq.o(i.USBD_StdItfReq)
    i.USBD_static_free                       0x0800591a   Section        0  usbd_conf.o(i.USBD_static_free)
    i.USBD_static_malloc                     0x0800591c   Section        0  usbd_conf.o(i.USBD_static_malloc)
    i.USB_IRQHandler                         0x08005924   Section        0  stm32l0xx_it.o(i.USB_IRQHandler)
    i.USB_process                            0x08005934   Section        0  usbdapp.o(i.USB_process)
    i.__0sprintf$1                           0x08005970   Section        0  printf1.o(i.__0sprintf$1)
    i.__ARM_common_switch8                   0x08005998   Section        0  menu.o(i.__ARM_common_switch8)
    i.__scatterload_copy                     0x080059b2   Section       14  handlers.o(i.__scatterload_copy)
    i.__scatterload_null                     0x080059c0   Section        2  handlers.o(i.__scatterload_null)
    i.__scatterload_zeroinit                 0x080059c2   Section       14  handlers.o(i.__scatterload_zeroinit)
    i._printf_core                           0x080059d0   Section        0  printf1.o(i._printf_core)
    _printf_core                             0x080059d1   Thumb Code   332  printf1.o(i._printf_core)
    i._sputc                                 0x08005b20   Section        0  printf1.o(i._sputc)
    _sputc                                   0x08005b21   Thumb Code    10  printf1.o(i._sputc)
    i.gde021a1_CloseChargePump               0x08005b2a   Section        0  gde021a1.o(i.gde021a1_CloseChargePump)
    i.gde021a1_DrawImage                     0x08005b40   Section        0  gde021a1.o(i.gde021a1_DrawImage)
    i.gde021a1_GetEpdPixelHeight             0x08005c8a   Section        0  gde021a1.o(i.gde021a1_GetEpdPixelHeight)
    i.gde021a1_GetEpdPixelWidth              0x08005c8e   Section        0  gde021a1.o(i.gde021a1_GetEpdPixelWidth)
    i.gde021a1_Init                          0x08005c94   Section        0  gde021a1.o(i.gde021a1_Init)
    i.gde021a1_RefreshDisplay                0x08005d3c   Section        0  gde021a1.o(i.gde021a1_RefreshDisplay)
    i.gde021a1_SetDisplayWindow              0x08005d52   Section        0  gde021a1.o(i.gde021a1_SetDisplayWindow)
    i.gde021a1_WritePixel                    0x08005d9a   Section        0  gde021a1.o(i.gde021a1_WritePixel)
    i.main                                   0x08005dac   Section        0  main.o(i.main)
    i.tsl_user_Exec                          0x08005dc0   Section        0  tsl_user.o(i.tsl_user_Exec)
    i.tsl_user_Init                          0x08005e3c   Section        0  tsl_user.o(i.tsl_user_Init)
    .constdata                               0x08005e54   Section       36  tsl_user.o(.constdata)
    .constdata                               0x08005e78   Section        6  tsl_user.o(.constdata)
    .constdata                               0x08005e80   Section       24  tsl_user.o(.constdata)
    .constdata                               0x08005e98   Section      160  tsl_user.o(.constdata)
    .constdata                               0x08005f38   Section       12  tsl_user.o(.constdata)
    .constdata                               0x08005f44   Section        6  tsl_user.o(.constdata)
    .constdata                               0x08005f4c   Section       36  tsl_user.o(.constdata)
    .constdata                               0x08005f70   Section        8  tsl_user.o(.constdata)
    .constdata                               0x08005f78   Section       22  usbd_desc.o(.constdata)
    .constdata                               0x08005f8e   Section       90  gde021a1.o(.constdata)
    .constdata                               0x08005fe8   Section        8  stm32l0538_discovery.o(.constdata)
    .constdata                               0x08005ff0   Section     4180  stm32l0538_discovery_epd.o(.constdata)
    .constdata                               0x08007044   Section     1995  stm32l0538_discovery_epd.o(.constdata)
    .constdata                               0x0800780f   Section      950  stm32l0538_discovery_epd.o(.constdata)
    .constdata                               0x08007bc8   Section       28  stm32l0xx_hal_rcc.o(.constdata)
    .constdata                               0x08007be4   Section       18  tsl_linrot.o(.constdata)
    .data                                    0x20000000   Section     2240  menu.o(.data)
    Background_pic                           0x2000006c   Data        1548  menu.o(.data)
    FullSlider_pic                           0x20000678   Data         584  menu.o(.data)
    .data                                    0x200008c0   Section        4  stm32l0xx_it.o(.data)
    ticks                                    0x200008c0   Data           4  stm32l0xx_it.o(.data)
    .data                                    0x200008c4   Section       28  tsl_user.o(.data)
    idx_bank                                 0x200008c8   Data           4  tsl_user.o(.data)
    config_done                              0x200008cc   Data           4  tsl_user.o(.data)
    .data                                    0x200008e0   Section       16  tsl_user.o(.data)
    .data                                    0x200008f0   Section        8  tsl_user.o(.data)
    .data                                    0x200008f8   Section       12  power.o(.data)
    .data                                    0x20000904   Section       28  usbd_desc.o(.data)
    .data                                    0x20000920   Section       26  usbd_desc.o(.data)
    .data                                    0x2000093a   Section        4  usbdapp.o(.data)
    .data                                    0x20000940   Section       32  gde021a1.o(.data)
    .data                                    0x20000960   Section       12  stm32l0538_discovery.o(.data)
    .data                                    0x2000096c   Section       24  stm32l0538_discovery_epd.o(.data)
    pFont                                    0x2000096c   Data           4  stm32l0538_discovery_epd.o(.data)
    epd_drv                                  0x20000970   Data           4  stm32l0538_discovery_epd.o(.data)
    .data                                    0x20000984   Section        8  stm32l0538_discovery_epd.o(.data)
    .data                                    0x2000098c   Section       29  system_stm32l0xx.o(.data)
    .data                                    0x200009ac   Section        4  stm32l0xx_hal.o(.data)
    uwTick                                   0x200009ac   Data           4  stm32l0xx_hal.o(.data)
    .data                                    0x200009b0   Section       25  stm32l0xx_hal_rcc.o(.data)
    PLLMulTable                              0x200009b0   Data           9  stm32l0xx_hal_rcc.o(.data)
    APBAHBPrescTable                         0x200009b9   Data          16  stm32l0xx_hal_rcc.o(.data)
    .data                                    0x200009ca   Section       10  tsl_linrot.o(.data)
    index1                                   0x200009ca   Data           1  tsl_linrot.o(.data)
    index2                                   0x200009cb   Data           1  tsl_linrot.o(.data)
    delta1                                   0x200009cc   Data           2  tsl_linrot.o(.data)
    delta2                                   0x200009ce   Data           2  tsl_linrot.o(.data)
    delta3                                   0x200009d0   Data           2  tsl_linrot.o(.data)
    CalibDiv                                 0x200009d2   Data           2  tsl_linrot.o(.data)
    .data                                    0x200009d4   Section       56  usbd_hid.o(.data)
    .data                                    0x20000a0c   Section      134  usbd_hid.o(.data)
    USBD_HID_CfgDesc                         0x20000a0c   Data          34  usbd_hid.o(.data)
    USBD_HID_Desc                            0x20000a30   Data           9  usbd_hid.o(.data)
    USBD_HID_DeviceQualifierDesc             0x20000a3c   Data          10  usbd_hid.o(.data)
    HID_MOUSE_ReportDesc                     0x20000a48   Data          74  usbd_hid.o(.data)
    .data                                    0x20000a92   Section        1  usbd_ctlreq.o(.data)
    cfgidx                                   0x20000a92   Data           1  usbd_ctlreq.o(.data)
    .bss                                     0x20000a94   Section      612  bsp.o(.bss)
    .bss                                     0x20000cf8   Section       24  menu.o(.bss)
    RCC_CRSInitStruct                        0x20000cf8   Data          24  menu.o(.bss)
    .bss                                     0x20000d10   Section       36  tsl_user.o(.bss)
    .bss                                     0x20000d34   Section       13  tsl_user.o(.bss)
    .bss                                     0x20000d44   Section       96  power.o(.bss)
    .bss                                     0x20000da4   Section      392  usbd_conf.o(.bss)
    mem                                      0x20000da4   Data          16  usbd_conf.o(.bss)
    .bss                                     0x20000f2c   Section      256  usbd_desc.o(.bss)
    .bss                                     0x2000102c   Section       84  stm32l0538_discovery.o(.bss)
    SpiHandle                                0x2000102c   Data          84  stm32l0538_discovery.o(.bss)
    .bss                                     0x20001080   Section       24  tsl_globals.o(.bss)
    STACK                                    0x20001098   Section     2048  startup_stm32l053xx.o(STACK)

    Global Symbols

    Symbol Name                              Value     Ov Type        Size  Object(Section)

    BuildAttributes$$THM_ISAv3M$S$PE$A:L22$X:L11$S22$IEEE1$IW$USESV6$~STKCKD$USESV7$~SHL$OSPACE$ROPI$EBA8$MICROLIB$REQ8$PRES8$EABIv2 0x00000000   Number         0  anon$$obj.o ABSOLUTE
    __ARM_use_no_argv                        0x00000000   Number         0  main.o ABSOLUTE
    _printf_a                                0x00000000   Number         0  stubs.o ABSOLUTE
    _printf_c                                0x00000000   Number         0  stubs.o ABSOLUTE
    _printf_charcount                        0x00000000   Number         0  stubs.o ABSOLUTE
    _printf_d                                0x00000000   Number         0  stubs.o ABSOLUTE
    _printf_e                                0x00000000   Number         0  stubs.o ABSOLUTE
    _printf_f                                0x00000000   Number         0  stubs.o ABSOLUTE
    _printf_flags                            0x00000000   Number         0  stubs.o ABSOLUTE
    _printf_fp_dec                           0x00000000   Number         0  stubs.o ABSOLUTE
    _printf_fp_hex                           0x00000000   Number         0  stubs.o ABSOLUTE
    _printf_g                                0x00000000   Number         0  stubs.o ABSOLUTE
    _printf_i                                0x00000000   Number         0  stubs.o ABSOLUTE
    _printf_int_dec                          0x00000000   Number         0  stubs.o ABSOLUTE
    _printf_l                                0x00000000   Number         0  stubs.o ABSOLUTE
    _printf_lc                               0x00000000   Number         0  stubs.o ABSOLUTE
    _printf_ll                               0x00000000   Number         0  stubs.o ABSOLUTE
    _printf_lld                              0x00000000   Number         0  stubs.o ABSOLUTE
    _printf_lli                              0x00000000   Number         0  stubs.o ABSOLUTE
    _printf_llo                              0x00000000   Number         0  stubs.o ABSOLUTE
    _printf_llu                              0x00000000   Number         0  stubs.o ABSOLUTE
    _printf_llx                              0x00000000   Number         0  stubs.o ABSOLUTE
    _printf_longlong_dec                     0x00000000   Number         0  stubs.o ABSOLUTE
    _printf_longlong_hex                     0x00000000   Number         0  stubs.o ABSOLUTE
    _printf_longlong_oct                     0x00000000   Number         0  stubs.o ABSOLUTE
    _printf_ls                               0x00000000   Number         0  stubs.o ABSOLUTE
    _printf_mbtowc                           0x00000000   Number         0  stubs.o ABSOLUTE
    _printf_n                                0x00000000   Number         0  stubs.o ABSOLUTE
    _printf_o                                0x00000000   Number         0  stubs.o ABSOLUTE
    _printf_p                                0x00000000   Number         0  stubs.o ABSOLUTE
    _printf_percent                          0x00000000   Number         0  stubs.o ABSOLUTE
    _printf_pre_padding                      0x00000000   Number         0  stubs.o ABSOLUTE
    _printf_return_value                     0x00000000   Number         0  stubs.o ABSOLUTE
    _printf_s                                0x00000000   Number         0  stubs.o ABSOLUTE
    _printf_sizespec                         0x00000000   Number         0  stubs.o ABSOLUTE
    _printf_str                              0x00000000   Number         0  stubs.o ABSOLUTE
    _printf_truncate_signed                  0x00000000   Number         0  stubs.o ABSOLUTE
    _printf_truncate_unsigned                0x00000000   Number         0  stubs.o ABSOLUTE
    _printf_u                                0x00000000   Number         0  stubs.o ABSOLUTE
    _printf_wc                               0x00000000   Number         0  stubs.o ABSOLUTE
    _printf_wctomb                           0x00000000   Number         0  stubs.o ABSOLUTE
    _printf_widthprec                        0x00000000   Number         0  stubs.o ABSOLUTE
    _printf_x                                0x00000000   Number         0  stubs.o ABSOLUTE
    __cpp_initialize__aeabi_                  - Undefined Weak Reference
    __cxa_finalize                            - Undefined Weak Reference
    _clock_init                               - Undefined Weak Reference
    _microlib_exit                            - Undefined Weak Reference
    __Vectors_Size                           0x000000c0   Number         0  startup_stm32l053xx.o ABSOLUTE
    __Vectors                                0x08000000   Data           4  startup_stm32l053xx.o(RESET)
    __Vectors_End                            0x080000c0   Data           0  startup_stm32l053xx.o(RESET)
    __main                                   0x080000c1   Thumb Code     0  entry.o(.ARM.Collect$$$$00000000)
    _main_stk                                0x080000c1   Thumb Code     0  entry2.o(.ARM.Collect$$$$00000001)
    _main_scatterload                        0x080000c5   Thumb Code     0  entry5.o(.ARM.Collect$$$$00000004)
    __main_after_scatterload                 0x080000c9   Thumb Code     0  entry5.o(.ARM.Collect$$$$00000004)
    _main_clock                              0x080000c9   Thumb Code     0  entry7b.o(.ARM.Collect$$$$00000008)
    _main_cpp_init                           0x080000c9   Thumb Code     0  entry8b.o(.ARM.Collect$$$$0000000A)
    _main_init                               0x080000c9   Thumb Code     0  entry9a.o(.ARM.Collect$$$$0000000B)
    __rt_final_cpp                           0x080000d1   Thumb Code     0  entry10a.o(.ARM.Collect$$$$0000000D)
    __rt_final_exit                          0x080000d1   Thumb Code     0  entry11a.o(.ARM.Collect$$$$0000000F)
    Reset_Handler                            0x080000d5   Thumb Code     8  startup_stm32l053xx.o(.text)
    ADC1_COMP_IRQHandler                     0x080000e9   Thumb Code     0  startup_stm32l053xx.o(.text)
    DMA1_Channel1_IRQHandler                 0x080000e9   Thumb Code     0  startup_stm32l053xx.o(.text)
    DMA1_Channel2_3_IRQHandler               0x080000e9   Thumb Code     0  startup_stm32l053xx.o(.text)
    DMA1_Channel4_5_6_7_IRQHandler           0x080000e9   Thumb Code     0  startup_stm32l053xx.o(.text)
    EXTI2_3_IRQHandler                       0x080000e9   Thumb Code     0  startup_stm32l053xx.o(.text)
    FLASH_IRQHandler                         0x080000e9   Thumb Code     0  startup_stm32l053xx.o(.text)
    I2C1_IRQHandler                          0x080000e9   Thumb Code     0  startup_stm32l053xx.o(.text)
    I2C2_IRQHandler                          0x080000e9   Thumb Code     0  startup_stm32l053xx.o(.text)
    LCD_IRQHandler                           0x080000e9   Thumb Code     0  startup_stm32l053xx.o(.text)
    LPTIM1_IRQHandler                        0x080000e9   Thumb Code     0  startup_stm32l053xx.o(.text)
    PVD_IRQHandler                           0x080000e9   Thumb Code     0  startup_stm32l053xx.o(.text)
    RCC_CRS_IRQHandler                       0x080000e9   Thumb Code     0  startup_stm32l053xx.o(.text)
    RNG_LPUART1_IRQHandler                   0x080000e9   Thumb Code     0  startup_stm32l053xx.o(.text)
    RTC_IRQHandler                           0x080000e9   Thumb Code     0  startup_stm32l053xx.o(.text)
    SPI1_IRQHandler                          0x080000e9   Thumb Code     0  startup_stm32l053xx.o(.text)
    SPI2_IRQHandler                          0x080000e9   Thumb Code     0  startup_stm32l053xx.o(.text)
    TIM21_IRQHandler                         0x080000e9   Thumb Code     0  startup_stm32l053xx.o(.text)
    TIM22_IRQHandler                         0x080000e9   Thumb Code     0  startup_stm32l053xx.o(.text)
    TIM2_IRQHandler                          0x080000e9   Thumb Code     0  startup_stm32l053xx.o(.text)
    TIM6_DAC_IRQHandler                      0x080000e9   Thumb Code     0  startup_stm32l053xx.o(.text)
    TSC_IRQHandler                           0x080000e9   Thumb Code     0  startup_stm32l053xx.o(.text)
    USART1_IRQHandler                        0x080000e9   Thumb Code     0  startup_stm32l053xx.o(.text)
    USART2_IRQHandler                        0x080000e9   Thumb Code     0  startup_stm32l053xx.o(.text)
    WWDG_IRQHandler                          0x080000e9   Thumb Code     0  startup_stm32l053xx.o(.text)
    __aeabi_uidiv                            0x080000f5   Thumb Code     0  uidiv.o(.text)
    __aeabi_uidivmod                         0x080000f5   Thumb Code    44  uidiv.o(.text)
    __aeabi_idiv                             0x08000121   Thumb Code     0  idiv.o(.text)
    __aeabi_idivmod                          0x08000121   Thumb Code    40  idiv.o(.text)
    __scatterload                            0x08000149   Thumb Code    28  init.o(.text)
    __scatterload_rt2                        0x08000149   Thumb Code     0  init.o(.text)
    __decompress                             0x0800016d   Thumb Code     0  __dczerorl2.o(.text)
    __decompress1                            0x0800016d   Thumb Code    86  __dczerorl2.o(.text)
    BSP_EPD_Clear                            0x080001c5   Thumb Code    40  stm32l0538_discovery_epd.o(i.BSP_EPD_Clear)
    BSP_EPD_DisplayChar                      0x080001f5   Thumb Code    70  stm32l0538_discovery_epd.o(i.BSP_EPD_DisplayChar)
    BSP_EPD_DisplayStringAt                  0x08000241   Thumb Code   150  stm32l0538_discovery_epd.o(i.BSP_EPD_DisplayStringAt)
    BSP_EPD_DrawHLine                        0x080002dd   Thumb Code    38  stm32l0538_discovery_epd.o(i.BSP_EPD_DrawHLine)
    BSP_EPD_DrawImage                        0x08000309   Thumb Code    88  stm32l0538_discovery_epd.o(i.BSP_EPD_DrawImage)
    BSP_EPD_DrawRect                         0x08000365   Thumb Code    52  stm32l0538_discovery_epd.o(i.BSP_EPD_DrawRect)
    BSP_EPD_DrawVLine                        0x08000399   Thumb Code    38  stm32l0538_discovery_epd.o(i.BSP_EPD_DrawVLine)
    BSP_EPD_GetXSize                         0x080003c5   Thumb Code     8  stm32l0538_discovery_epd.o(i.BSP_EPD_GetXSize)
    BSP_EPD_GetYSize                         0x080003d1   Thumb Code     8  stm32l0538_discovery_epd.o(i.BSP_EPD_GetYSize)
    BSP_EPD_Init                             0x080003dd   Thumb Code    34  stm32l0538_discovery_epd.o(i.BSP_EPD_Init)
    BSP_EPD_RefreshDisplay                   0x08000409   Thumb Code    48  stm32l0538_discovery_epd.o(i.BSP_EPD_RefreshDisplay)
    BSP_EPD_SetFont                          0x08000441   Thumb Code     6  stm32l0538_discovery_epd.o(i.BSP_EPD_SetFont)
    BSP_LED_Init                             0x0800044d   Thumb Code    64  stm32l0538_discovery.o(i.BSP_LED_Init)
    BSP_LED_Off                              0x08000499   Thumb Code    22  stm32l0538_discovery.o(i.BSP_LED_Off)
    BSP_LED_Toggle                           0x080004b9   Thumb Code    20  stm32l0538_discovery.o(i.BSP_LED_Toggle)
    BSP_PB_Init                              0x080004d5   Thumb Code    96  stm32l0538_discovery.o(i.BSP_PB_Init)
    BSP_TSL_Init                             0x08000545   Thumb Code    68  bsp.o(i.BSP_TSL_Init)
    BSP_USB_Init                             0x08000591   Thumb Code    28  bsp.o(i.BSP_USB_Init)
    Bsp_Init                                 0x080005b9   Thumb Code    32  bsp.o(i.Bsp_Init)
    DebugMon_Handler                         0x080005d9   Thumb Code     2  stm32l0xx_it.o(i.DebugMon_Handler)
    EPD_Delay                                0x080005db   Thumb Code     8  stm32l0538_discovery.o(i.EPD_Delay)
    EPD_IO_Init                              0x080005e5   Thumb Code   176  stm32l0538_discovery.o(i.EPD_IO_Init)
    EPD_IO_WriteData                         0x0800069d   Thumb Code    50  stm32l0538_discovery.o(i.EPD_IO_WriteData)
    EPD_IO_WriteReg                          0x080006d5   Thumb Code    50  stm32l0538_discovery.o(i.EPD_IO_WriteReg)
    EXTI0_1_IRQHandler                       0x0800070d   Thumb Code    10  stm32l0xx_it.o(i.EXTI0_1_IRQHandler)
    EXTI4_15_IRQHandler                      0x08000717   Thumb Code    12  stm32l0xx_it.o(i.EXTI4_15_IRQHandler)
    GetPointerData                           0x08000725   Thumb Code    52  usbdapp.o(i.GetPointerData)
    HAL_Delay                                0x0800075d   Thumb Code    22  stm32l0xx_hal.o(i.HAL_Delay)
    HAL_GPIO_DeInit                          0x08000775   Thumb Code   128  stm32l0xx_hal_gpio.o(i.HAL_GPIO_DeInit)
    HAL_GPIO_EXTI_Callback                   0x080007fd   Thumb Code    10  menu.o(i.HAL_GPIO_EXTI_Callback)
    HAL_GPIO_EXTI_IRQHandler                 0x0800080d   Thumb Code    18  stm32l0xx_hal_gpio.o(i.HAL_GPIO_EXTI_IRQHandler)
    HAL_GPIO_Init                            0x08000825   Thumb Code   342  stm32l0xx_hal_gpio.o(i.HAL_GPIO_Init)
    HAL_GPIO_ReadPin                         0x08000999   Thumb Code    10  stm32l0xx_hal_gpio.o(i.HAL_GPIO_ReadPin)
    HAL_GPIO_TogglePin                       0x080009a3   Thumb Code     8  stm32l0xx_hal_gpio.o(i.HAL_GPIO_TogglePin)
    HAL_GPIO_WritePin                        0x080009ab   Thumb Code    12  stm32l0xx_hal_gpio.o(i.HAL_GPIO_WritePin)
    HAL_GetTick                              0x080009b9   Thumb Code     6  stm32l0xx_hal.o(i.HAL_GetTick)
    HAL_I2C_DeInit                           0x080009c5   Thumb Code    44  stm32l0xx_hal_i2c.o(i.HAL_I2C_DeInit)
    HAL_I2C_Init                             0x080009f1   Thumb Code   156  stm32l0xx_hal_i2c.o(i.HAL_I2C_Init)
    HAL_I2C_Mem_Read                         0x08000a91   Thumb Code   272  stm32l0xx_hal_i2c.o(i.HAL_I2C_Mem_Read)
    HAL_I2C_Mem_Write                        0x08000ba5   Thumb Code   258  stm32l0xx_hal_i2c.o(i.HAL_I2C_Mem_Write)
    HAL_I2C_MspDeInit                        0x08000cad   Thumb Code    48  stm32l0xx_hal_msp.o(i.HAL_I2C_MspDeInit)
    HAL_I2C_MspInit                          0x08000ce5   Thumb Code    88  stm32l0xx_hal_msp.o(i.HAL_I2C_MspInit)
    HAL_IncTick                              0x08000d45   Thumb Code    10  stm32l0xx_hal.o(i.HAL_IncTick)
    HAL_Init                                 0x08000d55   Thumb Code    34  stm32l0xx_hal.o(i.HAL_Init)
    HAL_InitTick                             0x08000d7d   Thumb Code    34  stm32l0xx_hal.o(i.HAL_InitTick)
    HAL_MspInit                              0x08000d9f   Thumb Code     2  stm32l0xx_hal_msp.o(i.HAL_MspInit)
    HAL_NVIC_DisableIRQ                      0x08000da1   Thumb Code    14  stm32l0xx_hal_cortex.o(i.HAL_NVIC_DisableIRQ)
    HAL_NVIC_EnableIRQ                       0x08000db5   Thumb Code    14  stm32l0xx_hal_cortex.o(i.HAL_NVIC_EnableIRQ)
    HAL_NVIC_SetPriority                     0x08000dc9   Thumb Code     8  stm32l0xx_hal_cortex.o(i.HAL_NVIC_SetPriority)
    HAL_PCDEx_PMAConfig                      0x08000dd1   Thumb Code    56  stm32l0xx_hal_pcd_ex.o(i.HAL_PCDEx_PMAConfig)
    HAL_PCD_DataInStageCallback              0x08000e09   Thumb Code    22  usbd_conf.o(i.HAL_PCD_DataInStageCallback)
    HAL_PCD_DataOutStageCallback             0x08000e1f   Thumb Code    24  usbd_conf.o(i.HAL_PCD_DataOutStageCallback)
    HAL_PCD_DeInit                           0x08000e37   Thumb Code    40  stm32l0xx_hal_pcd.o(i.HAL_PCD_DeInit)
    HAL_PCD_EP_Close                         0x08000e61   Thumb Code   356  stm32l0xx_hal_pcd.o(i.HAL_PCD_EP_Close)
    HAL_PCD_EP_ClrStall                      0x08000fd1   Thumb Code   168  stm32l0xx_hal_pcd.o(i.HAL_PCD_EP_ClrStall)
    HAL_PCD_EP_Open                          0x08001085   Thumb Code   678  stm32l0xx_hal_pcd.o(i.HAL_PCD_EP_Open)
    HAL_PCD_EP_Receive                       0x08001345   Thumb Code   198  stm32l0xx_hal_pcd.o(i.HAL_PCD_EP_Receive)
    HAL_PCD_EP_SetStall                      0x08001419   Thumb Code   134  stm32l0xx_hal_pcd.o(i.HAL_PCD_EP_SetStall)
    HAL_PCD_EP_Transmit                      0x080014ad   Thumb Code   306  stm32l0xx_hal_pcd.o(i.HAL_PCD_EP_Transmit)
    HAL_PCD_IRQHandler                       0x080015f1   Thumb Code   210  stm32l0xx_hal_pcd.o(i.HAL_PCD_IRQHandler)
    HAL_PCD_Init                             0x080016e1   Thumb Code   146  stm32l0xx_hal_pcd.o(i.HAL_PCD_Init)
    HAL_PCD_MspDeInit                        0x08001775   Thumb Code    56  usbd_conf.o(i.HAL_PCD_MspDeInit)
    HAL_PCD_MspInit                          0x080017b1   Thumb Code    74  usbd_conf.o(i.HAL_PCD_MspInit)
    HAL_PCD_ResetCallback                    0x08001801   Thumb Code    22  usbd_conf.o(i.HAL_PCD_ResetCallback)
    HAL_PCD_ResumeCallback                   0x08001817   Thumb Code     2  usbd_conf.o(i.HAL_PCD_ResumeCallback)
    HAL_PCD_SOFCallback                      0x08001819   Thumb Code    14  usbd_conf.o(i.HAL_PCD_SOFCallback)
    HAL_PCD_SetAddress                       0x08001827   Thumb Code    44  stm32l0xx_hal_pcd.o(i.HAL_PCD_SetAddress)
    HAL_PCD_SetupStageCallback               0x08001853   Thumb Code    22  usbd_conf.o(i.HAL_PCD_SetupStageCallback)
    HAL_PCD_Start                            0x08001869   Thumb Code    18  stm32l0xx_hal_pcd.o(i.HAL_PCD_Start)
    HAL_PCD_Stop                             0x0800187b   Thumb Code    48  stm32l0xx_hal_pcd.o(i.HAL_PCD_Stop)
    HAL_PCD_SuspendCallback                  0x080018ab   Thumb Code     2  usbd_conf.o(i.HAL_PCD_SuspendCallback)
    HAL_PWREx_EnableFastWakeUp               0x080018ad   Thumb Code    12  stm32l0xx_hal_pwr_ex.o(i.HAL_PWREx_EnableFastWakeUp)
    HAL_PWREx_EnableUltraLowPower            0x080018bd   Thumb Code    12  stm32l0xx_hal_pwr_ex.o(i.HAL_PWREx_EnableUltraLowPower)
    HAL_PWR_EnterSLEEPMode                   0x080018cd   Thumb Code    38  stm32l0xx_hal_pwr.o(i.HAL_PWR_EnterSLEEPMode)
    HAL_RCCEx_CRSConfig                      0x080018fd   Thumb Code   116  stm32l0xx_hal_rcc_ex.o(i.HAL_RCCEx_CRSConfig)
    HAL_RCCEx_PeriphCLKConfig                0x08001979   Thumb Code   302  stm32l0xx_hal_rcc_ex.o(i.HAL_RCCEx_PeriphCLKConfig)
    HAL_RCC_ClockConfig                      0x08001ab5   Thumb Code   502  stm32l0xx_hal_rcc.o(i.HAL_RCC_ClockConfig)
    HAL_RCC_GetHCLKFreq                      0x08001cb9   Thumb Code    26  stm32l0xx_hal_rcc.o(i.HAL_RCC_GetHCLKFreq)
    HAL_RCC_GetSysClockFreq                  0x08001ce1   Thumb Code    96  stm32l0xx_hal_rcc.o(i.HAL_RCC_GetSysClockFreq)
    HAL_RCC_OscConfig                        0x08001d59   Thumb Code   936  stm32l0xx_hal_rcc.o(i.HAL_RCC_OscConfig)
    HAL_ResumeTick                           0x0800211d   Thumb Code    12  stm32l0xx_hal.o(i.HAL_ResumeTick)
    HAL_SPI_DeInit                           0x0800212d   Thumb Code    44  stm32l0xx_hal_spi.o(i.HAL_SPI_DeInit)
    HAL_SPI_GetState                         0x08002159   Thumb Code     6  stm32l0xx_hal_spi.o(i.HAL_SPI_GetState)
    HAL_SPI_Init                             0x0800215f   Thumb Code   130  stm32l0xx_hal_spi.o(i.HAL_SPI_Init)
    HAL_SPI_MspDeInit                        0x080021e1   Thumb Code     2  stm32l0xx_hal_spi.o(i.HAL_SPI_MspDeInit)
    HAL_SPI_MspInit                          0x080021e3   Thumb Code     2  stm32l0xx_hal_spi.o(i.HAL_SPI_MspInit)
    HAL_SPI_Transmit                         0x080021e5   Thumb Code   332  stm32l0xx_hal_spi.o(i.HAL_SPI_Transmit)
    HAL_SYSTICK_Config                       0x08002331   Thumb Code    38  stm32l0xx_hal_cortex.o(i.HAL_SYSTICK_Config)
    HAL_SuspendTick                          0x08002361   Thumb Code    12  stm32l0xx_hal.o(i.HAL_SuspendTick)
    HAL_TSC_DeInit                           0x08002371   Thumb Code    32  stm32l0xx_hal_tsc.o(i.HAL_TSC_DeInit)
    HAL_TSC_Init                             0x08002391   Thumb Code   162  stm32l0xx_hal_tsc.o(i.HAL_TSC_Init)
    HAL_TSC_MspDeInit                        0x08002435   Thumb Code    90  stm32l0xx_hal_msp.o(i.HAL_TSC_MspDeInit)
    HAL_TSC_MspInit                          0x08002499   Thumb Code   106  stm32l0xx_hal_msp.o(i.HAL_TSC_MspInit)
    HardFault_Handler                        0x0800250d   Thumb Code     2  stm32l0xx_it.o(i.HardFault_Handler)
    IDD_RestoreContext                       0x080027e5   Thumb Code   194  menu.o(i.IDD_RestoreContext)
    IDD_SaveContext                          0x080028c1   Thumb Code   298  menu.o(i.IDD_SaveContext)
    Idd_LPSleep_process                      0x08002a0d   Thumb Code   640  power.o(i.Idd_LPSleep_process)
    Idd_Run_process                          0x08002cb9   Thumb Code   414  power.o(i.Idd_Run_process)
    Idd_Sleep_process                        0x08002e75   Thumb Code   504  power.o(i.Idd_Sleep_process)
    Menu_Process                             0x080030c1   Thumb Code   786  menu.o(i.Menu_Process)
    MyLinRots_ErrorStateProcess              0x0800359d   Thumb Code     2  tsl_user.o(i.MyLinRots_ErrorStateProcess)
    MyLinRots_OffStateProcess                0x0800359f   Thumb Code     2  tsl_user.o(i.MyLinRots_OffStateProcess)
    NMI_Handler                              0x080035a1   Thumb Code     2  stm32l0xx_it.o(i.NMI_Handler)
    PCD_ReadPMA                              0x08003921   Thumb Code    30  stm32l0xx_hal_pcd.o(i.PCD_ReadPMA)
    PCD_WritePMA                             0x0800393f   Thumb Code    38  stm32l0xx_hal_pcd.o(i.PCD_WritePMA)
    PendSV_Handler                           0x08003965   Thumb Code     2  stm32l0xx_it.o(i.PendSV_Handler)
    SVC_Handler                              0x08003ad9   Thumb Code     2  stm32l0xx_it.o(i.SVC_Handler)
    SysTick_Handler                          0x08003ae5   Thumb Code    42  stm32l0xx_it.o(i.SysTick_Handler)
    SystemClock_Config                       0x08003b19   Thumb Code    78  menu.o(i.SystemClock_Config)
    SystemInit                               0x08003b71   Thumb Code    66  system_stm32l0xx.o(i.SystemInit)
    TSL_Init                                 0x08003be9   Thumb Code    34  tsl.o(i.TSL_Init)
    TSL_acq_BankConfig                       0x08003c19   Thumb Code    90  tsl_acq_tsc.o(i.TSL_acq_BankConfig)
    TSL_acq_BankGetResult                    0x08003c7d   Thumb Code   290  tsl_acq.o(i.TSL_acq_BankGetResult)
    TSL_acq_BankStartAcq                     0x08003da9   Thumb Code    38  tsl_acq_tsc.o(i.TSL_acq_BankStartAcq)
    TSL_acq_BankWaitEOC                      0x08003dd9   Thumb Code    32  tsl_acq_tsc.o(i.TSL_acq_BankWaitEOC)
    TSL_acq_CheckNoise                       0x08003dfd   Thumb Code     4  tsl_acq_tsc.o(i.TSL_acq_CheckNoise)
    TSL_acq_ComputeDelta                     0x08003e01   Thumb Code     6  tsl_acq_tsc.o(i.TSL_acq_ComputeDelta)
    TSL_acq_ComputeMeas                      0x08003e07   Thumb Code     6  tsl_acq_tsc.o(i.TSL_acq_ComputeMeas)
    TSL_acq_GetMeas                          0x08003e0d   Thumb Code    20  tsl_acq_tsc.o(i.TSL_acq_GetMeas)
    TSL_acq_TestFirstReferenceIsValid        0x08003e25   Thumb Code     4  tsl_acq_tsc.o(i.TSL_acq_TestFirstReferenceIsValid)
    TSL_acq_TestReferenceOutOfRange          0x08003e29   Thumb Code     4  tsl_acq_tsc.o(i.TSL_acq_TestReferenceOutOfRange)
    TSL_acq_UseFilter                        0x08003e2d   Thumb Code     4  tsl_acq_tsc.o(i.TSL_acq_UseFilter)
    TSL_dxs_FirstObj                         0x08003e31   Thumb Code     2  tsl_dxs.o(i.TSL_dxs_FirstObj)
    TSL_ecs_CalcK                            0x08003e35   Thumb Code   168  tsl_ecs.o(i.TSL_ecs_CalcK)
    TSL_ecs_Process                          0x08003ee1   Thumb Code   120  tsl_ecs.o(i.TSL_ecs_Process)
    TSL_ecs_ProcessK                         0x08003f61   Thumb Code   184  tsl_ecs.o(i.TSL_ecs_ProcessK)
    TSL_linrot_CalcPos                       0x08004021   Thumb Code   644  tsl_linrot.o(i.TSL_linrot_CalcPos)
    TSL_linrot_CalibrationStateProcess       0x080042b5   Thumb Code   186  tsl_linrot.o(i.TSL_linrot_CalibrationStateProcess)
    TSL_linrot_DTOGetTime                    0x0800437d   Thumb Code    42  tsl_linrot.o(i.TSL_linrot_DTOGetTime)
    TSL_linrot_DebCalibrationStateProcess    0x080043b1   Thumb Code    66  tsl_linrot.o(i.TSL_linrot_DebCalibrationStateProcess)
    TSL_linrot_DebDetectStateProcess         0x080043f9   Thumb Code   116  tsl_linrot.o(i.TSL_linrot_DebDetectStateProcess)
    TSL_linrot_DebErrorStateProcess          0x08004471   Thumb Code   102  tsl_linrot.o(i.TSL_linrot_DebErrorStateProcess)
    TSL_linrot_DebProxDetectStateProcess     0x080044dd   Thumb Code   114  tsl_linrot.o(i.TSL_linrot_DebProxDetectStateProcess)
    TSL_linrot_DebProxStateProcess           0x08004555   Thumb Code   116  tsl_linrot.o(i.TSL_linrot_DebProxStateProcess)
    TSL_linrot_DebProxTouchStateProcess      0x080045cd   Thumb Code   114  tsl_linrot.o(i.TSL_linrot_DebProxTouchStateProcess)
    TSL_linrot_DebReleaseDetectStateProcess  0x08004645   Thumb Code    88  tsl_linrot.o(i.TSL_linrot_DebReleaseDetectStateProcess)
    TSL_linrot_DebReleaseProxStateProcess    0x080046a1   Thumb Code    68  tsl_linrot.o(i.TSL_linrot_DebReleaseProxStateProcess)
    TSL_linrot_DebReleaseTouchStateProcess   0x080046e9   Thumb Code    88  tsl_linrot.o(i.TSL_linrot_DebReleaseTouchStateProcess)
    TSL_linrot_DetectStateProcess            0x08004745   Thumb Code   200  tsl_linrot.o(i.TSL_linrot_DetectStateProcess)
    TSL_linrot_GetStateMask                  0x08004815   Thumb Code    30  tsl_linrot.o(i.TSL_linrot_GetStateMask)
    TSL_linrot_Init                          0x08004839   Thumb Code   106  tsl_linrot.o(i.TSL_linrot_Init)
    TSL_linrot_Process                       0x080048a9   Thumb Code    74  tsl_linrot.o(i.TSL_linrot_Process)
    TSL_linrot_ProcessCh_All_ClearRef        0x080048f9   Thumb Code    34  tsl_linrot.o(i.TSL_linrot_ProcessCh_All_ClearRef)
    TSL_linrot_ProcessCh_All_DeltaBelowEqu   0x08004921   Thumb Code    40  tsl_linrot.o(i.TSL_linrot_ProcessCh_All_DeltaBelowEqu)
    TSL_linrot_ProcessCh_All_SetStatus       0x0800494d   Thumb Code    42  tsl_linrot.o(i.TSL_linrot_ProcessCh_All_SetStatus)
    TSL_linrot_ProcessCh_One_AcqStatusError  0x0800497d   Thumb Code    40  tsl_linrot.o(i.TSL_linrot_ProcessCh_One_AcqStatusError)
    TSL_linrot_ProcessCh_One_DataReady       0x080049a9   Thumb Code    44  tsl_linrot.o(i.TSL_linrot_ProcessCh_One_DataReady)
    TSL_linrot_ProcessCh_One_DeltaAbove      0x080049d9   Thumb Code    40  tsl_linrot.o(i.TSL_linrot_ProcessCh_One_DeltaAbove)
    TSL_linrot_ProcessCh_One_DeltaAboveEqu   0x08004a05   Thumb Code    40  tsl_linrot.o(i.TSL_linrot_ProcessCh_One_DeltaAboveEqu)
    TSL_linrot_ProcessCh_One_DeltaBelowEquMinus 0x08004a31   Thumb Code    42  tsl_linrot.o(i.TSL_linrot_ProcessCh_One_DeltaBelowEquMinus)
    TSL_linrot_ProxStateProcess              0x08004a61   Thumb Code   166  tsl_linrot.o(i.TSL_linrot_ProxStateProcess)
    TSL_linrot_ReleaseStateProcess           0x08004b11   Thumb Code   172  tsl_linrot.o(i.TSL_linrot_ReleaseStateProcess)
    TSL_linrot_SetStateCalibration           0x08004bc1   Thumb Code    78  tsl_linrot.o(i.TSL_linrot_SetStateCalibration)
    TSL_linrot_TouchStateProcess             0x08004c1d   Thumb Code   200  tsl_linrot.o(i.TSL_linrot_TouchStateProcess)
    TSL_obj_GroupInit                        0x08004ced   Thumb Code    88  tsl_object.o(i.TSL_obj_GroupInit)
    TSL_obj_GroupProcess                     0x08004d49   Thumb Code    88  tsl_object.o(i.TSL_obj_GroupProcess)
    TSL_obj_SetGlobalObj                     0x08004da5   Thumb Code    28  tsl_object.o(i.TSL_obj_SetGlobalObj)
    TSL_tim_CheckDelay_ms                    0x08004dc5   Thumb Code    80  tsl_time.o(i.TSL_tim_CheckDelay_ms)
    TSL_tim_CheckDelay_sec                   0x08004e1d   Thumb Code    78  tsl_time.o(i.TSL_tim_CheckDelay_sec)
    USBClock_Disable                         0x08004e75   Thumb Code    32  menu.o(i.USBClock_Disable)
    USBClock_Enable                          0x08004e99   Thumb Code    70  menu.o(i.USBClock_Enable)
    USBD_ClrClassConfig                      0x08004eed   Thumb Code    16  usbd_core.o(i.USBD_ClrClassConfig)
    USBD_CtlContinueRx                       0x08004efd   Thumb Code    16  usbd_ioreq.o(i.USBD_CtlContinueRx)
    USBD_CtlContinueSendData                 0x08004f0d   Thumb Code    16  usbd_ioreq.o(i.USBD_CtlContinueSendData)
    USBD_CtlError                            0x08004f1d   Thumb Code    20  usbd_ctlreq.o(i.USBD_CtlError)
    USBD_CtlReceiveStatus                    0x08004f31   Thumb Code    24  usbd_ioreq.o(i.USBD_CtlReceiveStatus)
    USBD_CtlSendData                         0x08004f49   Thumb Code    28  usbd_ioreq.o(i.USBD_CtlSendData)
    USBD_CtlSendStatus                       0x08004f65   Thumb Code    24  usbd_ioreq.o(i.USBD_CtlSendStatus)
    USBD_DeInit                              0x08004f7d   Thumb Code    42  usbd_core.o(i.USBD_DeInit)
    USBD_GetString                           0x08005087   Thumb Code    68  usbd_ctlreq.o(i.USBD_GetString)
    USBD_HID_ConfigStrDescriptor             0x080050cd   Thumb Code    16  usbd_desc.o(i.USBD_HID_ConfigStrDescriptor)
    USBD_HID_DeviceDescriptor                0x08005121   Thumb Code     8  usbd_desc.o(i.USBD_HID_DeviceDescriptor)
    USBD_HID_InterfaceStrDescriptor          0x08005175   Thumb Code    16  usbd_desc.o(i.USBD_HID_InterfaceStrDescriptor)
    USBD_HID_LangIDStrDescriptor             0x08005199   Thumb Code     8  usbd_desc.o(i.USBD_HID_LangIDStrDescriptor)
    USBD_HID_ManufacturerStrDescriptor       0x080051a5   Thumb Code    16  usbd_desc.o(i.USBD_HID_ManufacturerStrDescriptor)
    USBD_HID_ProductStrDescriptor            0x080051cd   Thumb Code    16  usbd_desc.o(i.USBD_HID_ProductStrDescriptor)
    USBD_HID_SendReport                      0x080051f9   Thumb Code    42  usbd_hid.o(i.USBD_HID_SendReport)
    USBD_HID_SerialStrDescriptor             0x08005225   Thumb Code    44  usbd_desc.o(i.USBD_HID_SerialStrDescriptor)
    USBD_Init                                0x080052f9   Thumb Code    50  usbd_core.o(i.USBD_Init)
    USBD_LL_ClearStallEP                     0x0800532b   Thumb Code    18  usbd_conf.o(i.USBD_LL_ClearStallEP)
    USBD_LL_CloseEP                          0x0800533d   Thumb Code    18  usbd_conf.o(i.USBD_LL_CloseEP)
    USBD_LL_DataInStage                      0x0800534f   Thumb Code   170  usbd_core.o(i.USBD_LL_DataInStage)
    USBD_LL_DataOutStage                     0x080053f9   Thumb Code   116  usbd_core.o(i.USBD_LL_DataOutStage)
    USBD_LL_DeInit                           0x0800546d   Thumb Code    18  usbd_conf.o(i.USBD_LL_DeInit)
    USBD_LL_Init                             0x08005481   Thumb Code    84  usbd_conf.o(i.USBD_LL_Init)
    USBD_LL_IsStallEP                        0x080054dd   Thumb Code    36  usbd_conf.o(i.USBD_LL_IsStallEP)
    USBD_LL_OpenEP                           0x08005501   Thumb Code    24  usbd_conf.o(i.USBD_LL_OpenEP)
    USBD_LL_PrepareReceive                   0x08005519   Thumb Code    18  usbd_conf.o(i.USBD_LL_PrepareReceive)
    USBD_LL_Reset                            0x0800552b   Thumb Code    70  usbd_core.o(i.USBD_LL_Reset)
    USBD_LL_SOF                              0x08005571   Thumb Code    30  usbd_core.o(i.USBD_LL_SOF)
    USBD_LL_SetSpeed                         0x0800558f   Thumb Code     6  usbd_core.o(i.USBD_LL_SetSpeed)
    USBD_LL_SetUSBAddress                    0x08005595   Thumb Code    18  usbd_conf.o(i.USBD_LL_SetUSBAddress)
    USBD_LL_SetupStage                       0x080055a7   Thumb Code    94  usbd_core.o(i.USBD_LL_SetupStage)
    USBD_LL_StallEP                          0x08005605   Thumb Code    18  usbd_conf.o(i.USBD_LL_StallEP)
    USBD_LL_Start                            0x08005617   Thumb Code    18  usbd_conf.o(i.USBD_LL_Start)
    USBD_LL_Stop                             0x08005629   Thumb Code    18  usbd_conf.o(i.USBD_LL_Stop)
    USBD_LL_Transmit                         0x0800563b   Thumb Code    18  usbd_conf.o(i.USBD_LL_Transmit)
    USBD_ParseSetupRequest                   0x0800564d   Thumb Code    40  usbd_ctlreq.o(i.USBD_ParseSetupRequest)
    USBD_RegisterClass                       0x08005675   Thumb Code    22  usbd_core.o(i.USBD_RegisterClass)
    USBD_SetClassConfig                      0x0800568b   Thumb Code    28  usbd_core.o(i.USBD_SetClassConfig)
    USBD_Start                               0x08005719   Thumb Code    10  usbd_core.o(i.USBD_Start)
    USBD_StdDevReq                           0x08005723   Thumb Code   238  usbd_ctlreq.o(i.USBD_StdDevReq)
    USBD_StdEPReq                            0x08005811   Thumb Code   208  usbd_ctlreq.o(i.USBD_StdEPReq)
    USBD_StdItfReq                           0x080058e1   Thumb Code    58  usbd_ctlreq.o(i.USBD_StdItfReq)
    USBD_static_free                         0x0800591b   Thumb Code     2  usbd_conf.o(i.USBD_static_free)
    USBD_static_malloc                       0x0800591d   Thumb Code     4  usbd_conf.o(i.USBD_static_malloc)
    USB_IRQHandler                           0x08005925   Thumb Code    10  stm32l0xx_it.o(i.USB_IRQHandler)
    USB_process                              0x08005935   Thumb Code    48  usbdapp.o(i.USB_process)
    __0sprintf$1                             0x08005971   Thumb Code    36  printf1.o(i.__0sprintf$1)
    __1sprintf$1                             0x08005971   Thumb Code     0  printf1.o(i.__0sprintf$1)
    __2sprintf                               0x08005971   Thumb Code     0  printf1.o(i.__0sprintf$1)
    __ARM_common_switch8                     0x08005999   Thumb Code    26  menu.o(i.__ARM_common_switch8)
    __scatterload_copy                       0x080059b3   Thumb Code    14  handlers.o(i.__scatterload_copy)
    __scatterload_null                       0x080059c1   Thumb Code     2  handlers.o(i.__scatterload_null)
    __scatterload_zeroinit                   0x080059c3   Thumb Code    14  handlers.o(i.__scatterload_zeroinit)
    gde021a1_CloseChargePump                 0x08005b2b   Thumb Code    22  gde021a1.o(i.gde021a1_CloseChargePump)
    gde021a1_DrawImage                       0x08005b41   Thumb Code   330  gde021a1.o(i.gde021a1_DrawImage)
    gde021a1_GetEpdPixelHeight               0x08005c8b   Thumb Code     4  gde021a1.o(i.gde021a1_GetEpdPixelHeight)
    gde021a1_GetEpdPixelWidth                0x08005c8f   Thumb Code     4  gde021a1.o(i.gde021a1_GetEpdPixelWidth)
    gde021a1_Init                            0x08005c95   Thumb Code   164  gde021a1.o(i.gde021a1_Init)
    gde021a1_RefreshDisplay                  0x08005d3d   Thumb Code    22  gde021a1.o(i.gde021a1_RefreshDisplay)
    gde021a1_SetDisplayWindow                0x08005d53   Thumb Code    72  gde021a1.o(i.gde021a1_SetDisplayWindow)
    gde021a1_WritePixel                      0x08005d9b   Thumb Code    18  gde021a1.o(i.gde021a1_WritePixel)
    main                                     0x08005dad   Thumb Code    18  main.o(i.main)
    tsl_user_Exec                            0x08005dc1   Thumb Code   118  tsl_user.o(i.tsl_user_Exec)
    tsl_user_Init                            0x08005e3d   Thumb Code    16  tsl_user.o(i.tsl_user_Init)
    MyChannels_Src                           0x08005e54   Data          36  tsl_user.o(.constdata)
    MyChannels_Dest                          0x08005e78   Data           6  tsl_user.o(.constdata)
    MyBanks                                  0x08005e80   Data          24  tsl_user.o(.constdata)
    MyLinRots_StateMachine                   0x08005e98   Data         160  tsl_user.o(.constdata)
    MyLinRots_Methods                        0x08005f38   Data          12  tsl_user.o(.constdata)
    MyLinRot0_DeltaCoeff                     0x08005f44   Data           6  tsl_user.o(.constdata)
    MyLinRots                                0x08005f4c   Data          36  tsl_user.o(.constdata)
    MyObjects                                0x08005f70   Data           8  tsl_user.o(.constdata)
    USBD_LangIDDesc                          0x08005f78   Data           4  usbd_desc.o(.constdata)
    USBD_DeviceDesc                          0x08005f7c   Data          18  usbd_desc.o(.constdata)
    WF_LUT                                   0x08005f8e   Data          90  gde021a1.o(.constdata)
    BUTTON_IRQn                              0x08005fe8   Data           1  stm32l0538_discovery.o(.constdata)
    BUTTON_PIN                               0x08005fea   Data           2  stm32l0538_discovery.o(.constdata)
    GPIO_PIN                                 0x08005fec   Data           4  stm32l0538_discovery.o(.constdata)
    Font16_Table                             0x08005ff0   Data        4180  stm32l0538_discovery_epd.o(.constdata)
    Font12_Table                             0x08007044   Data        1995  stm32l0538_discovery_epd.o(.constdata)
    Font8_Table                              0x0800780f   Data         950  stm32l0538_discovery_epd.o(.constdata)
    MSIRangeTable                            0x08007bc8   Data          28  stm32l0xx_hal_rcc.o(.constdata)
    TSL_POSOFF_3CH_LIN_H                     0x08007be4   Data          18  tsl_linrot.o(.constdata)
    Region$$Table$$Base                      0x08007bf8   Number         0  anon$$obj.o(Region$$Table)
    Region$$Table$$Limit                     0x08007c18   Number         0  anon$$obj.o(Region$$Table)
    menu_state                               0x20000000   Data           1  menu.o(.data)
    ButtonPressed                            0x20000004   Data           4  menu.o(.data)
    GPIOA_MODER                              0x20000008   Data           4  menu.o(.data)
    GPIOA_OTYPER                             0x2000000c   Data           4  menu.o(.data)
    GPIOA_OSPEEDR                            0x20000010   Data           4  menu.o(.data)
    GPIOA_AFRL                               0x20000014   Data           4  menu.o(.data)
    GPIOA_AFRH                               0x20000018   Data           4  menu.o(.data)
    GPIOB_MODER                              0x2000001c   Data           4  menu.o(.data)
    GPIOB_OTYPER                             0x20000020   Data           4  menu.o(.data)
    GPIOB_OSPEEDR                            0x20000024   Data           4  menu.o(.data)
    GPIOB_AFRL                               0x20000028   Data           4  menu.o(.data)
    GPIOB_AFRH                               0x2000002c   Data           4  menu.o(.data)
    GPIOC_MODER                              0x20000030   Data           4  menu.o(.data)
    GPIOC_OTYPER                             0x20000034   Data           4  menu.o(.data)
    GPIOC_OSPEEDR                            0x20000038   Data           4  menu.o(.data)
    GPIOC_AFRL                               0x2000003c   Data           4  menu.o(.data)
    GPIOC_AFRH                               0x20000040   Data           4  menu.o(.data)
    GPIOD_MODER                              0x20000044   Data           4  menu.o(.data)
    GPIOD_OTYPER                             0x20000048   Data           4  menu.o(.data)
    GPIOD_OSPEEDR                            0x2000004c   Data           4  menu.o(.data)
    GPIOD_AFRL                               0x20000050   Data           4  menu.o(.data)
    GPIOD_AFRH                               0x20000054   Data           4  menu.o(.data)
    GPIOH_MODER                              0x20000058   Data           4  menu.o(.data)
    GPIOH_OTYPER                             0x2000005c   Data           4  menu.o(.data)
    GPIOH_OSPEEDR                            0x20000060   Data           4  menu.o(.data)
    GPIOH_AFRL                               0x20000064   Data           4  menu.o(.data)
    GPIOH_AFRH                               0x20000068   Data           4  menu.o(.data)
    ECSLastTick                              0x200008c4   Data           2  tsl_user.o(.data)
    MyObjGroup                               0x200008d0   Data          16  tsl_user.o(.data)
    TSL_Params                               0x200008e0   Data          16  tsl_user.o(.data)
    MyLinRots_Data                           0x200008f0   Data           8  tsl_user.o(.data)
    aRxBuffer                                0x200008f8   Data           3  power.o(.data)
    RunModeMeasure                           0x200008fc   Data           4  power.o(.data)
    Idd_measurement                          0x20000900   Data           4  power.o(.data)
    HID_Desc                                 0x20000904   Data          28  usbd_desc.o(.data)
    USBD_StringSerial                        0x20000920   Data          26  usbd_desc.o(.data)
    HID_Buffer                               0x2000093a   Data           4  usbdapp.o(.data)
    gde021a1_drv                             0x20000940   Data          32  gde021a1.o(.data)
    BUTTON_PORT                              0x20000960   Data           4  stm32l0538_discovery.o(.data)
    GPIO_PORT                                0x20000964   Data           8  stm32l0538_discovery.o(.data)
    Font16                                   0x20000974   Data           8  stm32l0538_discovery_epd.o(.data)
    Font12                                   0x2000097c   Data           8  stm32l0538_discovery_epd.o(.data)
    Font8                                    0x20000984   Data           8  stm32l0538_discovery_epd.o(.data)
    SystemCoreClock                          0x2000098c   Data           4  system_stm32l0xx.o(.data)
    AHBPrescTable                            0x20000990   Data          16  system_stm32l0xx.o(.data)
    PLLMulTable                              0x200009a0   Data           9  system_stm32l0xx.o(.data)
    USBD_HID                                 0x200009d4   Data          56  usbd_hid.o(.data)
    TscHandle                                0x20000a94   Data          64  bsp.o(.bss)
    USBD_Device                              0x20000ad4   Data         548  bsp.o(.bss)
    MyChannels_Data                          0x20000d10   Data          36  tsl_user.o(.bss)
    MyLinRots_Param                          0x20000d34   Data          13  tsl_user.o(.bss)
    I2CxHandle                               0x20000d44   Data          56  power.o(.bss)
    str                                      0x20000d7c   Data          20  power.o(.bss)
    param                                    0x20000d90   Data          20  power.o(.bss)
    hpcd                                     0x20000db4   Data         376  usbd_conf.o(.bss)
    USBD_StrDesc                             0x20000f2c   Data         256  usbd_desc.o(.bss)
    TSL_Globals                              0x20001080   Data          24  tsl_globals.o(.bss)
    __initial_sp                             0x20001898   Data           0  startup_stm32l053xx.o(STACK)



==============================================================================

Memory Map of the image

  Image Entry point : 0x080000c1

  Load Region LR_IROM1 (Base: 0x08000000, Size: 0x000086ac, Max: 0x00010000, ABSOLUTE, COMPRESSED[0x00007f04])

    Execution Region ER_IROM1 (Base: 0x08000000, Size: 0x00007c18, Max: 0x00010000, ABSOLUTE)

    Base Addr    Size         Type   Attr      Idx    E Section Name        Object

    0x08000000   0x000000c0   Data   RO            3    RESET               startup_stm32l053xx.o
    0x080000c0   0x00000000   Code   RO         3947  * .ARM.Collect$$$$00000000  mc_p.l(entry.o)
    0x080000c0   0x00000004   Code   RO         4215    .ARM.Collect$$$$00000001  mc_p.l(entry2.o)
    0x080000c4   0x00000004   Code   RO         4218    .ARM.Collect$$$$00000004  mc_p.l(entry5.o)
    0x080000c8   0x00000000   Code   RO         4220    .ARM.Collect$$$$00000008  mc_p.l(entry7b.o)
    0x080000c8   0x00000000   Code   RO         4222    .ARM.Collect$$$$0000000A  mc_p.l(entry8b.o)
    0x080000c8   0x00000008   Code   RO         4223    .ARM.Collect$$$$0000000B  mc_p.l(entry9a.o)
    0x080000d0   0x00000000   Code   RO         4225    .ARM.Collect$$$$0000000D  mc_p.l(entry10a.o)
    0x080000d0   0x00000000   Code   RO         4227    .ARM.Collect$$$$0000000F  mc_p.l(entry11a.o)
    0x080000d0   0x00000004   Code   RO         4216    .ARM.Collect$$$$00002712  mc_p.l(entry2.o)
    0x080000d4   0x00000020   Code   RO            4    .text               startup_stm32l053xx.o
    0x080000f4   0x0000002c   Code   RO         3950    .text               mc_p.l(uidiv.o)
    0x08000120   0x00000028   Code   RO         3952    .text               mc_p.l(idiv.o)
    0x08000148   0x00000024   Code   RO         4245    .text               mc_p.l(init.o)
    0x0800016c   0x00000056   Code   RO         4267    .text               mc_p.l(__dczerorl2.o)
    0x080001c2   0x00000002   PAD
    0x080001c4   0x00000030   Code   RO         1065    i.BSP_EPD_Clear     stm32l0538_discovery_epd.o
    0x080001f4   0x0000004c   Code   RO         1067    i.BSP_EPD_DisplayChar  stm32l0538_discovery_epd.o
    0x08000240   0x0000009c   Code   RO         1068    i.BSP_EPD_DisplayStringAt  stm32l0538_discovery_epd.o
    0x080002dc   0x0000002c   Code   RO         1070    i.BSP_EPD_DrawHLine  stm32l0538_discovery_epd.o
    0x08000308   0x0000005c   Code   RO         1071    i.BSP_EPD_DrawImage  stm32l0538_discovery_epd.o
    0x08000364   0x00000034   Code   RO         1072    i.BSP_EPD_DrawRect  stm32l0538_discovery_epd.o
    0x08000398   0x0000002c   Code   RO         1073    i.BSP_EPD_DrawVLine  stm32l0538_discovery_epd.o
    0x080003c4   0x0000000c   Code   RO         1076    i.BSP_EPD_GetXSize  stm32l0538_discovery_epd.o
    0x080003d0   0x0000000c   Code   RO         1077    i.BSP_EPD_GetYSize  stm32l0538_discovery_epd.o
    0x080003dc   0x0000002c   Code   RO         1078    i.BSP_EPD_Init      stm32l0538_discovery_epd.o
    0x08000408   0x00000038   Code   RO         1079    i.BSP_EPD_RefreshDisplay  stm32l0538_discovery_epd.o
    0x08000440   0x0000000c   Code   RO         1080    i.BSP_EPD_SetFont   stm32l0538_discovery_epd.o
    0x0800044c   0x0000004c   Code   RO          960    i.BSP_LED_Init      stm32l0538_discovery.o
    0x08000498   0x00000020   Code   RO          961    i.BSP_LED_Off       stm32l0538_discovery.o
    0x080004b8   0x0000001c   Code   RO          963    i.BSP_LED_Toggle    stm32l0538_discovery.o
    0x080004d4   0x00000070   Code   RO          965    i.BSP_PB_Init       stm32l0538_discovery.o
    0x08000544   0x0000004c   Code   RO           12    i.BSP_TSL_Init      bsp.o
    0x08000590   0x00000028   Code   RO           13    i.BSP_USB_Init      bsp.o
    0x080005b8   0x00000020   Code   RO           14    i.Bsp_Init          bsp.o
    0x080005d8   0x00000002   Code   RO          397    i.DebugMon_Handler  stm32l0xx_it.o
    0x080005da   0x00000008   Code   RO          966    i.EPD_Delay         stm32l0538_discovery.o
    0x080005e2   0x00000002   PAD
    0x080005e4   0x000000b8   Code   RO          967    i.EPD_IO_Init       stm32l0538_discovery.o
    0x0800069c   0x00000038   Code   RO          969    i.EPD_IO_WriteData  stm32l0538_discovery.o
    0x080006d4   0x00000038   Code   RO          970    i.EPD_IO_WriteReg   stm32l0538_discovery.o
    0x0800070c   0x0000000a   Code   RO          398    i.EXTI0_1_IRQHandler  stm32l0xx_it.o
    0x08000716   0x0000000c   Code   RO          399    i.EXTI4_15_IRQHandler  stm32l0xx_it.o
    0x08000722   0x00000002   PAD
    0x08000724   0x00000038   Code   RO          850    i.GetPointerData    usbdapp.o
    0x0800075c   0x00000016   Code   RO         1233    i.HAL_Delay         stm32l0xx_hal.o
    0x08000772   0x00000002   PAD
    0x08000774   0x00000088   Code   RO         1788    i.HAL_GPIO_DeInit   stm32l0xx_hal_gpio.o
    0x080007fc   0x00000010   Code   RO          273    i.HAL_GPIO_EXTI_Callback  menu.o
    0x0800080c   0x00000018   Code   RO         1790    i.HAL_GPIO_EXTI_IRQHandler  stm32l0xx_hal_gpio.o
    0x08000824   0x00000174   Code   RO         1791    i.HAL_GPIO_Init     stm32l0xx_hal_gpio.o
    0x08000998   0x0000000a   Code   RO         1793    i.HAL_GPIO_ReadPin  stm32l0xx_hal_gpio.o
    0x080009a2   0x00000008   Code   RO         1794    i.HAL_GPIO_TogglePin  stm32l0xx_hal_gpio.o
    0x080009aa   0x0000000c   Code   RO         1795    i.HAL_GPIO_WritePin  stm32l0xx_hal_gpio.o
    0x080009b6   0x00000002   PAD
    0x080009b8   0x0000000c   Code   RO         1244    i.HAL_GetTick       stm32l0xx_hal.o
    0x080009c4   0x0000002c   Code   RO         1850    i.HAL_I2C_DeInit    stm32l0xx_hal_i2c.o
    0x080009f0   0x000000a0   Code   RO         1856    i.HAL_I2C_Init      stm32l0xx_hal_i2c.o
    0x08000a90   0x00000114   Code   RO         1868    i.HAL_I2C_Mem_Read  stm32l0xx_hal_i2c.o
    0x08000ba4   0x00000108   Code   RO         1871    i.HAL_I2C_Mem_Write  stm32l0xx_hal_i2c.o
    0x08000cac   0x00000038   Code   RO          347    i.HAL_I2C_MspDeInit  stm32l0xx_hal_msp.o
    0x08000ce4   0x00000060   Code   RO          348    i.HAL_I2C_MspInit   stm32l0xx_hal_msp.o
    0x08000d44   0x00000010   Code   RO         1246    i.HAL_IncTick       stm32l0xx_hal.o
    0x08000d54   0x00000028   Code   RO         1247    i.HAL_Init          stm32l0xx_hal.o
    0x08000d7c   0x00000022   Code   RO         1248    i.HAL_InitTick      stm32l0xx_hal.o
    0x08000d9e   0x00000002   Code   RO          350    i.HAL_MspInit       stm32l0xx_hal_msp.o
    0x08000da0   0x00000014   Code   RO         1419    i.HAL_NVIC_DisableIRQ  stm32l0xx_hal_cortex.o
    0x08000db4   0x00000014   Code   RO         1420    i.HAL_NVIC_EnableIRQ  stm32l0xx_hal_cortex.o
    0x08000dc8   0x00000008   Code   RO         1423    i.HAL_NVIC_SetPriority  stm32l0xx_hal_cortex.o
    0x08000dd0   0x00000038   Code   RO         2421    i.HAL_PCDEx_PMAConfig  stm32l0xx_hal_pcd_ex.o
    0x08000e08   0x00000016   Code   RO          584    i.HAL_PCD_DataInStageCallback  usbd_conf.o
    0x08000e1e   0x00000018   Code   RO          585    i.HAL_PCD_DataOutStageCallback  usbd_conf.o
    0x08000e36   0x00000028   Code   RO         2206    i.HAL_PCD_DeInit    stm32l0xx_hal_pcd.o
    0x08000e5e   0x00000002   PAD
    0x08000e60   0x00000170   Code   RO         2210    i.HAL_PCD_EP_Close  stm32l0xx_hal_pcd.o
    0x08000fd0   0x000000b4   Code   RO         2211    i.HAL_PCD_EP_ClrStall  stm32l0xx_hal_pcd.o
    0x08001084   0x000002c0   Code   RO         2214    i.HAL_PCD_EP_Open   stm32l0xx_hal_pcd.o
    0x08001344   0x000000d4   Code   RO         2215    i.HAL_PCD_EP_Receive  stm32l0xx_hal_pcd.o
    0x08001418   0x00000094   Code   RO         2216    i.HAL_PCD_EP_SetStall  stm32l0xx_hal_pcd.o
    0x080014ac   0x00000144   Code   RO         2217    i.HAL_PCD_EP_Transmit  stm32l0xx_hal_pcd.o
    0x080015f0   0x000000f0   Code   RO         2219    i.HAL_PCD_IRQHandler  stm32l0xx_hal_pcd.o
    0x080016e0   0x00000092   Code   RO         2222    i.HAL_PCD_Init      stm32l0xx_hal_pcd.o
    0x08001772   0x00000002   PAD
    0x08001774   0x0000003c   Code   RO          589    i.HAL_PCD_MspDeInit  usbd_conf.o
    0x080017b0   0x00000050   Code   RO          590    i.HAL_PCD_MspInit   usbd_conf.o
    0x08001800   0x00000016   Code   RO          591    i.HAL_PCD_ResetCallback  usbd_conf.o
    0x08001816   0x00000002   Code   RO          592    i.HAL_PCD_ResumeCallback  usbd_conf.o
    0x08001818   0x0000000e   Code   RO          593    i.HAL_PCD_SOFCallback  usbd_conf.o
    0x08001826   0x0000002c   Code   RO         2228    i.HAL_PCD_SetAddress  stm32l0xx_hal_pcd.o
    0x08001852   0x00000016   Code   RO          594    i.HAL_PCD_SetupStageCallback  usbd_conf.o
    0x08001868   0x00000012   Code   RO         2230    i.HAL_PCD_Start     stm32l0xx_hal_pcd.o
    0x0800187a   0x00000030   Code   RO         2231    i.HAL_PCD_Stop      stm32l0xx_hal_pcd.o
    0x080018aa   0x00000002   Code   RO          595    i.HAL_PCD_SuspendCallback  usbd_conf.o
    0x080018ac   0x00000010   Code   RO         2536    i.HAL_PWREx_EnableFastWakeUp  stm32l0xx_hal_pwr_ex.o
    0x080018bc   0x00000010   Code   RO         2538    i.HAL_PWREx_EnableUltraLowPower  stm32l0xx_hal_pwr_ex.o
    0x080018cc   0x00000030   Code   RO         2448    i.HAL_PWR_EnterSLEEPMode  stm32l0xx_hal_pwr.o
    0x080018fc   0x0000007c   Code   RO         2679    i.HAL_RCCEx_CRSConfig  stm32l0xx_hal_rcc_ex.o
    0x08001978   0x0000013c   Code   RO         2686    i.HAL_RCCEx_PeriphCLKConfig  stm32l0xx_hal_rcc_ex.o
    0x08001ab4   0x00000204   Code   RO         2584    i.HAL_RCC_ClockConfig  stm32l0xx_hal_rcc.o
    0x08001cb8   0x00000028   Code   RO         2588    i.HAL_RCC_GetHCLKFreq  stm32l0xx_hal_rcc.o
    0x08001ce0   0x00000078   Code   RO         2592    i.HAL_RCC_GetSysClockFreq  stm32l0xx_hal_rcc.o
    0x08001d58   0x000003c4   Code   RO         2595    i.HAL_RCC_OscConfig  stm32l0xx_hal_rcc.o
    0x0800211c   0x00000010   Code   RO         1253    i.HAL_ResumeTick    stm32l0xx_hal.o
    0x0800212c   0x0000002c   Code   RO         2744    i.HAL_SPI_DeInit    stm32l0xx_hal_spi.o
    0x08002158   0x00000006   Code   RO         2747    i.HAL_SPI_GetState  stm32l0xx_hal_spi.o
    0x0800215e   0x00000082   Code   RO         2749    i.HAL_SPI_Init      stm32l0xx_hal_spi.o
    0x080021e0   0x00000002   Code   RO         2750    i.HAL_SPI_MspDeInit  stm32l0xx_hal_spi.o
    0x080021e2   0x00000002   Code   RO         2751    i.HAL_SPI_MspInit   stm32l0xx_hal_spi.o
    0x080021e4   0x0000014c   Code   RO         2757    i.HAL_SPI_Transmit  stm32l0xx_hal_spi.o
    0x08002330   0x00000030   Code   RO         1427    i.HAL_SYSTICK_Config  stm32l0xx_hal_cortex.o
    0x08002360   0x00000010   Code   RO         1254    i.HAL_SuspendTick   stm32l0xx_hal.o
    0x08002370   0x00000020   Code   RO         2977    i.HAL_TSC_DeInit    stm32l0xx_hal_tsc.o
    0x08002390   0x000000a2   Code   RO         2985    i.HAL_TSC_Init      stm32l0xx_hal_tsc.o
    0x08002432   0x00000002   PAD
    0x08002434   0x00000064   Code   RO          351    i.HAL_TSC_MspDeInit  stm32l0xx_hal_msp.o
    0x08002498   0x00000074   Code   RO          352    i.HAL_TSC_MspInit   stm32l0xx_hal_msp.o
    0x0800250c   0x00000002   Code   RO          400    i.HardFault_Handler  stm32l0xx_it.o
    0x0800250e   0x00000002   PAD
    0x08002510   0x0000003c   Code   RO          536    i.I2C_Config        power.o
    0x0800254c   0x00000094   Code   RO         1891    i.I2C_IsAcknowledgeFailed  stm32l0xx_hal_i2c.o
    0x080025e0   0x00000066   Code   RO         1894    i.I2C_RequestMemoryRead  stm32l0xx_hal_i2c.o
    0x08002646   0x00000066   Code   RO         1895    i.I2C_RequestMemoryWrite  stm32l0xx_hal_i2c.o
    0x080026ac   0x00000024   Code   RO         1898    i.I2C_TransferConfig  stm32l0xx_hal_i2c.o
    0x080026d0   0x00000070   Code   RO         1899    i.I2C_WaitOnFlagUntilTimeout  stm32l0xx_hal_i2c.o
    0x08002740   0x00000050   Code   RO         1901    i.I2C_WaitOnSTOPFlagUntilTimeout  stm32l0xx_hal_i2c.o
    0x08002790   0x00000054   Code   RO         1902    i.I2C_WaitOnTXISFlagUntilTimeout  stm32l0xx_hal_i2c.o
    0x080027e4   0x000000dc   Code   RO          274    i.IDD_RestoreContext  menu.o
    0x080028c0   0x0000014c   Code   RO          275    i.IDD_SaveContext   menu.o
    0x08002a0c   0x000002ac   Code   RO          537    i.Idd_LPSleep_process  power.o
    0x08002cb8   0x000001bc   Code   RO          538    i.Idd_Run_process   power.o
    0x08002e74   0x00000220   Code   RO          539    i.Idd_Sleep_process  power.o
    0x08003094   0x0000002c   Code   RO          780    i.IntToUnicode      usbd_desc.o
    0x080030c0   0x000004dc   Code   RO          276    i.Menu_Process      menu.o
    0x0800359c   0x00000002   Code   RO          470    i.MyLinRots_ErrorStateProcess  tsl_user.o
    0x0800359e   0x00000002   Code   RO          471    i.MyLinRots_OffStateProcess  tsl_user.o
    0x080035a0   0x00000002   Code   RO          401    i.NMI_Handler       stm32l0xx_it.o
    0x080035a2   0x00000002   PAD
    0x080035a4   0x00000044   Code   RO         1429    i.NVIC_SetPriority  stm32l0xx_hal_cortex.o
    0x080035e8   0x00000338   Code   RO         2233    i.PCD_EP_ISR_Handler  stm32l0xx_hal_pcd.o
    0x08003920   0x0000001e   Code   RO         2234    i.PCD_ReadPMA       stm32l0xx_hal_pcd.o
    0x0800393e   0x00000026   Code   RO         2235    i.PCD_WritePMA      stm32l0xx_hal_pcd.o
    0x08003964   0x00000002   Code   RO          402    i.PendSV_Handler    stm32l0xx_it.o
    0x08003966   0x000000b2   Code   RO         2779    i.SPI_WaitOnFlagUntilTimeout  stm32l0xx_hal_spi.o
    0x08003a18   0x00000014   Code   RO          971    i.SPIx_Error        stm32l0538_discovery.o
    0x08003a2c   0x0000008c   Code   RO          972    i.SPIx_Init         stm32l0538_discovery.o
    0x08003ab8   0x00000020   Code   RO          973    i.SPIx_Write        stm32l0538_discovery.o
    0x08003ad8   0x00000002   Code   RO          403    i.SVC_Handler       stm32l0xx_it.o
    0x08003ada   0x0000000a   Code   RO         3150    i.SoftDelay         tsl_acq_tsc.o
    0x08003ae4   0x00000034   Code   RO          404    i.SysTick_Handler   stm32l0xx_it.o
    0x08003b18   0x00000058   Code   RO          277    i.SystemClock_Config  menu.o
    0x08003b70   0x00000054   Code   RO         1197    i.SystemInit        system_stm32l0xx.o
    0x08003bc4   0x00000024   Code   RO         2993    i.TSC_extract_groups  stm32l0xx_hal_tsc.o
    0x08003be8   0x00000030   Code   RO         3097    i.TSL_Init          tsl.o
    0x08003c18   0x00000064   Code   RO         3151    i.TSL_acq_BankConfig  tsl_acq_tsc.o
    0x08003c7c   0x0000012c   Code   RO         3119    i.TSL_acq_BankGetResult  tsl_acq.o
    0x08003da8   0x00000030   Code   RO         3152    i.TSL_acq_BankStartAcq  tsl_acq_tsc.o
    0x08003dd8   0x00000024   Code   RO         3153    i.TSL_acq_BankWaitEOC  tsl_acq_tsc.o
    0x08003dfc   0x00000004   Code   RO         3154    i.TSL_acq_CheckNoise  tsl_acq_tsc.o
    0x08003e00   0x00000006   Code   RO         3155    i.TSL_acq_ComputeDelta  tsl_acq_tsc.o
    0x08003e06   0x00000006   Code   RO         3156    i.TSL_acq_ComputeMeas  tsl_acq_tsc.o
    0x08003e0c   0x00000018   Code   RO         3157    i.TSL_acq_GetMeas   tsl_acq_tsc.o
    0x08003e24   0x00000004   Code   RO         3158    i.TSL_acq_TestFirstReferenceIsValid  tsl_acq_tsc.o
    0x08003e28   0x00000004   Code   RO         3159    i.TSL_acq_TestReferenceOutOfRange  tsl_acq_tsc.o
    0x08003e2c   0x00000004   Code   RO         3160    i.TSL_acq_UseFilter  tsl_acq_tsc.o
    0x08003e30   0x00000002   Code   RO         3229    i.TSL_dxs_FirstObj  tsl_dxs.o
    0x08003e32   0x00000002   PAD
    0x08003e34   0x000000ac   Code   RO         3249    i.TSL_ecs_CalcK     tsl_ecs.o
    0x08003ee0   0x00000080   Code   RO         3250    i.TSL_ecs_Process   tsl_ecs.o
    0x08003f60   0x000000c0   Code   RO         3251    i.TSL_ecs_ProcessK  tsl_ecs.o
    0x08004020   0x00000294   Code   RO         3328    i.TSL_linrot_CalcPos  tsl_linrot.o
    0x080042b4   0x000000c8   Code   RO         3329    i.TSL_linrot_CalibrationStateProcess  tsl_linrot.o
    0x0800437c   0x00000034   Code   RO         3330    i.TSL_linrot_DTOGetTime  tsl_linrot.o
    0x080043b0   0x00000048   Code   RO         3331    i.TSL_linrot_DebCalibrationStateProcess  tsl_linrot.o
    0x080043f8   0x00000078   Code   RO         3332    i.TSL_linrot_DebDetectStateProcess  tsl_linrot.o
    0x08004470   0x0000006c   Code   RO         3333    i.TSL_linrot_DebErrorStateProcess  tsl_linrot.o
    0x080044dc   0x00000078   Code   RO         3334    i.TSL_linrot_DebProxDetectStateProcess  tsl_linrot.o
    0x08004554   0x00000078   Code   RO         3335    i.TSL_linrot_DebProxStateProcess  tsl_linrot.o
    0x080045cc   0x00000078   Code   RO         3336    i.TSL_linrot_DebProxTouchStateProcess  tsl_linrot.o
    0x08004644   0x0000005c   Code   RO         3337    i.TSL_linrot_DebReleaseDetectStateProcess  tsl_linrot.o
    0x080046a0   0x00000048   Code   RO         3338    i.TSL_linrot_DebReleaseProxStateProcess  tsl_linrot.o
    0x080046e8   0x0000005c   Code   RO         3339    i.TSL_linrot_DebReleaseTouchStateProcess  tsl_linrot.o
    0x08004744   0x000000d0   Code   RO         3340    i.TSL_linrot_DetectStateProcess  tsl_linrot.o
    0x08004814   0x00000024   Code   RO         3342    i.TSL_linrot_GetStateMask  tsl_linrot.o
    0x08004838   0x00000070   Code   RO         3343    i.TSL_linrot_Init   tsl_linrot.o
    0x080048a8   0x00000050   Code   RO         3346    i.TSL_linrot_Process  tsl_linrot.o
    0x080048f8   0x00000028   Code   RO         3348    i.TSL_linrot_ProcessCh_All_ClearRef  tsl_linrot.o
    0x08004920   0x0000002c   Code   RO         3349    i.TSL_linrot_ProcessCh_All_DeltaBelowEqu  tsl_linrot.o
    0x0800494c   0x00000030   Code   RO         3350    i.TSL_linrot_ProcessCh_All_SetStatus  tsl_linrot.o
    0x0800497c   0x0000002c   Code   RO         3351    i.TSL_linrot_ProcessCh_One_AcqStatusError  tsl_linrot.o
    0x080049a8   0x00000030   Code   RO         3352    i.TSL_linrot_ProcessCh_One_DataReady  tsl_linrot.o
    0x080049d8   0x0000002c   Code   RO         3353    i.TSL_linrot_ProcessCh_One_DeltaAbove  tsl_linrot.o
    0x08004a04   0x0000002c   Code   RO         3354    i.TSL_linrot_ProcessCh_One_DeltaAboveEqu  tsl_linrot.o
    0x08004a30   0x00000030   Code   RO         3355    i.TSL_linrot_ProcessCh_One_DeltaBelowEquMinus  tsl_linrot.o
    0x08004a60   0x000000b0   Code   RO         3356    i.TSL_linrot_ProxStateProcess  tsl_linrot.o
    0x08004b10   0x000000b0   Code   RO         3357    i.TSL_linrot_ReleaseStateProcess  tsl_linrot.o
    0x08004bc0   0x0000005c   Code   RO         3359    i.TSL_linrot_SetStateCalibration  tsl_linrot.o
    0x08004c1c   0x000000d0   Code   RO         3361    i.TSL_linrot_TouchStateProcess  tsl_linrot.o
    0x08004cec   0x0000005c   Code   RO         3556    i.TSL_obj_GroupInit  tsl_object.o
    0x08004d48   0x0000005c   Code   RO         3557    i.TSL_obj_GroupProcess  tsl_object.o
    0x08004da4   0x00000020   Code   RO         3558    i.TSL_obj_SetGlobalObj  tsl_object.o
    0x08004dc4   0x00000058   Code   RO         3588    i.TSL_tim_CheckDelay_ms  tsl_time.o
    0x08004e1c   0x00000058   Code   RO         3589    i.TSL_tim_CheckDelay_sec  tsl_time.o
    0x08004e74   0x00000024   Code   RO          278    i.USBClock_Disable  menu.o
    0x08004e98   0x00000054   Code   RO          279    i.USBClock_Enable   menu.o
    0x08004eec   0x00000010   Code   RO         3698    i.USBD_ClrClassConfig  usbd_core.o
    0x08004efc   0x00000010   Code   RO         3893    i.USBD_CtlContinueRx  usbd_ioreq.o
    0x08004f0c   0x00000010   Code   RO         3894    i.USBD_CtlContinueSendData  usbd_ioreq.o
    0x08004f1c   0x00000014   Code   RO         3832    i.USBD_CtlError     usbd_ctlreq.o
    0x08004f30   0x00000018   Code   RO         3896    i.USBD_CtlReceiveStatus  usbd_ioreq.o
    0x08004f48   0x0000001c   Code   RO         3897    i.USBD_CtlSendData  usbd_ioreq.o
    0x08004f64   0x00000018   Code   RO         3898    i.USBD_CtlSendStatus  usbd_ioreq.o
    0x08004f7c   0x0000002a   Code   RO         3699    i.USBD_DeInit       usbd_core.o
    0x08004fa6   0x000000e0   Code   RO         3833    i.USBD_GetDescriptor  usbd_ctlreq.o
    0x08005086   0x00000044   Code   RO         3834    i.USBD_GetString    usbd_ctlreq.o
    0x080050ca   0x00000002   PAD
    0x080050cc   0x00000020   Code   RO          781    i.USBD_HID_ConfigStrDescriptor  usbd_desc.o
    0x080050ec   0x00000010   Code   RO         3635    i.USBD_HID_DataIn   usbd_hid.o
    0x080050fc   0x00000022   Code   RO         3636    i.USBD_HID_DeInit   usbd_hid.o
    0x0800511e   0x00000002   PAD
    0x08005120   0x0000000c   Code   RO          782    i.USBD_HID_DeviceDescriptor  usbd_desc.o
    0x0800512c   0x0000000c   Code   RO         3637    i.USBD_HID_GetCfgDesc  usbd_hid.o
    0x08005138   0x0000000c   Code   RO         3638    i.USBD_HID_GetDeviceQualifierDesc  usbd_hid.o
    0x08005144   0x0000002e   Code   RO         3640    i.USBD_HID_Init     usbd_hid.o
    0x08005172   0x00000002   PAD
    0x08005174   0x00000024   Code   RO          783    i.USBD_HID_InterfaceStrDescriptor  usbd_desc.o
    0x08005198   0x0000000c   Code   RO          784    i.USBD_HID_LangIDStrDescriptor  usbd_desc.o
    0x080051a4   0x00000028   Code   RO          785    i.USBD_HID_ManufacturerStrDescriptor  usbd_desc.o
    0x080051cc   0x0000002c   Code   RO          786    i.USBD_HID_ProductStrDescriptor  usbd_desc.o
    0x080051f8   0x0000002a   Code   RO         3641    i.USBD_HID_SendReport  usbd_hid.o
    0x08005222   0x00000002   PAD
    0x08005224   0x00000034   Code   RO          787    i.USBD_HID_SerialStrDescriptor  usbd_desc.o
    0x08005258   0x000000a0   Code   RO         3642    i.USBD_HID_Setup    usbd_hid.o
    0x080052f8   0x00000032   Code   RO         3700    i.USBD_Init         usbd_core.o
    0x0800532a   0x00000012   Code   RO          596    i.USBD_LL_ClearStallEP  usbd_conf.o
    0x0800533c   0x00000012   Code   RO          597    i.USBD_LL_CloseEP   usbd_conf.o
    0x0800534e   0x000000aa   Code   RO         3701    i.USBD_LL_DataInStage  usbd_core.o
    0x080053f8   0x00000074   Code   RO         3702    i.USBD_LL_DataOutStage  usbd_core.o
    0x0800546c   0x00000012   Code   RO          598    i.USBD_LL_DeInit    usbd_conf.o
    0x0800547e   0x00000002   PAD
    0x08005480   0x0000005c   Code   RO          602    i.USBD_LL_Init      usbd_conf.o
    0x080054dc   0x00000024   Code   RO          603    i.USBD_LL_IsStallEP  usbd_conf.o
    0x08005500   0x00000018   Code   RO          604    i.USBD_LL_OpenEP    usbd_conf.o
    0x08005518   0x00000012   Code   RO          605    i.USBD_LL_PrepareReceive  usbd_conf.o
    0x0800552a   0x00000046   Code   RO         3707    i.USBD_LL_Reset     usbd_core.o
    0x08005570   0x0000001e   Code   RO         3709    i.USBD_LL_SOF       usbd_core.o
    0x0800558e   0x00000006   Code   RO         3710    i.USBD_LL_SetSpeed  usbd_core.o
    0x08005594   0x00000012   Code   RO          606    i.USBD_LL_SetUSBAddress  usbd_conf.o
    0x080055a6   0x0000005e   Code   RO         3711    i.USBD_LL_SetupStage  usbd_core.o
    0x08005604   0x00000012   Code   RO          607    i.USBD_LL_StallEP   usbd_conf.o
    0x08005616   0x00000012   Code   RO          608    i.USBD_LL_Start     usbd_conf.o
    0x08005628   0x00000012   Code   RO          609    i.USBD_LL_Stop      usbd_conf.o
    0x0800563a   0x00000012   Code   RO          610    i.USBD_LL_Transmit  usbd_conf.o
    0x0800564c   0x00000028   Code   RO         3835    i.USBD_ParseSetupRequest  usbd_ctlreq.o
    0x08005674   0x00000016   Code   RO         3713    i.USBD_RegisterClass  usbd_core.o
    0x0800568a   0x0000001c   Code   RO         3715    i.USBD_SetClassConfig  usbd_core.o
    0x080056a6   0x00000002   PAD
    0x080056a8   0x00000070   Code   RO         3836    i.USBD_SetConfig    usbd_ctlreq.o
    0x08005718   0x0000000a   Code   RO         3716    i.USBD_Start        usbd_core.o
    0x08005722   0x000000ee   Code   RO         3837    i.USBD_StdDevReq    usbd_ctlreq.o
    0x08005810   0x000000d0   Code   RO         3838    i.USBD_StdEPReq     usbd_ctlreq.o
    0x080058e0   0x0000003a   Code   RO         3839    i.USBD_StdItfReq    usbd_ctlreq.o
    0x0800591a   0x00000002   Code   RO          611    i.USBD_static_free  usbd_conf.o
    0x0800591c   0x00000008   Code   RO          612    i.USBD_static_malloc  usbd_conf.o
    0x08005924   0x00000010   Code   RO          405    i.USB_IRQHandler    stm32l0xx_it.o
    0x08005934   0x0000003c   Code   RO          851    i.USB_process       usbdapp.o
    0x08005970   0x00000028   Code   RO         4001    i.__0sprintf$1      mc_p.l(printf1.o)
    0x08005998   0x0000001a   Code   RO          327    i.__ARM_common_switch8  menu.o
    0x080059b2   0x0000000e   Code   RO         4261    i.__scatterload_copy  mc_p.l(handlers.o)
    0x080059c0   0x00000002   Code   RO         4262    i.__scatterload_null  mc_p.l(handlers.o)
    0x080059c2   0x0000000e   Code   RO         4263    i.__scatterload_zeroinit  mc_p.l(handlers.o)
    0x080059d0   0x00000150   Code   RO         4006    i._printf_core      mc_p.l(printf1.o)
    0x08005b20   0x0000000a   Code   RO         4008    i._sputc            mc_p.l(printf1.o)
    0x08005b2a   0x00000016   Code   RO          881    i.gde021a1_CloseChargePump  gde021a1.o
    0x08005b40   0x0000014a   Code   RO          882    i.gde021a1_DrawImage  gde021a1.o
    0x08005c8a   0x00000004   Code   RO          883    i.gde021a1_GetEpdPixelHeight  gde021a1.o
    0x08005c8e   0x00000004   Code   RO          884    i.gde021a1_GetEpdPixelWidth  gde021a1.o
    0x08005c92   0x00000002   PAD
    0x08005c94   0x000000a8   Code   RO          885    i.gde021a1_Init     gde021a1.o
    0x08005d3c   0x00000016   Code   RO          887    i.gde021a1_RefreshDisplay  gde021a1.o
    0x08005d52   0x00000048   Code   RO          888    i.gde021a1_SetDisplayWindow  gde021a1.o
    0x08005d9a   0x00000012   Code   RO          889    i.gde021a1_WritePixel  gde021a1.o
    0x08005dac   0x00000012   Code   RO          253    i.main              main.o
    0x08005dbe   0x00000002   PAD
    0x08005dc0   0x0000007c   Code   RO          472    i.tsl_user_Exec     tsl_user.o
    0x08005e3c   0x00000018   Code   RO          473    i.tsl_user_Init     tsl_user.o
    0x08005e54   0x00000024   Data   RO          477    .constdata          tsl_user.o
    0x08005e78   0x00000006   Data   RO          478    .constdata          tsl_user.o
    0x08005e7e   0x00000002   PAD
    0x08005e80   0x00000018   Data   RO          479    .constdata          tsl_user.o
    0x08005e98   0x000000a0   Data   RO          480    .constdata          tsl_user.o
    0x08005f38   0x0000000c   Data   RO          481    .constdata          tsl_user.o
    0x08005f44   0x00000006   Data   RO          482    .constdata          tsl_user.o
    0x08005f4a   0x00000002   PAD
    0x08005f4c   0x00000024   Data   RO          483    .constdata          tsl_user.o
    0x08005f70   0x00000008   Data   RO          484    .constdata          tsl_user.o
    0x08005f78   0x00000016   Data   RO          789    .constdata          usbd_desc.o
    0x08005f8e   0x0000005a   Data   RO          891    .constdata          gde021a1.o
    0x08005fe8   0x00000008   Data   RO          975    .constdata          stm32l0538_discovery.o
    0x08005ff0   0x00001054   Data   RO         1082    .constdata          stm32l0538_discovery_epd.o
    0x08007044   0x000007cb   Data   RO         1083    .constdata          stm32l0538_discovery_epd.o
    0x0800780f   0x000003b6   Data   RO         1084    .constdata          stm32l0538_discovery_epd.o
    0x08007bc5   0x00000003   PAD
    0x08007bc8   0x0000001c   Data   RO         2596    .constdata          stm32l0xx_hal_rcc.o
    0x08007be4   0x00000012   Data   RO         3362    .constdata          tsl_linrot.o
    0x08007bf6   0x00000002   PAD
    0x08007bf8   0x00000020   Data   RO         4259    Region$$Table       anon$$obj.o


    Execution Region RW_IRAM1 (Base: 0x20000000, Size: 0x00001898, Max: 0x00002000, ABSOLUTE, COMPRESSED[0x000002ec])

    Base Addr    Size         Type   Attr      Idx    E Section Name        Object

    0x20000000   0x000008c0   Data   RW          281    .data               menu.o
    0x200008c0   0x00000004   Data   RW          406    .data               stm32l0xx_it.o
    0x200008c4   0x0000001c   Data   RW          485    .data               tsl_user.o
    0x200008e0   0x00000010   Data   RW          486    .data               tsl_user.o
    0x200008f0   0x00000008   Data   RW          487    .data               tsl_user.o
    0x200008f8   0x0000000c   Data   RW          542    .data               power.o
    0x20000904   0x0000001c   Data   RW          790    .data               usbd_desc.o
    0x20000920   0x0000001a   Data   RW          791    .data               usbd_desc.o
    0x2000093a   0x00000004   Data   RW          852    .data               usbdapp.o
    0x2000093e   0x00000002   PAD
    0x20000940   0x00000020   Data   RW          892    .data               gde021a1.o
    0x20000960   0x0000000c   Data   RW          976    .data               stm32l0538_discovery.o
    0x2000096c   0x00000018   Data   RW         1086    .data               stm32l0538_discovery_epd.o
    0x20000984   0x00000008   Data   RW         1087    .data               stm32l0538_discovery_epd.o
    0x2000098c   0x0000001d   Data   RW         1198    .data               system_stm32l0xx.o
    0x200009a9   0x00000003   PAD
    0x200009ac   0x00000004   Data   RW         1257    .data               stm32l0xx_hal.o
    0x200009b0   0x00000019   Data   RW         2597    .data               stm32l0xx_hal_rcc.o
    0x200009c9   0x00000001   PAD
    0x200009ca   0x0000000a   Data   RW         3363    .data               tsl_linrot.o
    0x200009d4   0x00000038   Data   RW         3643    .data               usbd_hid.o
    0x20000a0c   0x00000086   Data   RW         3644    .data               usbd_hid.o
    0x20000a92   0x00000001   Data   RW         3840    .data               usbd_ctlreq.o
    0x20000a93   0x00000001   PAD
    0x20000a94   0x00000264   Zero   RW           15    .bss                bsp.o
    0x20000cf8   0x00000018   Zero   RW          280    .bss                menu.o
    0x20000d10   0x00000024   Zero   RW          475    .bss                tsl_user.o
    0x20000d34   0x0000000d   Zero   RW          476    .bss                tsl_user.o
    0x20000d41   0x00000003   PAD
    0x20000d44   0x00000060   Zero   RW          541    .bss                power.o
    0x20000da4   0x00000188   Zero   RW          613    .bss                usbd_conf.o
    0x20000f2c   0x00000100   Zero   RW          788    .bss                usbd_desc.o
    0x2000102c   0x00000054   Zero   RW          974    .bss                stm32l0538_discovery.o
    0x20001080   0x00000018   Zero   RW         3307    .bss                tsl_globals.o
    0x20001098   0x00000800   Zero   RW            1    STACK               startup_stm32l053xx.o


==============================================================================

Image component sizes


      Code (inc. data)   RO Data    RW Data    ZI Data      Debug   Object Name

       148         20          0          0        612     225621   bsp.o
       640          4         90         32          0       6803   gde021a1.o
        18          0          0          0          0        475   main.o
      2046        560          0       2240         24       7651   menu.o
      1732        126          0         12         96       4712   power.o
        32         10        192          0       2048        708   startup_stm32l053xx.o
       744         94          8         12         84       8555   stm32l0538_discovery.o
       648         68       7125         32          0      11547   stm32l0538_discovery_epd.o
       156         26          0          4          0       4981   stm32l0xx_hal.o
       164         30          0          0          0      10747   stm32l0xx_hal_cortex.o
       562         44          0          0          0       5257   stm32l0xx_hal_gpio.o
      1408         26          0          0          0       9695   stm32l0xx_hal_i2c.o
       370         36          0          0          0       3218   stm32l0xx_hal_msp.o
      3364        146          0          0          0      13296   stm32l0xx_hal_pcd.o
        56          0          0          0          0       1198   stm32l0xx_hal_pcd_ex.o
        48         10          0          0          0        637   stm32l0xx_hal_pwr.o
        32          8          0          0          0       1145   stm32l0xx_hal_pwr_ex.o
      1640         80         28         25          0       5406   stm32l0xx_hal_rcc.o
       440         22          0          0          0       2086   stm32l0xx_hal_rcc_ex.o
       694          0          0          0          0       5404   stm32l0xx_hal_spi.o
       230          0          0          0          0       2484   stm32l0xx_hal_tsc.o
       100         16          0          4          0       4286   stm32l0xx_it.o
        84         18          0         29          0       1281   system_stm32l0xx.o
        48         14          0          0          0       1051   tsl.o
       300         10          0          0          0       1552   tsl_acq.o
       246         28          0          0          0       7464   tsl_acq_tsc.o
         2          0          0          0          0       1511   tsl_dxs.o
       492         20          0          0          0       3773   tsl_ecs.o
         0          0          0          0         24       1135   tsl_globals.o
      3276        184         18         10          0      23805   tsl_linrot.o
       216         12          0          0          0       2562   tsl_object.o
       176         18          0          0          0       2105   tsl_time.o
       152         14        288         52         49       5533   tsl_user.o
       572         22          0          0        392      13339   usbd_conf.o
       654          0          0          0          0       8639   usbd_core.o
       968         34          0          1          0       7004   usbd_ctlreq.o
       272        104         22         54        256       5870   usbd_desc.o
       322         14          0        190          0       6709   usbd_hid.o
       108          0          0          0          0       3720   usbd_ioreq.o
       116         16          0          4          0       1806   usbdapp.o

    ----------------------------------------------------------------------
     23312       1834       7812       2708       3588     434771   Object Totals
         0          0         32          0          0          0   (incl. Generated)
        36          0          9          7          3          0   (incl. Padding)

    ----------------------------------------------------------------------

      Code (inc. data)   RO Data    RW Data    ZI Data      Debug   Library Member Name

        86          0          0          0          0          0   __dczerorl2.o
         0          0          0          0          0          0   entry.o
         0          0          0          0          0          0   entry10a.o
         0          0          0          0          0          0   entry11a.o
         8          4          0          0          0          0   entry2.o
         4          0          0          0          0          0   entry5.o
         0          0          0          0          0          0   entry7b.o
         0          0          0          0          0          0   entry8b.o
         8          4          0          0          0          0   entry9a.o
        30          0          0          0          0          0   handlers.o
        40          0          0          0          0         72   idiv.o
        36          8          0          0          0         68   init.o
       386          8          0          0          0        228   printf1.o
        44          0          0          0          0         72   uidiv.o

    ----------------------------------------------------------------------
       644         24          0          0          0        440   Library Totals
         2          0          0          0          0          0   (incl. Padding)

    ----------------------------------------------------------------------

      Code (inc. data)   RO Data    RW Data    ZI Data      Debug   Library Name

       642         24          0          0          0        440   mc_p.l

    ----------------------------------------------------------------------
       644         24          0          0          0        440   Library Totals

    ----------------------------------------------------------------------

==============================================================================


      Code (inc. data)   RO Data    RW Data    ZI Data      Debug   

     23956       1858       7812       2708       3588     424699   Grand Totals
     23956       1858       7812        748       3588     424699   ELF Image Totals (compressed)
     23956       1858       7812        748          0          0   ROM Totals

==============================================================================

    Total RO  Size (Code + RO Data)                31768 (  31.02kB)
    Total RW  Size (RW Data + ZI Data)              6296 (   6.15kB)
    Total ROM Size (Code + RO Data + RW Data)      32516 (  31.75kB)

==============================================================================

